:020000040000FA
:040000006FD00400B9
:101000006F00907E00000000000000009020002093
:10101000AA220020A9BDF9F56C23002000000000E1
:10102000000000006C230020902000200000000041
:101030000000000090200020000000009020002010
:101040000000000090200020902000209020002030
:101050009020002090200020582F00209424002071
:101060000000000090200020902000201E2400207E
:1010700090200020D22300209020002090200020EB
:101080009020002090200020902000209020002020
:101090009020002001A04111B7170040985F3AC688
:1010A000945F3247E39CE6FE3245410182800111A4
:1010B00013078008F337078093F787083EC20100C3
:1010C0000100B7170040930570052380B70413068D
:1010D00080FA2380C7040100010083C6B70493F699
:1010E000F60DA385D704238007049246F3A6068055
:1010F0000100010093760502D5CEF336078093F602
:10110000860836C4010001002380B7042380C70489
:1011100001000100B70614007D89558D88C70100C4
:1011200001000100010023800704A246F3A6068007
:101130000100010073370780137787083AC6010062
:1011400001002380B7042380C704010001000100CF
:1011500001003727004093061005A303D7802380A2
:101160000704B247F3A70780010001009307800836
:10117000F3B7078093F787083ECE01000100B71749
:101180000040130770052380E704130780FA2380CB
:10119000E7040100010003C7B70413670708A3852C
:1011A000E70423800704F247F3A70780010001004A
:1011B0000561828093760504BDC6F336078093F6F9
:1011C000860836C8010001002380B7042380C704C5
:1011D00001000100B7061400938606047D89558D31
:1011E00088C7010001000100010023800704C246F6
:1011F000F3A6068001000100733707801377870884
:101200003ACA010001002380B7042380C70401000B
:1012100001003727004093062005A303D7802380D1
:101220000704D24781B773370780137787083ACC12
:10123000010001002380B7042380C70401000100DE
:1012400098471367070C98C723800704E24719BF24
:101250000111814601468145114506CE97000000E7
:10126000E780605893078008F3B7078093F78708F3
:101270003EC601000100B717004013077005238028
:10128000E704130780FA2380E7040100010003C785
:101290006704136717002383E70423800704B2471A
:1012A000F3A7078001000100F2400561828041112F
:1012B000814601468145114597000000E780A05214
:1012C00013078008F337078093F787083EC40100AF
:1012D0000100B7170040130670052380C70493066A
:1012E00080FA2380D70401000100FD552396B70240
:1012F00023800704A245F3A5058001000100733790
:101300000780137787083AC6010001002380C704CD
:101310002380D7040100010003C767041367170087
:101320002383E70423800704B247F3A70780010063
:10133000010001A0BD473305F50201007D1575FDD3
:101340008280411122C426C206C6AA8401446317C2
:101350009400B24022449244410182800504130566
:10136000803E420497000000E78000FD4180C5B741
:101370009305000273A04580824573901534924016
:101380002242B2424243D2436244F2440255925551
:101390002256B2564257D2576258F25806499649D9
:1013A000264AB64A464BD64B664CF64C065D965DD1
:1013B000265EB65E465FD65F09617300203041113C
:1013C000B7170040985F3AC6945F3247E39CE6FE49
:1013D000324541018280B71700401307000323887C
:1013E000E702854717170000232EF74673002030C9
:1013F000411122C42D6426C24AC006C637190040D6
:101400001304A4AAB704002023208900977000E0E9
:10141000E78040929C408297977000E0E78080913F
:10142000E5B737370040834747009146BD8B639E41
:10143000D702B73600401306F00F973500009385AA
:10144000E5209737000083D7673003C7A6001377DE
:10145000F70F1DE3B7E70400BC4F09468945171590
:1014600000000345A5F7829731A099466394D70001
:10147000834757007300203003C786001377F70FA8
:10148000E365F6FC13851700AE9717380000231F9D
:10149000A82A2380E70075B7B787004003C7670015
:1014A000098B6309071003C77700930600031377BE
:1014B0000703630DD708173800000348787A1736FA
:1014C00000001306E6760547B30606012380E60012
:1014D00083C577001737000013078777429793F586
:1014E000F50F2300B70003C58700973500009385EB
:1014F0002575C2951375F50F2380A50003470700D6
:1015000089451377F703630CB70C63E7E50A6306B5
:10151000071A8545630CB7129737000083C75774C5
:101520003307F600034707001377F70F19CB85073A
:1015300093F7F70F3D476363F71A17370000A301CE
:10154000F772B787004009472383E700B787004059
:1015500083C77700E207E18763DE0704973700005F
:1015600083C71770173700001307876C3E978546AF
:101570002300D700173700001307876D3E979306A7
:1015800000032300D700173700001307676B3E974F
:10159000A14685072300D70093F7F70F3D47636403
:1015A000F71417370000A30DF76AB7870040094703
:1015B0002383E70073002030930610026300D70EE8
:1015C000930620026305D70693060002E316D7F4BC
:1015D00003C727021377C70F13672700D5A803C7D0
:1015E00067001377070465CB03C7A702173800000D
:1015F00013088845173500001305C53C1347070835
:101600002385E70203C7A7021377370F1367870005
:101610002385E702814713070004B305F5008C41D9
:10162000B306F80091078CC2E399E7FEF5B503C74E
:10163000A702134707042385E70203C7A70213770E
:10164000C70F136727002385E702F9B503C76700B3
:101650001377070449C303C767021738000013084C
:101660006832173500001305A5291347070823839F
:10167000E70203C767021377370F136787002383D7
:10168000E702814713070004B305F5008C41B30658
:10169000F80091078CC2E399E7FEBDBD03C767025E
:1016A000134707042383E70203C767021377C70FB3
:1016B000136727002383E70285B503C76700137705
:1016C000070411CB03C727021377370F136787006F
:1016D0002381E70291B5238006003DBD97370000C6
:1016E000A3800758B9BD97370000A38B075675BD77
:1016F0002303048015472303E48001002302A48010
:10170000828083076480E3CE07FE23030480828007
:1017100083076480E3CE07FE03454480828083070D
:101720006480E3CE07FE2302A4808280411126C498
:101730004AC24EC006C61377F50BAD47AA892E895B
:101740009544630CF700194597000000E78080FA84
:1017500097000000E78020FB8D444E859700000035
:10176000E78040F9FD59FD1463983401B240A2446A
:101770001249824941018280135509011375F50F01
:1017800097000000E780E0F92209F1BF011126CCA3
:1017900006CEB704080097000000E780C0F61545A4
:1017A00097000000E78000F597000000E78080F6D2
:1017B00097000000E78000F62AC697000000E78047
:1017C00080F432459377150089EB13651500137586
:1017D000F50FF240E24405618280FD14E9F0014515
:1017E000CDBF397126DC4ADA4ED852D656D45AD2F9
:1017F0005ED006DE62CE66CCB7E700E07D5783AAF6
:10180000070022C603AA470023A0E71823A2E7186F
:10181000B7170040130770052380E704130780FA09
:101820002380E70483C74704930B75FFB684E20760
:1018300093FBFB0F8546AA892E8B32893724004003
:10184000E187015763FA76016308D50089461307DB
:1018500000026313D5000157D98F93F7F70FB71C18
:1018600000402382FC0411472303E4801305F00F9A
:1018700097000000E78000E8094C97000000E7802F
:1018800080E863657C15B7050700DA9537870700A0
:10189000795563FEE504B3879500636AF704370B57
:1018A0000800A94733EB65016395F90881E8814495
:1018B00097000000E78020E5268515A8DA85094510
:1018C00097000000E780C0E605090345F9FFFD1415
:1018D000050B97000000E780C0E481C49377FB0FFD
:1018E000E5F797000000E780A0EA69F17D55B7179A
:1018F0000040130770052380E704130780FA238054
:10190000E70403C74704418B2382E704F250B7E79B
:1019100000E023A0571123A24711E2543244525948
:10192000C259325AA25A125B825B724CE24C21615C
:101930008280A547639BF90685691309F00FB306FA
:101940009900B3742B01B6941349F9FFB37499004D
:10195000856B33796901416B9387F9FFB3F72701F1
:1019600099E363FC340193D94900C147E3E637FFAB
:101970003DBF0569C1697D19D9B71305800D63881D
:101980006901130500026384790113051008CA85F3
:1019900097000000E780C0D997000000E78040DF93
:1019A00031D54E99B38434416DBFDA852D4597000A
:1019B0000000E780E0D7CA94E30B99EE0509970091
:1019C0000000E78020D5A30FA9FEFDB79387F9FF9C
:1019D00093F7F70F636DFC0C83C71C0413073008E3
:1019E0006315F706370708006361EB06B3079B0032
:1019F000B706100063FBD704334BEB0089476399AC
:101A0000F9068980D549E38404EADA850945970017
:101A10000000E780E0D111090327C9FF9147232087
:101A2000E48003076480E34E07FE23033481FD173F
:101A3000EDFBFD14110B81C49377FB0FE9FF9700B9
:101A40000000E780E0D461F155B5B717004003C747
:101A50005704B70708001377070219E3B787070091
:101A60007955E376FBE833079B00E3F9E7F841B5E6
:101A70008547E380F9F0DA852D4597000000E7807F
:101A800020CB9389F4FFE38404E297000000E78011
:101A900060C893F7390091EB83260480032709007F
:101AA00093074900E396E6E03E89CE84D9BFB54767
:101AB0006399F9001305900B97000000E78080C33D
:101AC000FDB3B1471305B00AE388F9FE9947639760
:101AD000F904B7050800B365BB002D459700000069
:101AE000E78000C581448D4BA14997000000E78045
:101AF00060C263967401832704802320F900850463
:101B0000E39534FF8327048013172B0163550700E7
:101B10002312F90069BB2322F90051BB9D47639F43
:101B2000F90281451305B00497000000E78040C02A
:101B3000BD442320090023220900FD59970000001D
:101B4000E78040BD93F77400CA9703C70700FD14F0
:101B5000398D2380A700E39334FF91BBA14763979E
:101B6000F90697000000E780A0C28144630D0B00D6
:101B70008D479304C0036308FB00930400056304CE
:101B80008B01930440041375C507E30295D21945F0
:101B900097000000E78000B697000000E780A0B63D
:101BA000054597000000E780E0B426859700000017
:101BB000E78020B7094597000000E78080B69700CE
:101BC0000000E780E0BCE31405CE0DB39147639FAE
:101BD000F9001305600697000000E780A0B19700A8
:101BE0000000E78040B213059009F9B5E38109CC04
:101BF000F1547DB9BD6601471736000013068632E1
:101C0000938606A685458347060093F7F70F91C391
:101C100082800507E3F9E6FE973700002384B7309A
:101C2000DDB77D166206618693178601E18763D46E
:101C3000070001458280931726003307F500AE9711
:101C400018439C4363E7E7007D16E37FF7FC7D556F
:101C5000828005458280FD15E205E18513978501A7
:101C6000618793F7F50F63480700FD15139725006B
:101C70002A97584365D713851700620561858280CE
:101C80003308B5021C4283A80600B335B502C297DB
:101C900033B50701AE98469585486367B5006394F0
:101CA000A50063E3070181480C43C6950CC388C2B5
:101CB0001CC2828081471397870161876343B70005
:101CC0008280139727002A97232007008507E5B70E
:101CD0008147014793968701E18663C5B6001335B6
:101CE0001700828093962700AA9694428507558F05
:101CF000D5B793D755408A07AA979C430545331516
:101D0000B5007D8D828017F3FFDFE702833D2A84D3
:101D100097000000E78060F405C5931725003E9406
:101D20000327C4FF814711EB7D1516053E9542053B
:101D3000418517F3FFDF6700033D05838507E5B79E
:101D40000145C5BF81471397870161876343C7007A
:101D5000828013972700B386E50094422A9785076F
:101D600014C3D5B77D1662066186014793178601B5
:101D7000E18763D50700133517008280931726008B
:101D8000B306F500AE9794429C437D16B58F5D8FE8
:101D9000F1BF8A05AA9501476363B500828083A6D7
:101DA000C5FFF11593D71600D98F9CC11397F60183
:101DB000E5B72A830148014701456343D700828084
:101DC000B387050183A80700B30706019C43C697A4
:101DD000AA976384F80033B517010507B308030118
:101DE000620723A0F80061871108C1BF2A83014759
:101DF0008147014563C3D70082803388E50083288B
:101E00000800330EE600032E0E003388A840330886
:101E1000C8416384080133B508018507B308E300AE
:101E2000E20723A00801E1871107E9B717F3FFDFF5
:101E3000E702232B0111B286B2842E86AA850A8579
:101E400097000000E780C0FA2A84A6850A859700DB
:101E50000000E78020E833348000060413351500C5
:101E6000018D056117F3FFDF6700E32917F3FFDF3B
:101E7000E702A3244111AA89AE8A328BB68402C23A
:101E800002C402C60144131C8401135C8C416349E3
:101E90009C02939B1400FD1B0549138CF4FFF15C1D
:101EA00033048901620461846340740792478E049D
:101EB000CE9423AEF4FE410117F3FFDF67006323E6
:101EC00013192400B30B2B01014A93172A00D6974C
:101ED00083A50B0088437800340050009700000071
:101EE000E78040DA050A93178A01E187F11BE35E78
:101EF000FCFC92474E9905042320F900A2473EC2FC
:101F0000B24702C63EC441B7131A8901135A8A4127
:101F1000131D240093178A01E18763CF970092472E
:101F20000A044E941CC0A24705091379F90F3EC25A
:101F3000B24702C63EC4ADB7B3079A0313152A00D1
:101F400056950841780034005000050AEA97DA9760
:101F50008C4397000000E780E0D26DBF197106C284
:101F600012C416C61AC81ECA22CC26CE2AD02ED219
:101F700032D436D63AD83EDA42DC46DECAC0CEC2C9
:101F8000D2C4D6C6DAC8DECAE2CCE6CEEAD0EED2F9
:101F9000F2D4F6D6FAD8FEDA971500009385058CB0
:101FA0008841E700050092402242B2424243D243B8
:101FB0006244F244025592552256B2564257D257C5
:101FC0006258F25806499649264AB64A464BD64BBD
:101FD000664CF64C065D965D265EB65E465FD65F45
:101FE0000961730020300000972100209381810156
:101FF000175100201301018117F5FFFF1305C500DC
:102000009705002093850500171600201306C6FDCE
:1020100063FAC5008322050023A055001105910530
:10202000E3EAC5FE170502001305454E971500208B
:102030009385C5FB171600201306C66563FAC50015
:102040008322050023A0550011059105E3EAC5FE92
:1020500017150020130505649745002093858538E2
:102060006377B500232005001105E36DB5FEFD4241
:10207000739002BC8D4273904280B722000093821D
:10208000828873900230970200209382A2F793E235
:1020900032007390523097520000938262C0739066
:1020A00012346FB0F47573002030397101436EC67D
:1020B00019A0397141536AC866CA62CC5ECE19A0B4
:1020C000397101535AD056D252D44ED64AD826DA54
:1020D00022DC06DE33016140828241114AC026C201
:1020E00022C406C68282B24D4101024D924C224C5E
:1020F000B24B4101024B924A224AB2494101024984
:1021000092442244B240410182803D432A87637356
:10211000C3029377F700BDEFADE5937606FF3D8AE6
:10212000BA960CC34CC30CC74CC74107E36BD7FE30
:1021300011E28280B306C3408A0697020000969699
:102140006780A6002307B700A306B7002306B700E1
:10215000A305B7002305B700A304B7002304B70005
:10216000A303B7002303B700A302B7002302B700FD
:10217000A301B7002301B700A300B7002300B700F5
:10218000828093F5F50F93968500D58D9396050182
:10219000D58D61B7939627009702000096968682A8
:1021A000E78086FA9680C1171D8F3E96E374C3F8C8
:1021B000A5B73367B500FD530D8B79E7B7877F7FF0
:1021C0009387F7F710419441B372F6003363F6003A
:1021D000BE92B3E262006397720C6318D606504158
:1021E000D441B372F6003363F600BE92B3E26200EC
:1021F0006398720A631BD60410459445B372F600C7
:102200003363F600BE92B3E262006391720A631E0A
:10221000D6025045D445B372F6003363F600BE9241
:10222000B3E26200639A72086311D60210499449BE
:10223000B372F6003363F600BE92B3E262006393BA
:1022400072085105D105E30FD6F6131706019397CF
:102250000601631CF7001357060193D706013305E7
:10226000F7409375F50F91E982804183C18333056F
:10227000F7409375F50F91E182801377F70F93F78D
:10228000F70F3305F74082800346050083C605003B
:10229000050585056313D60065FA3305D6408280AF
:1022A00011059105E312D6FE014582802105A105A5
:1022B000E31CD6FC014582803105B105E316D6FC4E
:1022C000014582804105C105E310D6FC01458280AD
:1022D000B717004003C777051377E70FA38BE70411
:1022E000130700F8A38DE7043D47238CE704130789
:1022F0005003A38CE70403C7A7051377D70F238DDB
:10230000E7048280B717004003C7E7020D89411137
:102310001377C70F498F93068008F3B6068093F6AC
:10232000860836C601000100930670052380D70495
:10233000930680FA2380D704010001002387E70277
:1023400023800704B247F3A7078001000100410181
:10235000828041112A83014E930E407E130F001993
:10236000930F400663E56E129308001913034006AD
:10237000B3781503854E0D4FA14F337365020D8958
:102380001335150063EFBE121308F6FF79467298F5
:102390004208135808013307C70213D61700BE07B7
:1023A00032976146B3F6C60213068070B386C60242
:1023B0003697A166F58F42075D8FB716004083C739
:1023C000F60293F70708A303F1000346710083C7E1
:1023D000F60293F70708E394C7FE83477100B71628
:1023E000004093F7F70F6388071293078008F3B74D
:1023F000078093F787083EC401000100B71700402B
:10240000930670052380D704930680FA2380D704AF
:102410000100010023AA070383C6170393E60608F9
:10242000A388D70223800704A247F3A707800100EF
:1024300001001166B71700407D16D45BC85F938515
:102440004703A98EF18EF5FA93068008F3B606804D
:1024500093F6860836C601000100930670052380B6
:10246000D704930680FA2380D7040100010098C1A5
:1024700003C7170313670704A388E7022380070431
:10248000B247F3A7078001000100410182807D135C
:102490003368E3039308E016630E08003368F30320
:1024A0009308D016630808009378330093B8180097
:1024B0009388D81633081E01131E0801135E0E01FF
:1024C00055B56393E5030548638608000148630337
:1024D00003002A8871087298FD15131E0801C205B1
:1024E000135E0E01C18179BD13F8150063F4BF00BE
:1024F0007908D5B713381800E5BF83C7F60293F7FC
:102500000708A303F1000346710083C7F60293F79F
:102510000708E394C7FE8347710093F7F70FF1DFD5
:10252000E9B531714AD966CB06DF22DD26DB4ED70D
:1025300052D556D35AD15ECF62CD6AC96EC7AA8C26
:1025400002D897100000E78020B12A8993078008FD
:10255000F3B7078093F787083EDA01000100B71749
:102560000040130770052380E704130780FA2380D7
:10257000E7040100010003C7F7021377770FA38771
:10258000E70203C7F70213678700A387E7022380E8
:102590000704D257F3A70780010001000545970003
:1025A0000000E78060D6130780C13347E902116A53
:1025B00093070AE893065002BD69930BA004814A71
:1025C000014B13048008930470057D1AB347F90288
:1025D0003307D7023EC0FD873ECC938709A69309F7
:1025E000803E3347F7023AC27D873AC43347390306
:1025F0008549B399990193D93940B306D702B30BF2
:102600007703B3C6F602B3CBFB0236C6FD8636C8E7
:1026100093D6FB4136CEB7460F0093860624334946
:10262000D9028566938606FAB3969601B389E902C4
:10263000130760553309D90293060010B389E902E4
:102640003349D902B3C9F9029316390036CA37198A
:102650000040FD8636D0930D090493D7F9413ED250
:10266000F336048093F6860836DC010001009307F8
:1026700070052380FD00930680FA2380DD000100B1
:1026800001008346390593F6860FA309D9048346D2
:10269000390593E61600A309D90423800D00E256FC
:1026A000F3A6068001000100130C80FA116DF336C9
:1026B000048093F6860836DE01000100930770055A
:1026C0002380FD0023808D01010001008346390530
:1026D000216693E60602A309D90483560905B3E6E9
:1026E000A6012318D90483560905D18E2318D904CD
:1026F00023800D00F256F3A60680010001008346F8
:10270000390593F606026381061A03463905218AC4
:102710006DDE081897100000E7800098733604807B
:1027200013768608B2C20100010023809D00238039
:102730008D0101000100B717004003C6370513766D
:10274000F60DA389C70403C6370513660602A389DD
:10275000C704835609052166B3E6A6012318D904E8
:1027600083560905D18E2318D90423800D0096467F
:10277000F3A60680010001008346390593F60602A0
:10278000638B061483463905A18AEDFE970000206D
:10279000E7806090AA8636D497000020E780A08F5B
:1027A000A256E30AD5FE835609054255B3E6A601B3
:1027B0002318D90497100000E780C08F834639059D
:1027C000A18AEDDE03560905834629058247337643
:1027D000CA00B306DA0293D5F641B296B388F64042
:1027E000E24733B8C6002E983308F840A247B3B684
:1027F00016013308D84063C70701631DF8009247EC
:1028000063FA1701C247634FF80E63950701B24799
:1028100063EAF80E894663E9660FF24693151800DD
:1028200013D3F8015E8613951800B365B30042D642
:1028300046D497C00100E780A0313258050B137BC6
:10284000FB0F63470001631A0838A25863870838F2
:1028500013081500B336A800B69513D6F5013298C3
:10286000B336C800AE9613581800FE06B3E606014C
:102870007336048013768608B2C6010001002380F7
:102880009D0023808D01010001000356C902B2960C
:10289000C206C1822316D90223800D00B646F3A6D4
:1028A00006800100010021B5F336048093F6860806
:1028B000B6C00100010023809D0023808D0101002E
:1028C00001008346390593E60602A309D904238053
:1028D0000D0086460DB5F336048093F68608B6C41F
:1028E0000100010023809D0023808D010100010073
:1028F0008346390593E60602A309D90423800D0017
:10290000A646BDB5E30B0BF0F336048093F68608BC
:10291000B6C801000100930680FA23809D00238041
:10292000DD00010001008346390593F5FC0F93F6A5
:10293000860FA309D90483463905CD8EA309D9048E
:1029400023800D00C646F3A6068001000100130592
:1029500080FA03463905930639051D8A631C9629BA
:102960007336048013768608B2CC0100010013068A
:1029700080FA23809D002380CD000100010003C662
:1029800006001376F60D2380C60003C60600136604
:1029900006022380C600835609051166D18E2318CE
:1029A000D904835609052166D18E2318D9042380C2
:1029B0000D00E646F3A6068001000100130680FA2A
:1029C0008346390593F60602638006268346390559
:1029D000130C3905A18AFDDA081897000000E7807A
:1029E000A06BF336048093F68608B6D00100010090
:1029F000930680FA23809D002380DD000100010002
:102A000083460C00116693F6F60D2300DC00834626
:102A10000C0093E606022300DC0083560905D18EE4
:102A20002318D904835609052166D18E2318D904A9
:102A300023800D008656F3A60680010001001306D0
:102A400080FA8346390593F60602638A0620834698
:102A50003905A18AEDFE97F0FF1FE780C0632A8C3D
:102A600097F0FF1FE7802063E30C85FF835609057D
:102A700011664255D18E2318D90497000000E780D3
:102A800060638346390513063905A18AFDDAF336FA
:102A9000048093F68608B6D401000100930680FAFC
:102AA00023809D002380DD00010001008346060095
:102AB00093F6F60D2300D60023800D00A656F3A64C
:102AC0000680010001008356090503462905D24707
:102AD000B376DA003306CA021305800C9355F6412B
:102AE0003696330DF6408257333CD6002E9C333653
:102AF000A601330CFC40330CCC40330885039256BE
:102B00004E86B335A5033305A503C29597C00100D2
:102B1000E780000463468001631E0C16630C0D16EB
:102B2000130615003335A6002E959356F5013696FB
:102B3000B335D600AA959396F50105828585D18E89
:102B40006346B000639D051A638B061A0356C902DB
:102B500015823305D6003336C500B2956348B00000
:102B6000639105241306F00F637DA622894663F363
:102B7000561593078008F3B7078093F78708BED6EA
:102B80000100010037170040930770052300F70488
:102B9000930780FA2300F704010001008356C7025F
:102BA00089678117D58FC207C1832316F7022300D7
:102BB0000704B657F3A7078001000100FA506A54D2
:102BC000DA544A59BA592A5A9A5A0A5BFA4B6A4C49
:102BD000DA4C4A4DBA4D296182801308F5FF33352E
:102BE000A800FD152E951356F5013298B336C8008E
:102BF000AA9695B9F336048093F68608B6CA010002
:102C0000010023809D002380AD0001000100834668
:102C10003905CD8EA309D90423800D00D646F3A62D
:102C200006800100010035B3F336048093F6860870
:102C3000B6CE0100010023809D002380CD0001005D
:102C400001008346390593E60602A309D9042380CF
:102C50000D00F646F3A606800100010095B3F33699
:102C6000048093F68608B6D20100010023809D00FF
:102C70002380CD00010001008346390593E606025A
:102C8000A309D90423800D009656F3A606800100FF
:102C9000010045BB9306F5FF33B5A600FD152E9543
:102CA0009355F501AE96B3B5B600AA951396F50106
:102CB000858269B5F336048093F68608B6D801009C
:102CC0000100930680FA23809D002380DD0001002F
:102CD00001008356C9020566011693F6F60FD18EE0
:102CE000C206C1822316D90223800D00C656F3A660
:102CF000068001000100850A93FAFA0F95B233E6C7
:102D0000B60045C20356C9023305D0403338A0008F
:102D1000B305B040B385054115826345B000D1E1EC
:102D20006371A608894663F0560593078008F3B7D8
:102D3000078093F78708BEDA01000100B71700404B
:102D4000130770052380E704130780FA2380E70444
:102D50000100010003D7C7027D8B2396E702238081
:102D60000704D65781BDF336048093F68608B6DC97
:102D700001000100930680FA23809D002380DD007E
:102D8000010001008356C9020566011693F6F60F8D
:102D9000D18EC206C1822316D90223800D00E656C9
:102DA000B9B793078008F3B7078093F78708BEDEAB
:102DB0000100010037170040930770052300F70456
:102DC000930780FA2300F704010001000356C702AD
:102DD00093975600B297C207C1832316F7022300C8
:102DE0000704F657C1BB914763EEB70217D701003E
:102DF000130707748A05BA959C41BA978287B7175B
:102E0000004003A7470B1345F5FF698F23AAE70A84
:102E100003A7070B698F23A8E70A03A7070A798D81
:102E200023A0A70A8280B717004083A6470B134749
:102E3000F5FFF98E23AAD70A83A6070B558D23A881
:102E4000A70A83A6070A758F23A0E70A8280B7170F
:102E5000004003A7470B498F23AAE70A03A7070BE4
:102E60001345F5FF45BFB717004083A6470B13472F
:102E7000F5FF758F23AAE70A03A7070A598D4DB7F7
:102E8000B717004003A7470B498FEDB7914763EE93
:102E9000B70217D701001307E76A8A05BA959C4164
:102EA000BA978287B717004003A7470D1345F5FF70
:102EB000698F23AAE70C03A7070D698F23A8E70CE6
:102EC00003A7070C798D23A0A70C8280B7170040B9
:102ED00083A6470D1347F5FFF98E23AAD70C83A6C7
:102EE000070D558D23A8A70C83A6070C758F23A06B
:102EF000E70C8280B717004003A7470D498F23AA2C
:102F0000E70C03A7070D1345F5FF45BFB7170040B2
:102F100083A6470D1347F5FF758F23AAE70C03A778
:102F2000070C598D4DB7B717004003A7470D498FC0
:102F3000EDB7797122D43714004026D24AD0035914
:102F400024028354040206D64209C2044ECE52CC57
:102F500056CA13590901C1802DE11379F9F793F489
:102F6000F49F4209C20413590901C18093078008E4
:102F7000F3B7078093F787083EC401000100930769
:102F800070052300F404930780FA2300F404010081
:102F90000100231124032310940223000404A247F8
:102FA000F3A7078001000100B25022549254025945
:102FB000F249624AD24A45618280B7F507008146EC
:102FC0003000B105194597000020E7808081A247B5
:102FD00013972701E34A07FC1369090893E40440A7
:102FE00093098008F3B7098093F787083EC0010072
:102FF0000100930A700523005405130A80FA230088
:10300000440501000100231124032310940223002E
:1030100004048247F3A7078001000100294597F0C7
:10302000FF1FE7802031F3B9098093F989084EC268
:1030300001000100230054052300440501000100A4
:103040008357040293E707202310F40223000404AB
:103050009247B9B7B7170040884742054181937737
:10306000050491EB9377F5013755E80113050580C9
:103070003345F50282809377050C130700046397AC
:10308000E7009377F50137459C1CCDB72165130503
:1030900005D0828037E700E01C435443A183E20659
:1030A000D58F1CC1FD572320F7182322F7188280E3
:1030B00013178500B7E700E023A0E710618123A282
:1030C000A7108280B7F700E08847CC47828081470D
:1030D00037370040A14663C4C7003285828003456C
:1030E000B740E38EA6FE3385F5000345050085074E
:1030F0002304A740CDB797070020938727EF9C4371
:10310000173700201307072E3E95636EE50017372B
:1031100000201307273F6368A70017070020232715
:10312000A7EC3E858280FD57EDBF8280411122C40D
:1031300006C62A8497000000E78000F22947B307FB
:10314000E502B2408D83B3D7870222449507B3D7F7
:10315000E70237370040C207C1832316F700410159
:103160008280411137150E0006C697000000E780E7
:1031700020FCB7370040130770F82381E7000D47A4
:10318000A381E70013070004A380E7000547238716
:10319000E700B24041018280373700408347270073
:1031A0001A0593F7F703C98F93F7F70F2301F70079
:1031B0008280B737004003C7170019C9D98DA38093
:1031C000B70003C70700136787002380E7008280EA
:1031D00093C5F5FFF98DA380B7008280AE872A875B
:1031E000B736004021463738004089E71703000012
:1031F0006700E3F383C8B600E30916FF05078348B9
:10320000F7FFFD17C20723041801C183F9BF41115D
:1032100022C406C62A8497000000E780E0E329471D
:10322000B307E502B2408D83B3D7870222449507E6
:10323000B3D7E70237370040C207C1832316F740F0
:1032400041018280716541111305052006C6970072
:103250000000E78000FCB7370040130770F82381B7
:10326000E7400D47A381E74013070004A380E74030
:1032700005472387E740B24041018280CC4141119C
:1032800006C6328503C6150083C5050022064D8E8D
:1032900042068D654186138875A2630C0611634B47
:1032A000C804138845A26300060D634AC8009385CD
:1032B00035A26301B6082390060029464DA0138865
:1032C00055A26305060D938565A2E316B6FE8D45EE
:1032D0001D4663E6E5081146198E63F3C7003E8676
:1032E000B7E704002390C600FC4797D501009385FB
:1032F000A5279DA0138895A263030611634E060DB2
:103300001388A5A263000613938505A5E315B6FAF5
:1033100099451D4663E5E504198E63F3C7003E86B3
:10332000B7E704002390C600FC479705002093856B
:1033300025D61DA09D451D4663E3E5022146198E55
:1033400063F3C7003E86B7E70400FC472390C6003E
:103350009705002093858534BA9582970146B2403F
:10336000328541018280AD451D46E3EAE5FE3146E6
:10337000198E63F3C7003E86B7E704002390C600AA
:10338000FC4797D501009385A520F9B7B1451D46A7
:10339000E3E7E5FC3546198E63F3C7003E86B7E7E1
:1033A00004002390C600FC4797D501009385451F74
:1033B00065B78D451D46E3E4E5FA1146198E63F3C2
:1033C000C7003E86B7E704002390C600FC4797D5A8
:1033D00001009385251A49B78D451D46E3E1E5F8BF
:1033E0001146198E63F3C7003E86B7E704002390A9
:1033F000C600FC4797D501009385451CB1BFA54584
:103400001D46E3EEE5F42946198E63F3C7003E86B8
:10341000B7E704002390C600FC4797D501009385C9
:1034200025161DBFB5451D46E3EBE5F23946198E5D
:1034300063F3C7003E86B7E704002390C600FC474D
:1034400097D501009385451101BFB7E7040003A399
:103450000713970600209386A6C24146A545170587
:1034600000201305E5B802832D455DE703C505007F
:103470000947631FE50803A84500411106C6034735
:10348000180032850346080022074168518F9308CF
:1034900028FE6307170563E9E800051863030703BF
:1034A00023900600294591A8130648FE630AC70425
:1034B0001518E31707FF15463E87637BF60015478F
:1034C00001A8130600023E876374F600130700028A
:1034D000B7E704002390E600FC471316070111A884
:1034E0003E8691C30546B7E70400FC472390C6001B
:1034F0004206CC45418282970145B240410182801B
:10350000130600083E87E375F6FC13070008C9B7E9
:103510002390060005458280828041677917630405
:10352000E504411122C406C685472A84639FF5003D
:10353000B7E7040022852244B24003A3871397050E
:1035400000209385E52F4101028389476399F500A7
:10355000B7E7040083A7070B8545829771D9B2406E
:103560002244410182808280797126D252CCAE847D
:103570002A8A97D501009385650617D501001305A2
:10358000650806D63AC622D44AD0368432894ECE51
:1035900097C00100E78000A7A28517D50100130599
:1035A000650797C00100E780E0A5294597C00100A5
:1035B000E78020AA83C7840093F70702F9E383C951
:1035C00004008947054532476396F908D44083C70C
:1035D000160083C60600A207D58FC166138616FEA5
:1035E000638CC7028D16638FD7068D6693862690EF
:1035F00029456391D706B7E70400A286225403A3A6
:103600004714B250F2494A86A6850259925452850F
:10361000624A8547456102832D450DEF93070002FD
:10362000354563E98702B7E70400FC47C844130641
:103630000002CA8582978149970700209387072156
:103640009C43014581CB9C4391C74E852286CA8508
:1036500082970145B250225492540259F249624A6B
:10366000456182802D457DF79307700F3545E3E373
:1036700087FEB7E70400FC47C8442286CA858297C4
:1036800065BF2145C1BF411122C437E4040083272F
:10369000841326C2AA84416506C697050020938537
:1036A000251A7D1582978327C40A17050000130584
:1036B00005E78588829795C0032304132244B2400E
:1036C000924497060020938626AE4146C5451705CD
:1036D00000201305659C41010283B24022449244BC
:1036E00001454101828019C59707002023A0A71634
:1036F00001458280454582801147636AA70A97D6B3
:103700000100938666EC0A0536951841411106C6FC
:103710003697AE87B2850287130700026145639D25
:10372000E700B7E70400FC47130600021705002076
:10373000130545F782970145B24041018280054754
:103740006145E39BE7FEB7E70400FC470546170524
:103750000020130525F7F9BF1307700F6145E39D9E
:10376000E7FCB7E70400FC471306700F17050020BD
:10377000130585F5C1B7130700086145E39EE7FA15
:10378000B7E70400FC4713060008170500201305DF
:1037900025034DB715476145E390E7FAB7E7040005
:1037A000FC471546170500201305C50961B70945F3
:1037B0008280411126C2B7E4040083A7C41322C447
:1037C0004AC006C62E8497050020938565072A897E
:1037D0008297058905C5970700209387E78B83D7D4
:1037E000A70BA28503A3440D2310F4002244B2408A
:1037F00092444A850249014641010283B240224473
:103800009244024949454101828097070020238163
:1038100007049707002023AF0702B717004003A74C
:10382000070CB706C0FFFD16758F23A0E70C03A792
:10383000070DB7064000558F23A8E70C03A7070C18
:103840003D9B23A0E70C03A7070D1367070123A8DF
:10385000E70C8280B717004003A5470C83A7470CED
:10386000598113451500C18B058999E3136525001E
:103870009707002083C7C7FD6380A7029707002032
:103880002388A7FC11C9970700209387A7FC03A3EF
:1038900007006303030002838280114517F3FFFFD3
:1038A000670063C8011122CC06CE3714004026CA37
:1038B0004AC84EC652C483447405034AB4058349BA
:1038C00084050349940597F0FFFFE780A0A0834794
:1038D000A40593F4F40F137AFA0F93E71700230D5E
:1038E000F40493F9F90F1379F90FB717004003C7E0
:1038F000A705058B6DFF03D5C705A38D4705238C51
:103900003705A38C2705A38B9704F2406244D24469
:103910004249B249224A05618280411193970501CB
:1039200022C406C626C2C1872E8463DC0700B7E422
:103930000400FC54829719C1BC5482972165218DE3
:1039400015A893F7150013C515008DE793F725000B
:103950009DC797000000E78020F0B7E70400BC4F48
:103960001306000A894517050020034525EF8297B5
:1039700013452400B240224492444101828093972F
:10398000250163D80702B7E4040083A7C41E829709
:1039900097000000E780A0F0BC4C375607001306E4
:1039A0000630896517050020034545EB82970965B8
:1039B00079B7939715010145E3DE07FA17D50100A2
:1039C000130545CD97B00100E780A07BB7E7040061
:1039D000BC4F13060064916517050020034505E8F8
:1039E00082971165A9BF1D71A2CC37E404005C5C0D
:1039F000485886CE494697D50100938525C58297BC
:103A000011E917D501001305A5C597B00100E7809E
:103A1000407701A0B7F600E0795798CAFD57DCCA95
:103A20000567B7E700E023A0E7101306F00290C295
:103A300023A0E718010001003707002018471306EC
:103A4000000481459706002023A8E6E04157A38A99
:103A5000E7403C4408088297970700209387877EB9
:103A60003EC8856713870740938757D1231AE10023
:103A70002312F1021307B00F97F7FFFF9387C76474
:103A80002310E1023ED81547970700009387C7E14E
:103A9000B7F50700A30FE1003EDC054797070000DC
:103AA0009387E7DF81463000E10519452301E102F4
:103AB0003EDE97F0FF1FE780C0D218088147994685
:103AC00030003E960346060085070507A30BC70096
:103AD000E398D7FEC24791C70357410185676373D7
:103AE000F70001A0B7E7040083A7470A08088297F8
:103AF000AA8511C917D501001305C5B797B00100F4
:103B0000E780405001A0F640664425618280411163
:103B100026C2B7E4040083A7040806C622C417051A
:103B200000001305C5DF829717040020130404D397
:103B30002300A40097000000E780800297000000A7
:103B4000E780E0CC03450400224403A38405B2408F
:103B5000924413060032896541010283797106D6C9
:103B600022D413078008F337078093F787083EC2F3
:103B700001000100B7170040930570052380B704CA
:103B8000130680FA2380C7040100010083C6F702F0
:103B900093F6A60FA387D702238007049246F3A6C5
:103BA00006800100010073370780137787083AC445
:103BB000010001002380B7042380C7040100010035
:103BC00003C7F70213672700A387E70223800704D0
:103BD000A247F3A7078001000100054597E0FFFF1A
:103BE000E780807297000000E78060CB0147814644
:103BF0008147054685451305407E97E0FFFFE78036
:103C0000807537E404003C44680051468145829742
:103C1000B707C0A83EC8B787E803938707D03ECA56
:103C200097E7FF1F9387A7793EC67C586800829765
:103C3000B250225445618280411197D5010093858D
:103C4000650917D501001305E59B06C697B001006D
:103C5000E780403B17D501001305851F97B0010091
:103C6000E780403AB2402945410117B3010067009F
:103C7000433E411197D501009385050717D50100F3
:103C80001305459806C697B00100E780A03717D501
:103C900001001305A51A97B00100E780A036B240D5
:103CA0002945410117B301006700A33A411122C41D
:103CB00006C6834705002A849DC797D501009385D2
:103CC000650817D501001305E59397B00100E7805B
:103CD00060334C4017D501001305052D97B0010046
:103CE000E78040323DA058410DEF97D50100938504
:103CF000650517D501001305E59097B00100E78031
:103D0000603017D501001305A52B97B00100E7809F
:103D1000602F2244B2402945410117B301006700DA
:103D20004333A1679386D7036313D70297D5010066
:103D30009385450117D501001305C58C97B0010087
:103D4000E780402C17D50100130585287DBFED07BE
:103D500097D50100938505FF17D501001305858AC6
:103D6000631BF70097B00100E780C02917D5010059
:103D70001305452759BF97B00100E780A0284C40A4
:103D800017D501001305052891BF411197D50100F2
:103D90009385C5F617D501001305C58606C697B0ED
:103DA0000100E7802026B2402945410117B30100F8
:103DB0006700232A397122DC26DA4AD82E842A8920
:103DC0008145B2844808714636C606DE97E0FFFF9B
:103DD000E780E03397F7FF1F9387075EDC4783D7C1
:103DE0000700231C2101231BF10097500000E780EE
:103DF000803D9307800CB2463ECE03576101FD57CC
:103E00002302F102C167230DA100A30DD100FD170C
:103E10007D556309F7002686A28548089750000063
:103E2000E780403DF2506254D25442592161828071
:103E3000854617030000670023F84111814617F6F5
:103E4000FF1F1306A654854517050020035585223C
:103E500006C697D00000E780A08C15C997D5010051
:103E6000938505ED17C501001305C57997B00100CD
:103E7000E780401917D501001305050F97B0010021
:103E8000E7804018294597B00100E780801C97D54E
:103E900001009385E5E917C501001305A57697B0E4
:103EA0000100E780201617D501001305250D97B0F6
:103EB0000100E7802015294597B00100E7806019CF
:103EC00097F7FF1F9387474FDC47054797D50100BA
:103ED000938505E62390E70017C501001305857259
:103EE00097B00100E780001217D501001305450ABD
:103EF00097B00100E7800011B2402945410117B396
:103F000001006700031531C9A9C9411122C406C6C1
:103F100026C2930700022E8463F4B7001304000244
:103F2000B7E40400FC4413160401AA854182170576
:103F300000201305E51D829797070020239A871E0E
:103F4000224403A30405B240924417050020034510
:103F5000659193050040410102838280411122C492
:103F600097D50100938545DF2A8417C50100130505
:103F7000656906C697B00100E780C0084C4017D5B8
:103F800001001305E5FB97B00100E780A007294574
:103F900097B00100E780E00B034704009307F00FA0
:103FA000631FF70297D50100938505DB17C5010054
:103FB0001305456597B00100E780C0044C4017D554
:103FC00001001305E5F897B00100E780A003224443
:103FD000B2402945410117B3010067008307B24091
:103FE000224441018280411122C426C22A84AE8427
:103FF00017C501001305056197D50100938585D18B
:1040000006C697B00100E780E0FF17D50100130551
:10401000250497B00100E780E0FE294597B0010034
:10402000E780200397D501009385C5CE9707002030
:104030002392870417C501001305C55C0544970743
:104040000020239797029707002023948702971751
:104050000020239C976E97B00100E780A0FA971587
:10406000002083D5856E17D501001305E5FE97B0B6
:104070000100E78020F9294597B00100E78060FD45
:10408000971700202380875C97F7FF1F9387C7321D
:10409000DC4717F5FF1F0345E57C03D70700C16721
:1040A000FD17631EF700B7E7040003A38705130697
:1040B000000A85452244B240924441010283B7E799
:1040C000040003A387051306001493050010DDB751
:1040D000B1C1411122C417C501001305A5522E8498
:1040E00097D50100938545C206C697B00100E780C9
:1040F00060F1A28517D501001305C5F497B0010042
:10410000E78040F02244B2402945410117B3010045
:10411000670023F48280011122CC06CE26CA4AC849
:104120004EC693F715002E84B5CB97000000E780AC
:1041300000D1930710F8170700202309F70097070D
:10414000002083D7E7F217070020A301F70091456D
:10415000A18317050020130565FF1707002023081A
:10416000F7FE97070020A38407FE97600000E78012
:10417000C0C6B7E70400BC4F130600149305001037
:1041800017F5FF1F0345056E829713451400F24093
:104190006244D2444249B2490561828093F70520C6
:1041A00081CB97070020238307F613C50520C5B7E9
:1041B00093F705408DC79705002083D565F789CD16
:1041C000170500201305C5F497F0FFFFE7804001B5
:1041D00097070020239E07F4134504404DBF93F733
:1041E0000510B1C3054597600000E78000C81715AA
:1041F00000200355855597600000E7808093972045
:104200000000E780C0509707002083C7770389E745
:1042100097600000E780A0E997600000E780E0EA8F
:1042200013450410ADB793F72500E9CF1707002019
:10423000035727F069C7AD64B71900409384A4AA57
:1042400023A0990097060020938606EF944297D703
:104250000100938727E3170600200346A6ED81455A
:1042600017D50100130505E397700000E780C067CC
:1042700023A0990097F7FF1F2394A7042A8941C11F
:1042800097D50100938585B117C5010013058537C2
:1042900097B00100E78000D7CA8517C50100130554
:1042A000E54F97B00100E780E0D5294597B00100C0
:1042B000E78020DA97070020239D07E6930710F890
:1042C000170700202304F7E89707002083D747DA71
:1042D00017070020A30CF7E6A18317070020230887
:1042E000F7E691458D4717050020130525E61707CA
:1042F0000020A30EF7E497600000E78000AE1345AE
:10430000240071B593F74500D1C397D5010093857B
:10431000E5A817C501001305E52E97B00100E78059
:1043200060CE17C501001305254997B00100E7804D
:1043300060CD294597B00100E780A0D1930720F810
:10434000170700202304F7E09707002083D787D4BE
:1043500017070020A30CF7DEA1831707002023080E
:10436000F7DE854717070020A303F7DE975000000C
:10437000E78060FC17050020130545DD9145976037
:104380000000E78080A51345440011B593F7850030
:10439000A9C797D50100938565A017C5010013052E
:1043A000652697B00100E780E0C517C50100130539
:1043B000E54197B00100E780E0C4294597B00100CE
:1043C000E78020C997070020239507D69770000043
:1043D000E7806061134584005DBB93F70501D1C39D
:1043E0008545170500200355E5CA97600100E78061
:1043F000601697D501009385659A17C501001305CE
:10440000652097B00100E780E0BF17C501001305E4
:10441000253D97B00100E780E0BE294597B0010037
:10442000E78020C3930730F8170700202300F7D256
:104430009707002083D707C617070020A308F7D0E7
:1044400017050020130585D0A1838D45170700208F
:10445000230FF7CE97600000E780209813450401F2
:104460003DB393F70502D1C797D501009385059316
:1044700017C501001305051997B00100E78080B842
:1044800017C501001305053897B00100E78080B714
:10449000294597B00100E780C0BB930740F8170794
:1044A00000202305F7CA9707002083D7E7BC17072A
:1044B0000020A30DF7C8A183170700202309F7C820
:1044C000854717070020A304F7C897070020239506
:1044D00007BA97500000E78000E617050020130593
:1044E000E5C6914597600000E780208F13450402E0
:1044F00079B993F70504FDC397D501009385058A23
:1045000017C501001305051097B00100E78080AFC3
:1045100017C501001305853097B00100E78080AE14
:10452000294597B00100E780C0B29707002083C7F4
:10453000E7C11307700A6386E7061307800A638CD6
:10454000E7081307600A6393E704930760F8170707
:104550000020230DF7BE9707002083D707BB17075E
:104560000020A305F7BEA183170700202301F7BE93
:10457000854717070020A300F7BEB14517050020A7
:104580001305C5BC97600000E780208597500000A8
:10459000E78060DA1345040497070020239707B6E5
:1045A000FDB6930770F8170700202301F7BA9707A5
:1045B000002083D787B517070020A309F7B8A18388
:1045C000170700202305F7B8854717070020A30128
:1045D000F7B8994565B7930780F8F1B793F70508E1
:1045E0000145E38607BA97C501009385257B17C56A
:1045F00001001305250197B00100E780A0A017C5B1
:1046000001001305252397B00100E780A09F2945ED
:1046100097B00100E780E0A39307A0F817070020F8
:104620002306F7B29707002083D747B1170700206A
:10463000A30EF7B0A18317070020230AF7B0854720
:1046400017070020A305F7B097070020239807AEAF
:1046500097500000E78020CE17050020130505AF16
:10466000914597500000E78040771345040805B650
:1046700097F7FF1F83C7771F17F5FF1F0345051F18
:104680003D8D220597F7FF1F83C7571E3D8D4605B9
:10469000458111C5D1476315F50055458280054513
:1046A00082804111971700202391070A9717002055
:1046B000238A07F806C617070020034727A9930790
:1046C000F00A6315F7029307F0F8894517050020F3
:1046D0001305C5A717070020230AF7A69707002090
:1046E000A38607A697500000E780206F9760000020
:1046F000E780E09B97600000E780209D81453705BB
:1047000004009707002023A907A29707002023830E
:1047100007A297070020239F079697070020239D55
:104720000794970700202392079E9707002023975E
:1047300007A097300000E780E00001459750000097
:10474000E780A07297000000E780C0F29707002082
:104750002391A79EB7E70400BC4F130600148945B8
:1047600017F5FF1F03450510829797C50100938534
:10477000655B17C501001305E5E897B00100E78008
:1047800060889705002083D5C59A17D501001305C9
:10479000A58D97B00100E780E086B2402945410130
:1047A00017B301006700E38A011122CC37E404004B
:1047B0005C5C06CE26CA354697C501009385856A9E
:1047C00017D501001305453A829711E917C5010075
:1047D000130505E997B00100E780A09A01A097F7BB
:1047E000FF1F9387E7083EC4B7F5070085679387E7
:1047F0000780814617F6FF1F13060607E1051945D6
:104800003EC697E0FF1FE780C0FD7C44194697F540
:10481000FF1F93856505170500201305E58782971F
:10482000340017F6FF1F1306260497D50100938561
:10483000A5AE17D501001305A5AF97700000E7805E
:10484000A0DFAA8421C197C501009385255417C50F
:104850000100130525DB97A00100E780A07AA6855B
:1048600017C501001305056197A00100E780807955
:10487000294597A00100E780C07DF2406244D24400
:104880000561828097E00000E780C04417C5010001
:104890001305455597600000E780C0D3976001007D
:1048A000E78000FE17F5FF1F130585AD9760010037
:1048B000E780A0E617C501001305C5539760010006
:1048C000E78080FEAA8497600000E780803A971016
:1048D0000100E780E0D597800100E780006F9780B6
:1048E0000000E780609697700000E78080B09740F6
:1048F0000100E780409797C501009385254917C5BA
:104900000100130525D099C897A00100E780806FAA
:10491000A68517C5010013052558B9B797A0010052
:10492000E780406E17C501001305455997A00100A7
:10493000E780406D294597A00100E780807197309E
:104940000100E780207397000100E780E0916DC5CA
:1049500085453705040097300000E780A0DE97C545
:1049600001009385A54217C501001305A5C997A0AD
:104970000100E780206917C501001305A55597A020
:104980000100E7802068294597A00100E780606C5E
:1049900097F7FF1F9387C79183D70700171700204A
:1049A0002315F7DA854717170020230DF7C897F767
:1049B000FF1F938767A0DC4703D70700C167FD1778
:1049C0006316F70097F0FFFFE780604797700000DD
:1049D000E780A0118567938707E33E9597700000F5
:1049E000E780601197200000E78060D21715002053
:1049F0000355A5D597500000E780A01305459750B3
:104A00000000E780804697500000E780006C97C563
:104A100001009385A53717C501001305A5BE97A012
:104A20000100E780205E17C501001305255097A0FF
:104A30000100E780205D2DBD97000000E78080C366
:104A400097F7FF1F2397A76E97C50100938505343D
:104A500017C50100130505BB97A00100E780805A28
:104A600017C601001306464997F5FF1F83D5656CED
:104A700017C501001305C54897A00100E7808058BD
:104A8000294597A00100E780C05C3C4C1306000A52
:104A9000894517F5FF1F0345E5DC829701459750CF
:104AA0000000E780803CA5B7411122C437E4040030
:104AB0008327041A06C6829797500000E780200BD0
:104AC0008327040817F5FFFF13052565829797F7DD
:104AD000FF1F2389A7D817F5FF1F1305E58D9750F2
:104AE0000000E78000BC2244B240410117030000EF
:104AF0006700C3CBB7E70400FC4741112E8606C60A
:104B000022C426C24AC02E842A89AA8517F5FF1F0F
:104B10001305C563829797C501009385252B17C59B
:104B20000100130525AE97A00100E780A04D97F581
:104B3000FF1F83C5A56117C50100130525D197A0E7
:104B40000100E780204C294597A00100E7806050D4
:104B500097F4FF1F9384845F83C7040041479387C2
:104B6000070693F7F70F636FF75A17C7010013078C
:104B7000A7B28A07BA979C43BA9782879D47630773
:104B8000F40297C501009385652417C5010013053C
:104B900065A797A00100E780E04617C5010013054F
:104BA00065CB97A00100E780E04595A497F7FF1F2C
:104BB00083C7D759DDCB17F7FF1F0347575997F71F
:104BC000FF1F83C7C75822075D8F97F7FF1F83C753
:104BD0002758C2075D8F97F7FF1F83C77757E207F4
:104BE000D98F17F7FF1F2329F75483C7640097C590
:104BF00001009385A51D17C501001305A5A017F792
:104C0000FF1F2309F75297A00100E780A03F97F705
:104C1000FF1F938767528C4317F6FF1F0346865189
:104C200017C501001305C5C497A00100E780803DAA
:104C3000294597A00100E780C04197F7FF1FA38790
:104C400007502244B24092440249930700F817F7F4
:104C5000FF1F230DF74E9D4517F5FF1F1305054F49
:104C60004101175300006700431797700000E78069
:104C700000E797F7FF1F238CA74C9357850017F782
:104C8000FF1FA306F74C935705012A8417F7FF1F50
:104C90002300F74C93578501014517F7FF1FA30920
:104CA000F74A97700000E780E0E797F7FF1F23823D
:104CB000A74A97C501009385651117C50100130523
:104CC000659497A00100E780E03317F6FF1F0346C5
:104CD0004648A28517C50100130505BBB1B7CD47EE
:104CE0006303F40297C501009385450E17C50100C3
:104CF0001305459197A00100E780C03017C501005A
:104D0000130505BA79BD97F7FF1F83C7474517F706
:104D1000FF1F0347B744A207D98FC207C18717F700
:104D2000FF1F2318F740634AF00097000000E78058
:104D3000609497F7FF1F239EA73EB7E7040003A3E5
:104D400087051306000A89452244B240924402496D
:104D500017F5FF1F034505B1410102838D4763032A
:104D6000F40297C501009385650617C50100130578
:104D7000658997A00100E780E02817C501001305A9
:104D8000A5B305B517F4FF1F0344643C97F7FF1F55
:104D900083C7D73B97C5010093854503220417C5F8
:104DA0000100130525865D8C97A00100E780802512
:104DB000A28517C501001305A5B197A00100E780E2
:104DC0006024294597A00100E780A0280D4697F5AB
:104DD000FF1F9385A537228597F0FFFFE7808005A9
:104DE000AA8421C197C50100938545FE17C501001E
:104DF0001305458197A00100E780C020A68517C54F
:104E00000100130525AE97A00100E780A01F2244F2
:104E1000B240924402492945410117A301006700AD
:104E2000432397F7FF1F23978726B7E704001166F0
:104E300003A38705130606E8914539B78D47630339
:104E4000F40297C50100938565F817B501001305B5
:104E5000657B97A00100E780E01A17C501001305E4
:104E6000A5A981B317F4FF1F0344642E97F7FF1F12
:104E700083C7D72D97C50100938545F5220417B543
:104E80000100130525785D8C97A00100E78080174D
:104E9000A28517C501001305A5A797A00100E7800B
:104EA0006016294597A00100E780A01A0D4697F5E6
:104EB000FF1F9385A529228597F0FFFFE78080F7E4
:104EC000AA841DC197C50100938545F017B501005F
:104ED0001305457397A00100E780C012A68517C58A
:104EE0000100130525A405B797F7FF1F2396871820
:104EF000B7E70400116603A38705130606E89305C8
:104F0000000299B5894763E3870297C5010093853D
:104F1000E5EB17B501001305E56E97A00100E780EA
:104F2000600E17C50100130565A1A5B997F4FF1F11
:104F300083C4E42197F7FF1F83C7572197C501005A
:104F40009385C5E8A20417B501001305A56BDD8C98
:104F500097A00100E780000BA68517C50100130587
:104F6000259F97A00100E780E009294597A001004F
:104F7000E780200E228697F5FF1F9385251D268545
:104F800097F0FFFFE78000EB2A84630E051A97C5B0
:104F900001009385A5E317B501001305A56697A049
:104FA0000100E7802006A28517C501001305859B37
:104FB00099BD854763F98718834519002244B2409B
:104FC00092440249B335B00097F7FF1F238EB70C08
:104FD00017C501001305459A410117A30100670099
:104FE0006302A2852244B24092444A8502494101AB
:104FF00017130000670003F199476303F40297C594
:1050000001009385A5DC17B501001305A55F97A0E6
:105010000100E78020FF17C501001305659751B611
:1050200017F4FF1F0344A41297F7FF1F83C717123B
:1050300097C50100938585D9220417B50100130592
:10504000655C5D8C97A00100E780C0FBA28517C559
:1050500001001305259597A00100E780A0FA2945D6
:1050600097A00100E780E0FE194697F5FF1F9385A2
:10507000E50D228597F0FFFFE780C0DBAA841DC104
:1050800097C50100938585D417B501001305855791
:1050900097A00100E78000F7A68517C5010013055A
:1050A000659195B397F7FF1F239A8708B7E7040028
:1050B000116603A38705130606E89305000869B186
:1050C000854797C50100938565D017B50100130585
:1050D0006553630BF40097A00100E780A0F217C5A9
:1050E00001001305658E75BC97A00100E78080F173
:1050F00017C501001305C58E97A00100E78080F059
:10510000294597A00100E780C0F42244B2409244B0
:10511000024997F7FF1F239E070041011773000004
:105120006700638C97C50100938545CA17B50100D8
:105130001305454D97A00100E780C0EC17C501009D
:105140001305458BB9BCB240224492440249410147
:105150008280411106C622C426C239C12A8497F032
:105160000000E7806010AA8411EDB7E70400BC4797
:105170004146814522858297B24022442685924449
:105180004101828041657D1597F00000E780A00E07
:10519000B7E7040001E9BC47414681452285829773
:1051A0008144D9BF0347E501FC479305900819E303
:1051B00093050003AA9541462285829785446DBFD9
:1051C00093170501C1876359F00297F7FF1F2390DA
:1051D000A7F4854717F7FF1F230AF7F2B7E7040084
:1051E00003A387050566130606C89305002017E587
:1051F000FF1F0345256702838280B7E70400FC4751
:105200001171A2DDA6DBCAD986DFCED72A892E840A
:10521000B2842E86AA8517F5FF1F130525F3829702
:1052200017F7FF1F130787F2834707009306F00263
:105230009387E70793F7F70FE3E4F614BA898A0731
:1052400017B7010013078749BA979C43BA9782871B
:105250008D4797C501009385A5B517B501001305C6
:10526000653A630AF40297A00100E780A0D917B558
:1052700001001305656497A00100E780A0D82945C7
:1052800097A00100E780E0DCFE506E54DE544E59DA
:10529000BE591161828097A00100E780A0D617B5A2
:1052A00001001305257697A00100E780A0D52945C8
:1052B00097A00100E780E0D9930720F8114697F501
:1052C000FF1F9385A5E8268517F7FF1F2300F7E842
:1052D00097F7FF1FA38D07E697F0FFFFE78080B5E4
:1052E0002A841DC997C50100938585AC17B50100B7
:1052F0001305453197A00100E780C0D0A28517B5FE
:1053000001001305E57397A00100E780A0CF2945B0
:1053100097A00100E780E0D397C50100938545A9D8
:1053200017B501001305052E97A00100E78080CD79
:1053300017B501001305057297A00100E78080CC26
:10534000294597A00100E780C0D04165930730FA56
:10535000054697F5FF1F938565DF7D1517F7FF1F3E
:105360002306F7DE97F0FFFFE780C0AC2A841DC953
:1053700097C501009385C5A317B5010013058528BE
:1053800097A00100E78000C8A28517B501001305AA
:10539000256B97A00100E780E0C6294597A0010092
:1053A000E78020CBB7E70400BC4F0566130606C8AC
:1053B000A14517E5FF1F0345E54A8297F1B59147DF
:1053C0006303F40297C501009385859E17B501001C
:1053D0001305452397A00100E780C0C217B501005F
:1053E0001305856A49BDB7E70400FC4F914517E5F1
:1053F000FF1F03452547829797C501009385459B6D
:1054000017B501001305052097A00100E78080BFB4
:1054100017B501001305056997A00100E78080BE5C
:10542000294597A00100E780C0C297400000E780AF
:1054300080F091451DA485476303F40297C50100E0
:105440009385059717B501001305C51B97A00100AB
:10545000E78040BB17B501001305456629BD97F7E6
:10546000FF1F239997C2B7E704000566BC4F1306D8
:1054700006C8C1453DBF8D476303F40297C50100CF
:105480009385059317B501001305C51797A0010073
:10549000E78040B717B5010013050546E9BB930740
:1054A00040F8114697F5FF1F938545CA268517F7E3
:1054B000FF1F230DF7C897F7FF1FA38A07C897F0B0
:1054C000FFFFE78020972A84E30005DC97C50100F1
:1054D0009385058E17B501001305C51297A001002D
:1054E000E78040B2A28517B501001305655597A066
:1054F0000100E78020B161B39147E311F4F8B7E709
:105500000400FC4F9305000217E5FF1F0345853596
:10551000829797C501009385A58917B501001305EA
:10552000650E97A00100E780E0AD17B501001305F7
:10553000A55ADDB5894763E3870297C501009385C6
:10554000258717B501001305E50B97A00100E7803B
:1055500060AB17B501001305653E31BB17F9FF1F9E
:105560000349E9BE97F7FF1F83C757BE97C50100E0
:1055700093850584220917B501001305A508336931
:10558000F90097A00100E780E0A7A28517B5010008
:105590001305C55597A00100E780C0A6420929451B
:1055A00097A00100E780E0AA135909419305D4FFB1
:1055B00093160901C182268693F5F50F17F5FF1F93
:1055C0001305F5B897200000E780801BE35E20CB31
:1055D000930750F817F7FF1F230AF7B683C7390060
:1055E000228697F5FF1F938565B68507268517F7F1
:1055F000FF1FA30EF7B497F0FFFFE780A0832A8474
:10560000E30405C897B501009385857A17B50100B5
:10561000130545FF97A00100E780C09EA28517C52E
:105620000100130525A1E1B5894763E3870297B51A
:1056300001009385E57717B501001305A5FC97A038
:105640000100E780209C17B501001305E54B25B14B
:1056500097400000E78020CEA28517F5FF1F1305B5
:10566000E5AE97400000E780407739B98D47630386
:10567000F40297B501009385A57317B501001305D2
:1056800065F897A00100E780E09717B501001305C2
:105690006549D5B6B76602000146B77502000545F3
:1056A00097D0FF1FE780E013930760F817F7FF1FFD
:1056B000230EF7A897F7FF1FA38B07A893070006F1
:1056C00017F7FF1F2306F7A8894717F7FF1FA30146
:1056D000F7A897F7FF1F238E07A697F7FF1FA38A48
:1056E00007A6C14717F7FF1F2306F7A6930720F960
:1056F00017F7FF1FA300F7A6314697F7FF1FA38CEC
:10570000A7A497F5FF1F938565A4268597F7FF1F2C
:10571000238307A497E0FFFFE780C0712A84E30595
:1057200005B697B501009385A56817B50100130567
:1057300065ED97A00100E780E08CA28517B5010018
:105740001305C53F6DB3B1476303F40297B501007C
:105750009385056617B501001305C5EA97A00100FA
:10576000E780408A17B501001305053F29B6B7E762
:105770000400FC4F9305000417E5FF1F0345850E49
:10578000829797400000E78000BBB145F9B591478B
:1057900063E3870297B501009385856117B5010022
:1057A000130545E697A00100E780C08517B5010005
:1057B0001305453CC9B417F9FF1F0349699997F7C9
:1057C000FF1F83C7D79822093369F9000E09B777FD
:1057D00002006D143E992286CA8517B50100130593
:1057E000A53A97A00100E780E081B7E70400FC47F5
:1057F000228697F5FF1F9385B5952800829793160B
:105800000401C1823000CA85094597D0FF1FE78097
:1058100040FD2A8409C917B501001305A53897A0D2
:105820000100E7800096930770F8194697F5FF1F6F
:105830009385C591268517F7FF1F2309F79097F7E2
:10584000FF1FA387879097E0FFFFE780A05E2A8471
:10585000E30C05A297B501009385855517B50100A6
:10586000130545DA97900100E780C079A28517B546
:10587000010013052534A5B99947630CF41297B5B7
:1058800001009385E55217B501001305A5D7979040
:105890000100E780207717B5010013052533E1BA31
:1058A000914763E3870297B501009385655017B56B
:1058B0000100130525D597900100E780A07417B566
:1058C00001001305253245BA17F9FF1F034949881E
:1058D00097F7FF1F83C7B78722093369F9000E09BD
:1058E000B77702006D143E992286CA8517B501006C
:1058F0001305853097900100E780C070B7E704007A
:10590000FC47228697F5FF1F938595842800829790
:1059100093160401C1823000CA850D4597D0FF1F40
:10592000E78020EC2A8409C917B501001305852EEC
:1059300097A00100E780E084930780F8194697F567
:10594000FF1F9385A580268517F7FF1F2300F7808B
:1059500097E7FF1FA38E877E97E0FFFFE780804DCC
:105960002A84E303059297B501009385654417B532
:105970000100130525C997900100E780A068A28562
:1059800017B501001305452A9DB699476303F40234
:1059900097B501009385C54117B50100130585C66C
:1059A00097900100E780006617B5010013054529AF
:1059B000D9B0B7E70400FC4F9305000417E5FF1FBB
:1059C000034545EA829797400000E780C0969945D5
:1059D00069B18D476303F40297B501009385453D96
:1059E00017B50100130505C297900100E78080619B
:1059F00017B5010013054526BDB817B501001305FD
:105A0000A52697900100E780C0771305C01297D0B4
:105A1000FF1FE7800093014597D0FFFFE780C06735
:105A20000D4597000000E780A047294597D0FF1F4C
:105A3000E780209197D0FF1FE7808081B1B0994720
:105A40006303F40297B501009385853617B501000D
:105A5000130545BB97900100E780C05A17B50100B8
:105A6000130505F309B817E7FF1F0347776E97E79C
:105A7000FF1F83C7E76D22075D8F9166BA96C20646
:105A80001166C1821306F6EF8D476365D60297E76C
:105A9000FF1F938767929C4B17E6FF1F0346366BE9
:105AA0009386C7002DC203D607006DCE8907E39CFD
:105AB000D7FE89471307A0F8114697E5FF1F938586
:105AC000E568268597E6FF1F2382E66817E7FF1F34
:105AD000A30FF76697E0FFFFE780C0352A846305D0
:105AE00005FA97B501009385A52C17B5010013059C
:105AF00065B197900100E780E050A28517B50100DD
:105B000013054517EDB203D607006302E60E8907B9
:105B1000E39BF6FE8D4779BF91476304F40297B586
:105B200001009385E52817B501001305A5AD9790F1
:105B30000100E780204D17B50100130525156FF012
:105B40008FF3B7E70400FC4F9305000817E5FF1F2C
:105B5000034545D18297D1B8854763F787F22685FB
:105B600097F0FFFFE78000669305F4FFC205C1814F
:105B70001305190097E0FFFFE78020396FF0CFF0A1
:105B800097B501009385C52217B50100130585A7B8
:105B900097900100E780004717B50100130585E5E0
:105BA0006FF06FED2390E70017E5FF1F1305C58029
:105BB00097200100E780807197B501009385451F0C
:105BC00017B50100130505A497900100E7808043F5
:105BD00017B501001305050D97900100E78080427D
:105BE000294597900100E780C0468147E1B52390A1
:105BF000070017D5FF1F1305257C97200100E780BC
:105C0000E06C97B501009385A51A17B5010013053F
:105C1000659F97900100E780E03E17B501001305EE
:105C2000E5095DBF011126CA06CE22CC4AC88347CA
:105C30000500AA849DC797B501009385251317B564
:105C400001001305259C97900100E780A03BCC4004
:105C500017B501001305054597900100E780803ACC
:105C600025A25841B707CF009387777D631DF70CB6
:105C700000450359C50085470356E5000347040066
:105C800063FA27098346140093178700D58FC2074C
:105C9000F176C1879386C655639AD712970700207D
:105CA00083D7A7AA638CC71422856244F240D244EA
:105CB000CA854249056117D3FFFF670063529547C4
:105CC00063FA2705930730056316F704834614002B
:105CD000930750046390F60483462400930710044E
:105CE000639AF602834734006396E7020347440051
:105CF0009307B0046310F70203475400930790051D
:105D0000631AF700328597F0FFFFE780A04BCA8542
:105D10002285E1A89707002083D727A3638AC700BD
:105D2000CA85228532C697D0FFFFE780604B324696
:105D300022856244F240D244CA854249056117F384
:105D4000FFFF6700C34BB707CC009387777D6317CE
:105D5000F70497B501009385650117B50100130598
:105D6000658A97900100E780E0299C4483D6E4008F
:105D700083D5C40003C6070017B501001305053419
:105D800097900100E78000286244F240D2444249E3
:105D900029450561179301006700A32BB707CE00C3
:105DA0009387777D630CF70497B50100938505FC15
:105DB00017B501001305058597900100E780802441
:105DC000CC4017B501001305E52379B59307100BF7
:105DD000E317F7EE328597F0FFFFE780A03E9305CB
:105DE000F9FFC205C181130514006244F240D24498
:105DF0004249056117E3FFFF67002311F240624447
:105E0000D24442490561828097E7FF1F83C707306C
:105E1000B9C397E7FF1F238B072EB7E70400FC4F9A
:105E2000411122C406C62A849305002017E5FF1FEE
:105E3000034545A38297854711C897E7FF1F9387BE
:105E4000072D83D707002310F4008547B240224472
:105E50003E85410182803E858280411106C697E0E1
:105E6000FFFFE78020FD0DC197E7FF1F83D7E723E2
:105E7000850717E7FF1F231AF72297E7FF1F2397CE
:105E8000A722B2404101828097E7FF1F83D72722D4
:105E9000850717E7FF1F231CF720E5B7411122C430
:105EA00091462A8417E6FF1F130646389D652D4547
:105EB00006C697D0FF1FE780C092B7F7070003C759
:105EC0000701A5476313F70001A0930600100146E0
:105ED0009D65254597D0FF1FE780A09097E7FF1F9E
:105EE000238687342244B240914617E6FF1F1306EB
:105EF000E6339D652945410117D3FF1F6700638E77
:105F00001171CED7B7E9040083A7C904CAD917E92C
:105F1000FF1F1309A923A2DD2E8686DFA6DB2E84B0
:105F2000AA854A85829797E7FF1F83C72722130711
:105F3000700A6385E710636DF7001307600A6385D5
:105F4000E704FE506E54DE544E59BE5911618280F2
:105F50001307800A6385E7161307900AE393E7FEA9
:105F60008D476306F41C97B501009385A52017A5FE
:105F700001001305256997900100E780A00817B577
:105F800001001305651C25A08D47630CF40297B52D
:105F900001009385251E17A501001305A56697909E
:105FA0000100E780200617B501001305251397901F
:105FB0000100E7802005294597900100E7806009EE
:105FC00049B7854717B501001305051317E7FF1FEC
:105FD000230CF70C97900100E780A01AB775020018
:105FE000B76602000146054597C0FF1FE780607F46
:105FF000930760F817E7FF1F230AF71497E7FF1FBF
:10600000A38707149307002617E7FF1F2322F7141F
:10601000E5779387072117E7FF1F231DF712B14587
:1060200097E7FF1F2389071297E7FF1FA385A71292
:106030004A8597000000E780E01621B7914763E3A7
:10604000870297B501009385E51217A50100130596
:10605000655B97900100E780E0FA17B50100130532
:10606000A50BB1B797E4FF1F83C4840E97E7FF1F0A
:1060700083C7F70DA204DD8C83A7C9046D142286A3
:1060800097E5FF1F9385D50C280082978E04931601
:106090000401B7750200C1823000A695094597C07A
:1060A000FF1FE7800074930770F817E7FF1F230FA7
:1060B000F708994597E7FF1FA38CA70895BF91475D
:1060C00063E3870297B501009385C50A17A5010010
:1060D0001305455397900100E780C0F217B5010002
:1060E00013050505E9B597E4FF1F83C4640697E728
:1060F000FF1F83C7D705A204DD8C83A7C9046D14D5
:10610000228697E5FF1F9385B504280082978E04A9
:1061100093160401B7750200C1823000A6950D45A3
:1061200097C0FF1FE780E06B930780F8BDBF17B5EE
:1061300001001305A50297900100E78080049307F2
:1061400090F82304F100834719008D452800A3042B
:10615000F100834729002305F10097000000E78044
:1061600060041305C01297C0FF1FE780801D014522
:1061700097D0FFFFE78040F20D4597000000E780D1
:1061800020D2294597C0FF1FE780A01B97C0FF1FA3
:10619000E780000C7DB397E7FF1F23A1A70A828049
:1061A00097E7FF1F9387870903A307006303030093
:1061B000028317430000670043C241114AC097F6AB
:1061C000FF1F83D68658328917D6FF1F0356E62055
:1061D00022C426C206C62A84AE8497000000E78047
:1061E000406829C921C8994763F69704834714007A
:1061F00003470400A207D98F13978700A183D98F83
:10620000C2073167C1831307C7556395E70297D764
:10621000FF1F83D7871CA301F400A1832302F4008E
:1062200097F7FF1F83D7675291C7A302F400A1839A
:106230002303F40097F7FF1F83C7C740A1CB26862F
:10624000A28517D5FF1F0355451997000000E78069
:1062500000C1630F090297F7FF1F83C7A73E8DEBAD
:1062600097E7FF1F83C7C7FD85C79DC097E7FF1F3F
:1062700083C787E391EF22852244B2400249A68575
:106280009244410117430000670023B5E31A09FC5B
:10629000B240224492440249410182808347550022
:1062A0008345450017B50100130585EFA207DD8D75
:1062B00017930100670003D517B50100130545EDDD
:1062C000179301006700E3EB8D4763F6B7080111F0
:1062D00026CA06CE22CC0344350097E4FF1F83C4B0
:1062E00034F697B501009385E5ECB337800017E7E6
:1062F000FF1FA307F7F409C497B50100938545EC88
:1063000017B50100130545EC97900100E78080CF99
:1063100097E7FF1F83C7D7F26386970097000000B7
:10632000E780004397400000E78020DA9967938771
:1063300057EE2316F100680085479145A3078100B9
:106340002307F10097000000E780C0E5F2406244B7
:10635000D244056182808280894763F7B7080111C2
:1063600022CC06CE26CA8344250085472A84639D15
:10637000F404914763F5B7040345450083473400AF
:1063800022055D8D97D7FF1F2399A7049700000072
:10639000E78000569967938767EE2314F1008347DF
:1063A000340023059100A305F1008347440095457F
:1063B00028002306F10097000000E780A0DEF240ED
:1063C0006244D24405618280FDF89967938767EE45
:1063D0002314F10097D7FF1F83D72700A305F100EF
:1063E00023050100A183E1B782800111996722CCC6
:1063F000D51717F4FF1F1304E4242314F100834777
:10640000040026CA97F4FF1F938424342305F10067
:1064100083D7040028009545A305F100A18306CE8B
:106420002306F10097000000E780C0D703D60400E0
:106430008345040017B50100130505DA97900100A4
:10644000E78040BCF2406244D244056182809D678F
:106450007971D9172316F10097F7FF1F9387871ECD
:1064600083C707001305F10006D62307F10097F054
:10647000FFFFE78040CE09E9B7E70400BC4741468B
:1064800081451305F10082976800CD459700000013
:10649000E78040D197F5FF1F83C5C51A17B50100E6
:1064A000130585D697900100E780C0B5B2504561CD
:1064B000828063080516411126C206C622C44AC05E
:1064C00097E7FF1F83C7D7D797F4FF1F83C48417AD
:1064D00099C393E424002A8497100000E78020E306
:1064E00019C193E4040137E9040083278904228554
:1064F0001306200381458297930750FA2300F40086
:106500009307A005A300F4008D472301F4009147F1
:10651000A301F4009307F004A302F40097F7FF1F10
:1065200083D7A7222304F400A183A304F40097D700
:10653000FF1F83D787EA230394002305F400930405
:10654000C400A18323020400A305F400268597F06C
:10655000FFFFE78040C019E5832789044146814554
:106560002685829797D7FF1F83D7C7E4230EF400B1
:10657000A183A30EF40093070002230FF4009307F6
:1065800010FAA30FF4009D472300F402A3000402B5
:10659000B7E70400FC4713052402194697D5FF1FEF
:1065A0009385852C829797E7FF1F83D747B02304F5
:1065B000F402A183A304F40297E7FF1F83D7E7AE99
:1065C0002305F402A183A305F40297E7FF1F938735
:1065D000E7AD839707002285930500032306F402A5
:1065E000C207C183A183A306F40297D7FF1F938735
:1065F00027CD839707002307F402C207C183A18335
:10660000A307F40297000000E780A0212308A4025A
:106610002181A308A402B2402244924402494101CC
:10662000828082805D71E17793C777FF1305E10077
:1066300086C62316F10097000000E780C0E76800D7
:106640009305400397000000E780C0B5B640616144
:1066500082805DC9411122C426C206C6930750FA42
:106660002300F5009307A005A300F5008947230147
:10667000F5009147A301F5009307F004A302F5008C
:1066800097F7FF1F938707FC83C707009304C50094
:106690002A842303F50097E7FF1F938777BA83C700
:1066A000070023020500A303F50097F7FF1F83D718
:1066B000C7092304F500A183A304F50097D7FF1FA2
:1066C00083D7A7D12305F500A183A305F50026856F
:1066D00097F0FFFFE78020A801E9B7E70400BC4777
:1066E00041468145268582972285F1459700000025
:1066F000E7802013230EA4002181A30EA400B24042
:10670000224492444101828082805D710A8586C65E
:10671000A2C497000000E78000F437E404007C4442
:106720008A850810794682973C441305E10309469F
:1067300081458297101093050002014597D0FFFF15
:10674000E780C0FBB6402644616182800111B7C773
:10675000A55A22CC9387C73317E4FF1F130454AE06
:106760003EC483470400856601469965254506CEEB
:106770003EC697C0FF1FE780C0063000A14699655E
:10678000294597C0FF1FE780C0058345040017B562
:1067900001001305E5B197900100E780A086F24063
:1067A0006244056182800111A146300099652D4542
:1067B00022CC06CE97C0FF1FE780A002A24737C4B5
:1067C000A55A1304C43363958702B24517B5010077
:1067D0001305C5A5B335B00097E7FF1FA382B7A681
:1067E00097900100E7800082F24062440561828058
:1067F0009165A1463000938505F02D4597C0FF1F98
:10680000E78020FEA247E38287FC97E7FF1FA3896A
:1068100007A2814517B50100130585A3D1B7C1674C
:1068200069768146FD170506139706014183636467
:10683000B7003E8582803307D50003470700B98F34
:10684000214713F81700858363050800B18FC2073D
:10685000C1837D171377F70F6DF78506F1B741C533
:10686000A547054763F2B7088347150003470500AE
:106870003168A207D98F13978700A183D98FC207E8
:10688000C1831308C855054763900707411106C621
:1068900022C426C203442500914763F0870493076E
:1068A000540063ECF502A301C50021822302C50058
:1068B0009304340091C6A302D500A1822303D5001E
:1068C0002A84A68597000000E780A0F5269423007F
:1068D000A4002181A300A4000147B24022449244B5
:1068E0003A854101828005473A8582800111B7C708
:1068F000A55A22CC9387E7342A842AC685660146A6
:106900009565254506CE3EC497C0FF1FE78060ED24
:106910003000A1469565294597C0FF1FE78060ECD0
:10692000A28517B501001305A59A97800100E7809D
:10693000606D97000000E78080DDF24062440561F1
:1069400082800111A146300095652D4522CC06CEEE
:1069500097C0FF1FE780E0E8A24737C4A55A130499
:10696000E43463958702B24517B5010013054590DD
:1069700097D7FF1F2393B7A6C205C1819780010057
:10698000E7804068F2406244056182809165A146DB
:106990003000938505EE2D4597C0FF1FE78060E42A
:1069A000A247E38287FCD14717D7FF1F2317F7A21F
:1069B000D14517B501001305A58DC9B7011122CC2A
:1069C0002A841305E10026CA06CEAE8497F0FFFFA5
:1069D000E780C04309C90355E1002686A28597F0E8
:1069E000FFFFE780C047A685228597100000E7805B
:1069F000A09297E7FF1F83C7A78499C7A685228522
:106A000097300000E780603DF2406244D244056167
:106A1000828001114EC606CE22CC26CA4AC893F700
:106A20001500AE899DCBAD67371700409387A7AAA5
:106A30001CC3B7E70400BC4F13060019854517D5E2
:106A4000FF1F03456599829713C51900F240624400
:106A5000D2444249B2490561828093F7250001453D
:106A6000F5D717F7FF1F035727CE954763FAE70CB3
:106A7000014417F6FF1F130626BD930630051305C4
:106A80005004130810049308B004130390059307EF
:106A900064006374F7043A847D5997F4FF1F83C43C
:106AA000A4BA97F7FF1F83C737BAA204DD8CAD677E
:106AB0009387B755638CF41463E4970AA9679387A7
:106AC000A755638FF414A28517F5FF1F1305C5B7EB
:106AD00097000000E780C0EEF1A0B307860083C5F1
:106AE0000700639BD50483C517006397A50483C57E
:106AF00027006393050583C53700639FD50283C5CF
:106B00004700639B150383C7570063976702228979
:106B100015E897F5FF1F83D525C3B3852541C20529
:106B2000C181F1CD17F5FF1F130505B24A959700F6
:106B30000000E780E0E8E1A005044204418081BF55
:106B40003A847D598547E3EA87F45DC4854517F5A6
:106B5000FF1F130565AF97000000E78060E669A896
:106B6000B1679387C7556389F404B5679387D75591
:106B7000E39BF4F4A28517F5FF1F1305E5AC9730EE
:106B80000000E78080258947630EF4009305E4FF49
:106B9000C205C18117F5FF1F130525AB9700000043
:106BA000E7808077A68517A50100130525749780D7
:106BB0000100E780204589A097200000E78040176A
:106BC00097000000E780A07411C9A28517F5FF1F88
:106BD000130585A797000000E78000740546A2858D
:106BE00017F5FF1F130545A697F0FFFFE780205D0F
:106BF00097200000E780C013FD57E31CF9F097F7DA
:106C0000FF1F239307B413C5290089B5A28517F583
:106C1000FF1F130565A397F0FFFFE780606859B772
:106C2000A28517F5FF1F130525A297F0FFFFE78048
:106C3000E0688DBF411122C437E404005C5C06C6E5
:106C4000354697A501009385E52117B50100130589
:106C5000A5F1829711E917A501001305656A9780D0
:106C60000100E780005201A08327041C82972A8438
:106C7000054597C00000E780400597700100E78058
:106C8000608A97600100E780605F97B00000E7804E
:106C9000C0162285B240224441018280411105453F
:106CA00006C622C426C297C0FFFFE780C02813058E
:106CB000A00497B0FF1FE780803F757585457D155F
:106CC00097C0FFFFE78060127D7585451305F53697
:106CD00097C0FFFFE780C01B371400408327840A5A
:106CE0008D451305002093E707202324F40A97C05D
:106CF000FFFFE780800FB7E4040097C0FFFFE78045
:106D0000A054C85897800100E780A04717B501003C
:106D1000130585E597800100E780A0468327840C52
:106D20008545414593E707082324F40C97C0FFFFEE
:106D3000E78000168D451305000897C0FFFFE78028
:106D4000201597C0FFFFE780004237A50700130515
:106D5000051297C0FFFFE780A03D014597C0FFFFE8
:106D6000E780C04395450545894717F7FF1F230F67
:106D7000F79C97C0FFFFE7800044B7E700E01307E8
:106D80000006238DE7403707000423A0E71097D0C3
:106D9000FFFFE78080C597D0FFFFE78080D797008F
:106DA0000000E78060E997000000E78000A09700FE
:106DB0000000E78040B997E0FFFFE78020CF970011
:106DC0000000E780A05697000000E780801083A7AE
:106DD000040817050000130505C4829797C7FF1F15
:106DE000238CA75EBC4C130600648545829797B040
:106DF000FF1FE780E05F01458280AD6737170040E5
:106E00009387A7AA1CC3B7E700E03707400023A079
:106E1000E71801000100B7F7070003C70701A547FE
:106E20006316F7009397450191C301A04111AE8607
:106E30000146AA85254506C697C0FF1FE780609AD0
:106E4000B240B7E700E03707400023A0E710410158
:106E500082804111B2862E86AA852D4506C697C02E
:106E6000FF1FE7800098B2400145410182809307EF
:106E7000000463ECC7041D71A2CC2A840808A6CACA
:106E8000CAC886CE32C697800100E780400CAD6745
:106E9000371700409387A7AA1CC3B7E400E037095F
:106EA000400023A0241901000100B2461008A28569
:106EB000294597C0FF1FE780C092F640664423A093
:106EC0002411D6444649256182803955828041117A
:106ED0000D658D4506C697C0FFFFE78000F1B71727
:106EE00000408D6623A6D70A17F5FF1F13054586B8
:106EF0001387C70A9387870A1CC15CC585668967A3
:106F00005CC958C114C518C9B7E70400B24003A34F
:106F1000871E410102838145B307B50083870700BF
:106F200089E717230000670043E78505C205C18193
:106F3000E5B7011106CE2307010001ED17A50100F9
:106F40001305055E97000000E78020FDF240056113
:106F500082805800A947BA8529462548B376C502DC
:106F6000FD1793F7F70F93860603A304D700B356D4
:106F7000C5026375A8007D173685EDF33385F500EE
:106F8000D1B797A701009387E7591357C5003E97DC
:106F900003470700011106CE2304E10013578500C3
:106FA0003D8B3E970347070023060100A304E10041
:106FB000135745003D8B3D893E97AA97034707002D
:106FC00083C7070028002305E100A305F10097000F
:106FD0000000E78080F4F24005618280797117A596
:106FE00001001305254D06D622D426D24AD04ECE16
:106FF00097000000E78060F217E5FF1F0355E57476
:1070000097000000E78020F897E7FF1F83C787639A
:1070100017A501001305854789C717A501001305AA
:10702000654697000000E78040EF17A501001305B3
:10703000A54897000000E78040EE17A50100130562
:10704000254897000000E78040ED114597000000BB
:10705000E78060EE17B50100130505A59700000055
:10706000E780A0EB014597000000E780C0EC17B572
:107070000100130565A397000000E78000EA1305EF
:10708000F00497000000E78000EB97D7FF1F83C74D
:10709000371B17A501001305E53F89E717A5010078
:1070A0001305C53F97000000E78020E717A5010002
:1070B0001305854197000000E78020E637A507000B
:1070C0001305051297000000E780E0E617A5010010
:1070D0001305054097000000E78020E497E7FF1FB5
:1070E00083C7876817A501001305C53B89E717A566
:1070F00001001305A53B97000000E78000E217A5FB
:1071000001001305A53D97000000E78000E117A5E9
:1071100001001305253D97000000E78000E017A55A
:1071200001001305A53C97000000E78000DF17C5AC
:10713000FF1F0355252897000000E780C0E417A52E
:1071400001001305E53A97000000E78000DD17C550
:10715000FF1F0355852897000000E780C0E217A5B0
:1071600001001305653997000000E78000DB17D5A3
:10717000FF1F0355C5F397000000E780C0E017A587
:1071800001001305E53797000000E78000D917D507
:10719000FF1F035585F197000000E780C0DE17A5AB
:1071A00001001305653697000000E78000D717D56A
:1071B000FF1F0355A5EF97000000E780C0DC17A56F
:1071C00001001305A53497000000E78000D517C51E
:1071D000FF1F0355E50E97000000E780C0DA17A5F2
:1071E00001001305253397000000E78000D3014418
:1071F00097C9FF1F9389496797A40100938484323C
:107200001949B307340183C707000A85050413D75A
:107210004700BD8B2697A6970347070083C7070043
:10722000230101002300E100A300F100970000000A
:10723000E780A0CEE31724FD17A501001305052E56
:1072400097000000E78060CD0A8597E0FFFFE780A8
:1072500080F00A84040883470400034514000904ED
:10726000A2075D8D97000000E780E0D1E39584FEE2
:10727000B250225492540259F24945618280411120
:1072800026C2E97797E4FF1F9384045D22C49387A5
:10729000A7552E842381B4002E86AA8517E5FF1FEB
:1072A0001305C55B06C62390F400A38104009780F4
:1072B0000100E780C0C993052400C205C18117E51C
:1072C000FF1F1305855997F0FFFFE7808055B387AF
:1072D00084002382A7002181A382A7009305640074
:1072E0002244B24026859244C205C1814101172340
:1072F0000000670083AA09C99307000463E6B7008A
:10730000170300006700E3F7828017E5FF1F0345BE
:10731000A545828097E7FF1F83C7C75389E71723D7
:107320000000670083A7828097E7FF1F83C7275766
:1073300099EF411106C697200000E780E09DB2401A
:10734000854717E7FF1F230CF75441018280828095
:107350006307053E6385053E1D71CAC8CEC686CE4D
:10736000A2CCA6CAD2C4D6C2DAC05EDE62DC66DABD
:107370006AD86ED6B947AA892E8963F9B706394605
:1073800097A50100938585FE97800100E780C0B92D
:1073900031ED83C7E900130710036394E7028547C3
:1073A00017E7FF1F2308F74A17A50100130505FD7E
:1073B00097E7FF1F239F074897000000E780E0B58D
:1073C000E5A01307000317A50100130525FEE395AB
:1073D000E7FE97E7FF1F238F074697E7FF1F239AD4
:1073E000074617A501001305E5FAF9B797E7FF1F50
:1073F00083C74746639F0728B706400001475946A1
:10740000A50613140701418063742433B384E90093
:1074100083C70400D91793F7F70F6367F600B3D754
:10742000F600858B0507F1FF330489404204418053
:10743000BD4763FE8726414697A50100938545F920
:10744000268597800100E78020AE6314052617A5E6
:107450000100130525F997000000E78000AC9700B4
:107460000000E780E0B7179501001305657AA9B71A
:10747000B387490183C6070097E7FF1F83D7673D9E
:10748000B9E39307A005639BF600854717E7FF1F45
:107490002311F73C97E7FF1F238AD72C050A931780
:1074A0000A01C183E3E627FDF6406644D644464917
:1074B000B649264A964A064BF25B625CD25C425D54
:1074C000B25D25618280854D639BB7039307500AA7
:1074D000639EF600894717E7FF1F231CF7369307C3
:1074E00050FA17E7FF1FA303F7284DBF9307A00526
:1074F000E386F6FA97E7FF1F239D073445B7138706
:1075000017004207DA9741832380D70017E6FF1F51
:107510002311E6348D47E3F3E7F817E4FF1F034434
:10752000142597E7FF1F83C7872422045D8C9307E8
:10753000F4FFC207C1839306F00DE3EDF6FA93075B
:107540006400C207C183E31BF7F493052400C2055E
:10755000C18117E5FF1F1305852197F0FFFFE78025
:10756000402C33078B008347570003474700A2078F
:10757000D98F17E7FF1F231E072C6311F5108144D5
:10758000630CB40197E4FF1F83C4841EA20497E731
:10759000FF1F83C7F71DDD8C170500001305E5D518
:1075A00097F0FFFFE78060BF6385740963EF9B027C
:1075B0006388A4059307EC656383F40697E7FF1FD0
:1075C00083C7071B05476380E70881CB1387A7059F
:1075D0001377F70F8D4663F9E6081307F0072300CA
:1075E000E100A300F100894595A86389940593877C
:1075F000FA77E395F4FC97F0FFFFE780E00211A82B
:10760000A28517E5FF1F1305A51697F0FFFFE7807A
:10761000E0CB014597F0FFFFE78020B841B5A28598
:1076200017E5FF1F1305C51497F0FFFFE78000D390
:10763000CDB797F0FFFFE78080DBE1BF97F0FFFF5A
:10764000E78020E1F9B7930710F813051100230034
:10765000F10097F0FFFFE7800000FD450A859700E5
:107660000000E78000C275B7A28517E5FF1F13056C
:10767000251097F0FFFFE780E08861BF9307F007D0
:1076800089450A852310F10097000000E78060BF5C
:1076900031B5BD6A396C014A17EBFF1F130B0B0D97
:1076A000938BFA55938CFA66130DEC55CDBB631191
:1076B000F4083D4697A50100938505D4268597805B
:1076C0000100E780608611E517A501001305C5D309
:1076D00059B3C14763FE8704414697A501009385CE
:1076E000E5D3268597800100E780008431E183C7D8
:1076F000040113071003639CE700854717E7FF1F8A
:107700002304F70617A50100130585D275B11307E9
:10771000000317A501001305A5D4E39FE7C897E769
:10772000FF1F2383070417A501001305E5D169B1E5
:10773000CA854E8597C0FFFFE78080AAB5B38280D7
:10774000411126C2AE848D4522C406C62A8497B054
:10775000FFFFE780E073B717004099C803A5C70C87
:10776000418D23A6A70CB24022449244410182805D
:1077700003A5870C418D23A4A70CF5B7834705000B
:1077800003471500A207D98FC2076177C187130786
:107790002720639AE7008345250037050400170377
:1077A0000000670023FA828017E6FF1F1306860F8A
:1077B0008147B2861303F00FA9483308F600034847
:1077C000080013F7F70F6307A80C63066800850726
:1077D000E39517FF2947B387E6002380A70097E7C3
:1077E000FF1F9387E70C5DA8411113D7650013476E
:1077F000170006C693F63500058B954791CA0546D6
:1078000099476387C60009469D476383C600A14721
:1078100013F645003336C00093F68503050685C28E
:10782000A145638BB604E145638AB60493058002E3
:107830006388B604930580036393B600914697E589
:10784000FF1F238CF52C97E5FF1F2387C52C97E599
:10785000FF1FA383D52CBE8517A50100130585D076
:1078600097700100E780007AB240854717E7FF1F55
:10787000A305F72A410182808546D1B78946C1B761
:107880008D4675BF17A50100130545D0177301007C
:107890006700437717E7FF1F13078701BA97238015
:1078A000B700E147E302F5F493077002E30CF5FC3F
:1078B00082802A8723800500814717E5FF1F130573
:1078C00065FE1308F00F2946B306F50083C60600CF
:1078D0006396E60297E6FF1F938686FDB69783C7F9
:1078E000070005452380F5009947636EF7029D4721
:1078F00063FDE700E147630DF700828063850601C1
:107900008507E393C7FC0145C5B723800500828046
:10791000B737004003C7370083C7050093F7070454
:10792000D98F2380F50082805D7152DC56DA5ED6F5
:10793000716A97EBFF1F938B6B2F8D6AA6C24EDE89
:1079400062D486C6A2C4CAC05AD866D26AD06ECEE5
:10795000C1495E8C97E4FF1F938444F6130A0A2002
:10796000938A7ADC17E9FF1F0349492FB3872B015C
:1079700083C7070093F7F70FC9EFB787004003C726
:107980006700058BE310077C03C76700118BE30DCD
:10799000077E83C75700918B99E36F10200317E789
:1079A000FF1F0347C72B85476304F7006F10400193
:1079B00097E7FF1FA383E71697E7FF1F238007FCC6
:1079C00097E7FF1F238E070697E7FF1F238C0712F9
:1079D00097E7FF1F2389071297E7FF1FA38007FA86
:1079E00097E7FF1FA38E070497E7FF1FA38C0710DD
:1079F00097E7FF1FA389071097E7FF1FA3800712D0
:107A000097E7FF1FA38D0724B787004011476F003A
:107A100070779307190093F7F70F3D476364F706F4
:107A200017E7FF1F230CF72297E7FF1F9387072213
:107A3000CA9783C707001307100293F7F703638EF3
:107A4000E71E6366F70405446385871CE38C0762C1
:107A50000947638EE71013070002E384E74EB7E798
:107A600000E03707400023A0E718010001006299F9
:107A700023000900FD1923A0E71093F9F90FE39300
:107A800009EEE5BD97E7FF1F238A071C71BF1307A7
:107A900030026388E70C63E8E71613074002638C43
:107AA000E70A13070003E39CE7FA97E7FF1F9387B2
:107AB000E718CA9703C70700A1471377F70FE31B1F
:107AC000F71483C7640097E6FF1F238FF60297E73A
:107AD000FF1F83C717DF91C7FD5797E6FF1F238559
:107AE000F60297E5FF1F83C575DD97E7FF1FA38D9E
:107AF000B70097E7FF1F83C767DC13FB07089306F0
:107B0000000493F70706639FD74C9307A009638D82
:107B1000F51663EAB7129307F0056386F54A9307F3
:107B200050096384F52A014497E7FF1F83C7D7FDF7
:107B30001547E392E736B7E700E03707400023A098
:107B4000E71801000100B786004023808602130673
:107B500080FC6F00500EFD5717E7FF1F2305F7FA53
:107B6000FDBDFD5717E7FF1F230EF7F8CDBD17A585
:107B70000100130525B397700100E780806097E747
:107B8000FF1F9387A70BCA9703C40700014B97EC0D
:107B9000FF1F938C2CEB1374F40F17AD0100130D22
:107BA000EDB063478B04294597700100E780604A78
:107BB000854717E7FF1FA305F7E817E7FF1F230215
:107BC00087E817E7FF1F230BF7F437E700E0B70656
:107BD00040002320D718010001003786004083476A
:107BE000A60293F7370F2305F6022320D71085BD91
:107BF000B3876C0183C507006A85050B9770010088
:107C0000E780404079BF854717E7FF1F230AF7E267
:107C1000B9B517E7FF1F130767024A970347070025
:107C200097E6FF1FA38CF6D497E6FF1F2389E6D4BF
:107C300017E7FF1F2304F7EE1DB5854717E7FF1F62
:107C4000230EF7D229BD9307400A6389F5349307C1
:107C5000200B6384F5369307100AE396F5EC8387CF
:107C600024000144E3D207EC97E7FF1F83C737C521
:107C700093F63700638A061A0546638AC6220946C8
:107C80006395C61A1D4755A217E5FF1F034525C377
:107C9000C94797ECFF1F83CC9CC297E5FF1F83C5A4
:107CA00025C217E4FF1F0344B4C16315F510CD4787
:107CB0006392FC1093077008639CF5021307300F62
:107CC000B7170E006308E4001307900DB7B7040060
:107CD0006314E40817E7FF1F232EF7E2BE8517A5FC
:107CE00001001305259D97700100E780A03125BD97
:107CF00093078008639DF500B307804013F4F70FE6
:107D0000B7774600938787CDB3D78702E1B793074C
:107D10009008639AF500B307804013F4F70F91675A
:107D20009387C766D5B79307A008639BF500B30791
:107D3000804013F4F70FB7173D0093870790E9B71A
:107D40009307B008639AF500B307804013F4F70F68
:107D50009167938797D04DBF93F5F5078D47639B48
:107D6000F500B307804013F4F70FB7975B009387D4
:107D700007D859BF8947639BF500B307804013F4C8
:107D8000F70FB7770B009387071BBDBF8547639A33
:107D9000F500B307804013F4F70FDD67938767E3BF
:107DA000A5B7D28785F9B307804093F7F70FB3D70C
:107DB000FA020DB797000000E780409FA285668514
:107DC00097000000E780809EB9BB9305610017E52E
:107DD000FF1F0345C5AE17E4FF1F034454AE9700D1
:107DE0000000E78040AD93057100228597000000F8
:107DF000E78060AC3C0017E7FF1F2327F7E28347CB
:107E000061002304F10083477100A304F100894756
:107E100017E7FF1F230AF7CE8357810017E7FF1FDD
:107E2000231EF7A8094409B3154793F64700B33654
:107E3000D00093F78703850685C32146638BC70669
:107E40006146638AC706130680026388C706130665
:107E500080036393C700914717E6FF1F230ED6CA1E
:107E600097E6FF1FA38AF6CA97E7FF1F2387E7CA93
:107E700017E7FF1F0347C7A49376070497E7FF1F81
:107E800083C717A48DEE1377770C93067008630CE5
:107E9000D7021377F7078D466312D70CB307F0406C
:107EA000B7955B0093F7F70F938505D849A8194755
:107EB000ADBF854755B7894745B78D4771BF930615
:107EC00070086311D7021307300FB7150E006389CE
:107ED000E7021307900DB7B504006383E7021307A9
:107EE000700845BF9306800C6311D702B307F040BA
:107EF000B775460013F7F70F938785CDB3D5E70223
:107F000097E7FF1F23A8B7C0D9BB9306900C631C4B
:107F1000D700B307F04093F5F70F91679387C766D3
:107F2000B3D5B702F1BF9306A00C631DD700B3070A
:107F3000F040B7153D0093F7F70F93850590B3D543
:107F4000F5027DBF9306B00CE315D7F4B307F040FC
:107F500093F5F70F9167938797D0D9B78946631B3D
:107F6000D700B307F040B7750B0093F7F70F938571
:107F7000051BF1B78546631AD700B307F040DD65EE
:107F800093F7F70F938565E35DBFD28535FBB305A6
:107F9000F04093F5F50FB3D5BA029DB783C724001F
:107FA000C18B99C7854717E7FF1F2302F7B6A5BE08
:107FB00097E7FF1F238D07B4BDB6854717E7FF1F5F
:107FC000A30DF7B48DB63C0017E7FF1F232EF7C4AF
:107FD0000947930700032314F10097E6FF1F238549
:107FE000E6B22DBD63940756A94763E5B7421797DC
:107FF0000100130767548A05BA959C41BA97828796
:1080000017E4FF1F0344B48B894C6306940D63E6A9
:108010008C0685476303F4089307F00F17E7FF1FEB
:10802000034787AE63F6E70017E7FF1F230EF7ACA1
:1080300097ECFF1F83CC4CAD9307000413F4FC0FA7
:1080400063F497011304000497E7FF1F9387C7BDEC
:1080500003AD070022862685EA85B38C8C40229DDD
:1080600097700100E780A0EE97E7FF1F238E97A986
:1080700097E7FF1F23AAA7BB45BC8D47630CF40AF3
:108080009947E31BF4F8979701009387675117E727
:10809000FF1F232BF7B8A94751B717E7FF1F034767
:1080A00007BC97E7FF1F938727A8494697950100CC
:1080B000938505586306870097950100938545537E
:1080C0003E8597700100E78080E817E7FF1F232DAA
:1080D000A7B4C947A1B797E6FF1F83C646B80547AF
:1080E00097E7FF1F938747A46394E6023E85130634
:1080F0007002979501009385255197700100E780E4
:1081000000E517E7FF1F2321A7B29307700239B7D5
:108110003E85130630049795010093852549977095
:108120000100E780C0E217E7FF1F232FA7AE9307E8
:108130003004EDB597D5FF1F83C56578179501000D
:108140001305855897700100E780C0EB054D97ED4A
:10815000FF1F83CDCDB097D5FF1F83C545761795FB
:108160000100130565566398AD0B97700100E78019
:1081700060E997D7FF1F83C78774B5CBE36EF4E838
:10818000179401001304044F638CB7011794010086
:108190001304C44E63869701179401001304844F9F
:1081A000228597700100E78000FF1375F50F930794
:1081B0001500860717E7FF1F2308F7968D4717E777
:1081C000FF1FA303F79697E7FF1F9387E7950147E4
:1081D000BE861376F70F89076365A60297E7FF1F30
:1081E00023A4D7A497E7FF1F83C7079405BD9797DC
:1081F00001009387274117E7FF1F2327F7A2914725
:1082000031BD3306E40003460600A38007000507DE
:108210002380C7007DBF97700100E780A0DE97D75D
:10822000FF1F83C7C769E1D7E368F4DE1794010035
:1082300013044441638CA701179401001304044103
:1082400063869701179401001304C4412285977037
:108250000100E78040F41375F50F930715008607BA
:1082600017E7FF1F2302F78C8D4717E7FF1FA30DAA
:10827000F78A97E7FF1F9387278B0147BE86137600
:10828000F70F8907E37CA6F43306E40003460600F3
:10829000A380070005072380C700D5B797D5FF1F28
:1082A00083C5E561179501001305C542977001006C
:1082B000E78040D597E7FF1F83C7D78693E747003E
:1082C00017E7FF1FA300F78683C7240017E7FF1FE8
:1082D000A308F78489B8179501001305E540977046
:1082E0000100E78000EA97E7FF1F9387678383C752
:1082F000070017D7FF1F2303F75C17E4FF1F034492
:10830000A480333480000DB0179501001305053F9C
:1083100097700100E780E0E697E7FF1F83C797802B
:1083200093E7070117D7FF1FA30EF77E83C724002B
:1083300017D7FF1F2306F77E6FF0EFFE179501009A
:108340001305053D97700100E780A0E303C7040013
:108350007D8B51EFB787004003C767021377C70BC8
:10836000136727002383E70203C7A7021377C70B0E
:10837000136727002385E70203C7E7021377C70BBC
:10838000136727002387E70203C727031377C70B69
:10839000136727002389E702854717D7FF1F230F9D
:1083A000F75C17D7FF1F230DF76817D7FF1F230BA5
:1083B000F77417D7FF1F2308F77497D7FF1FA38FF2
:1083C000075A97D7FF1FA38D076697D7FF1FA38B69
:1083D000077297D7FF1FA388077297D7FF1FA38F36
:1083E000077297E7FF1FA38C07866FF0CFF38947CB
:1083F0006312F70297D7FF1F83C7874C9146638CA0
:10840000D70863E0F604638EE70C6369F70A054753
:108410006380E70EFD5717D7FF1FA307F76E3707D7
:108420004000B7E700E023A0E71801000100B7868D
:1084300000401306F0FC2381C60223A0E7106FF072
:108440000FE2130720086382E7086362F70213074D
:108450001008E391E7FC378700408347670293F7F2
:10846000C70B93E727002303F7026FF0CFEB130747
:1084700030086389E70213074008E39DE7F8378770
:1084800000408347270393F7C70B93E7270023098F
:10849000F7026FF04FE9378700408347270393F7D0
:1084A0003707F5B7378700408347E70293F7C70BD5
:1084B00093E727002307F7026FF0EFE637870040C6
:1084C0008347E70293F73707F5B7378700408347BD
:1084D000A70293F7C70B93E727002305F7026FF076
:1084E0008FE4378700408347A70293F73707F5B734
:1084F000378700408347670293F73707ADB7179573
:1085000001001305E52197700100E78080C797D728
:10851000FF1F2385073AD5B31795010013054521A1
:1085200097700100E780E0C597D7FF1F23980738B1
:1085300097D7FF1F9387475D03C40700894763F3FD
:10854000870009441374F40F6FF00FDE1307000265
:10855000E392E7EC631B0B0A638FF500930720029D
:108560006383F50817950100130505209770010036
:10857000E78040A945B5179501001305251C9770A4
:108580000100E78000C00144179D0100130D4D1C40
:10859000A14CB387840083C507006A8505049770E2
:1085A0000100E78020A6E31694FF1785010013055C
:1085B000256C97700100E780C0BC17D4FF1F0344EF
:1085C000243001E897D7FF1F238C072C014B6FF055
:1085D000AFD58947E310F4E4854717D7FF1F230180
:1085E000F72C6FF04FD417D6FF1F0346562D97D5A3
:1085F000FF1F83C5C52C179501001305E51597705E
:108600000100E78020A06FF00FD26380F50693078A
:108610001002E399F5F497D5FF1F83C5652A1795D6
:1086200001001305651597700100E780A09D97D79D
:10863000FF1F23AB975E97D7FF1F9387A74D9443E8
:1086400083D7470017D7FF1F0347274D17D6FF1FB4
:108650002326D6261D4497D6FF1F2393F62697D7A9
:10866000FF1F2380E7266FF02FCC97D5FF1F83C510
:108670002525179501001305A51197700100E780C6
:10868000609897D7FF1F238D072097D7FF1F239749
:1086900007226FF02FF92547638FE7C89946378780
:1086A00000406394D70223008702B7E700E0B706D3
:1086B000400023A0D71801000100130600FC23018D
:1086C000C70223A0D7106FF08FB99306100A639FDB
:1086D000D70023008702B7E700E0B706400023A0D9
:1086E000D71801000100130680FCD1BF9306A00932
:1086F000E381D7FE9306400AE38DD7FC9306200260
:10870000639DD700B7E700E0B706400023A0D71865
:108710000100010023008702F9B78546E384D7FEF4
:1087200093070008E300FBFEB7E700E0B706400050
:1087300023A0D71801000100130620FC23008702A4
:10874000BDBF17D7FF1F0347373C6302F71E63E720
:10875000E70295476300F7109947630AF704B78665
:10876000004023800602B7E700E03707400023A05F
:10877000E718010001001306A0FC75B99307F00586
:10878000630AF700930750096306F7009307100286
:10879000E317F7FCB7E700E03707400023A0E7182E
:1087A00001000100B7860040130620FC69B117DB09
:1087B000FF1F034B6B35930700045A8D63F4670169
:1087C000130D000497D7FF1F9387074683AC07005C
:1087D0001374FD0F2286E685268597600100E780E9
:1087E0000077B3078B40669417D7FF1F230EF7302F
:1087F00097D7FF1F23AA8742B7870040630C0B025D
:108800002380A703B7E600E03706400023A0C61880
:108810000100010003C72702134707042381E70271
:1088200003C727021377C70F2381E70223A0C610CF
:108830006FF0EFA22380070237E700E0B7064000A1
:108840002320D71801000100130620FC2381C70252
:108850006FF0AFB9378700408347370097D6FF1FC7
:1088600083C6162C93F70708D58FA301F700B70628
:108870004000B7E700E023A0D7180100010013066D
:10888000A0FC35BD97D7FF1F9387473BCA9783C787
:10889000070093F7F70FC1CF97D7FF1F83C7273C78
:1088A000D9E717D7FF1F0347372693070002631046
:1088B000F70883AD040017DDFF1F034D6D0097DC43
:1088C000FF1F83CCFCFF17DBFF1F034B8BFFE687EB
:1088D0006A87DA866E8697D5FF1F83C565FC179574
:1088E0000100130565EC97600100E780A07197D740
:1088F000FF1F23A1B72397D7FF1F238FA72197D748
:10890000FF1FA38B972197D7FF1F2388672197D736
:10891000FF1FA38687F8B7E700E03707400023A0D2
:10892000E71801000100B78600406FF04FA2B7E7DB
:1089300000E03707400023A0E71801000100B786D8
:10894000004015BD97D6FF1F83C666310547639C5F
:10895000E60429472381E70209472383E7022385A9
:10896000E70297D7FF1FA38B071A97D7FF1FA3888C
:10897000072EB7870040A381070017D7FF1FA30169
:10898000071A05472383E700B64026449644064964
:10899000F259625AD25A425BB25B225C925C025D2F
:1089A000F24D6161828029472381E70209472383D1
:1089B000E7022385E7022387E7022389E70255B709
:1089C00017D7FF1FA30DF7EC6FE01FFF854717D7E1
:1089D000FF1F2305F7FA17D7FF1F2303F70617D743
:1089E000FF1F2301F71217D7FF1F230EF7106FE0A9
:1089F000BFFE854717D7FF1F2302F7F817D7FF1FC2
:108A00002300F70417D7FF1F230EF70E17D7FF1FFA
:108A1000230BF70E17D7FF1FA30207F617D7FF1F69
:108A2000A300070217D7FF1FA30E070C97D7FF1F3E
:108A3000A38B070C8280411106C697000000E780D7
:108A400080FBB787004023800700130740FC238684
:108A5000E7001307C004A386E70017D7FF1F13071B
:108A6000E7E52398E70017D7FF1F130727E9239AA5
:108A7000E70017D7FF1F1307A7F4239CE70017D7BA
:108A8000FF1F13072700239EE70029472381E702E2
:108A900009472383E7022385E7022387E702238927
:108AA000E702A3810700930600F8A380D70093068E
:108AB00090022380D700FD562383D7002381E7004F
:108AC0009306000537E700E0230BD740B7064000C8
:108AD0002320D71003C7170013671700A380E700F0
:108AE000B24097D7FF1F239D0702410182804111A9
:108AF00006C697000000E78000F0B787004023809B
:108B00000700130700FC2386E7003147A386E70030
:108B100017D7FF1F130787DA2398E70017D7FF1F20
:108B20001307C7DD239AE70017D7FF1F130747E98D
:108B3000239CE70029472381E70209472383E702B3
:108B40002385E702A3810700930600F8A380D700DE
:108B5000930690022380D700FD562383D7002381FC
:108B6000E7009306000537E700E0230BD740B70680
:108B700040002320D71003C7170013671700A380F6
:108B8000E700B24097D7FF1F239C07F8410182807E
:108B9000F1679387072017D7FF1F232DF7F6854727
:108BA00017D7FF1F231AF7F6A14717D7FF1F230672
:108BB000F7F697D7FF1FA38207F697D7FF1F238FDC
:108BC00007F497D7FF1F238D07CC97D7FF1FA388E4
:108BD00007CC814717D5FF1F1305C5CCFD5517D608
:108BE000FF1F1306E6CC2947B306F5002380B60025
:108BF000B306F600238006008507E397E7FE97D7C4
:108C0000FF1FA38407F097D7FF1FA38207F097D712
:108C1000FF1F238D07EE97D7FF1F238807EE97D7F7
:108C2000FF1F238707EE97D7FF1FA38107EE97D774
:108C3000FF1F238E07EC814717D6FF1F130606FF81
:108C40004147B306F600238006008507E39BE7FE55
:108C5000828017D7FF1F0347870085476316F700F9
:108C6000170300006700E3E8170300006700E3DC78
:108C7000411122C406C617D7FF1F034747FE854789
:108C80002E8613F4F50FAA856317F70417D5FF1F77
:108C9000130505D797600100E780602B97D7FF1F6A
:108CA000238007DAB787004023848702B7E600E015
:108CB0003706400023A0C6180100010003C7A70221
:108CC0001377C70F2385E702B240224423A0C610C2
:108CD00001454101828017D5FF1F130525C6976006
:108CE0000100E780C02697D7FF1F238907C8B787F1
:108CF000004023828702B7E600E03706400023A049
:108D0000C6180100010003C767021377C70F23834A
:108D1000E7025DBF411106C697000000E78080E7CB
:108D2000B2404101170300006700E3F2411106C69B
:108D300097F0FFFFE78080BF97D7FF1F83C717C457
:108D4000A1CB97D5FF1F83C585C389C917D5FF1F41
:108D5000130505C397E0FFFFE780C05F97D7FF1FAC
:108D6000A38E07C097D7FF1F238A07DA37E700E0F3
:108D7000B70640002320D7180100010037860040C5
:108D80008347660293F7370F2303F6022320D71099
:108D9000B2404101828041C9D9C597D7FF1F83C71F
:108DA00027D8D1C3011122CC4AC84EC656C25AC0D8
:108DB00006CE26CA52C42E89AA890144930A000409
:108DC000371B030063772403B3078940C207C183BD
:108DD000BE8463F4FA0093040004C204C180130A41
:108DE0001BD497D7FF1F83C767B99DE37D1A631C08
:108DF0000A00F2406244D2444249B249224A924AAD
:108E0000024B0561828097F0FFFFE78020B2D1BF5F
:108E1000338589002694A685420497000000E780E8
:108E200060E5418045B7828097D7FF1F938787F51C
:108E300018429C4383D645000345070083C5C700FD
:108E4000035646006396A50083D5E700638DD502DF
:108E5000011106CE2386A7002397D700B705CF00C0
:108E6000DC4B9385757D05077D162EC2230001001E
:108E70003AC42316C1002317D10099C30A858297EB
:108E8000F240056182808280411122C417A4FF1F35
:108E9000130404575C4C06C691CBC84B01C9B7E715
:108EA0000400BC5782975C4C23AA0700B2402244BE
:108EB00041018280DC4DDC4B81CFB7E70400904557
:108EC00003A38705914517D5FF1F0345E5EB0283F3
:108ED0008280B7E7040003A30705A14517D5FF1F4C
:108EE000034585EA02836D713C083EC6B707E5007D
:108EF000232291103EC8AA843C08328523261110F3
:108F00003ECA23248110232021112E89973000008E
:108F1000E780605A2A84979501009385658C1775C0
:108F200001001305256E97600100E780A00DA28562
:108F3000179501001305859797600100E780800C65
:108F4000294597600100E780C010B705CB009385E5
:108F5000757D680097100000E780E05FA2856800DB
:108F600097300000E7808047014781467000CA853E
:108F7000268597200000E780608305CD2A84979599
:108F800001009385E585177501001305A5679760B6
:108F90000100E7802007A285179501001305C59100
:108FA00097600100E7800006294597600100E7808F
:108FB000400A8320C1100324811083244110032917
:108FC00001105161828097D7FF1F9387A7DB18425A
:108FD0009C43797122D406D60348070083C8070151
:108FE0002A8483D64500035546006396080183D83A
:108FF0002701638DD8022388070105072399D7002D
:109000003708CC00DC4B1308787D3ACC1307F5FF0A
:1090100042CA23080100231EE100231FD10099C783
:10902000080832C62EC482973246A2452285970090
:109030000000E78080EBB250225445618280797154
:109040003146977501009385A54C280006D6976098
:109050000100E780C0EF97A7FF1F83D7673A231B64
:109060000100231C0100231D0100231E0100231FFA
:10907000010099E3C167FD17231AF10097A7FF1FAD
:1090800083D7273891EB97D7FF1F9387A7CF9C43B0
:109090009C43DC4783D7070097A6FF1F938646367D
:1090A000231BF100D84E83D74600231CF1005C4BF4
:1090B00091CB97A7FF1F83C7173581EB970000005F
:1090C000E780C0DCB25045618280FD1717A6FF1F04
:1090D000A30BF6320356070183C706014C4728004D
:1090E000230FF10097300000E780602C97D7FF1F17
:1090F000938747C99C430147978601009386C677AB
:10910000884330004C0897100000E780206A5DD942
:1091100075B799C9B7E7040003A30705A14517D59B
:10912000FF1F034565C6028382805C4EDC4BB9CFCE
:10913000B1CD411122C4177501001305A54C2E8431
:10914000978501009385056F06C697600100E7804B
:1091500060EBA2851785010013050570976001007B
:10916000E78040EA294597600100E78080EEB7E795
:1091700004002244B24003A3870517D5FF1F03450F
:10918000A5C013064006914541010283828041112A
:1091900022C417A4FF1F130464241C4C06C689C7ED
:1091A000DC4399C34C488297584CB7E70400BC573E
:1091B000484B82975C4CB240224423AA07004101ED
:1091C000828017A7FF1F13076723834707009306B3
:1091D000F00B850793F7F70F63E9F60097A6FF1FDB
:1091E000238EF620034507008280930700F8FDB721
:1091F0008357450099E37D558280011122CC17A445
:10920000FF1F1304E41F5C4C4AC84EC6DC4B52C41B
:1092100006CE26CA56C2B2892E8A2A898DC7B7E7DA
:109220000400FC5F829797D7FF1F9387A7B39C43E7
:109230001307301FB307F54071556375F7069700A4
:109240000000E780A0C49307D00D7D5563EC37057F
:10925000B7E4040093878900B858832AC4011395A2
:1092600007014181029723AAAA00484C584921E7E7
:10927000978501009385055A1775010013058538F8
:1092800097600100E78000D8178501001305856508
:1092900097600100E78000D7294597600100E780CB
:1092A00040DB5D55F2406244D2444249B249224A11
:1092B000924A0561828013874900B705CF002319C0
:1092C000E5009385757D310597100000E780A028A3
:1092D000484C83456900310597300000E780001055
:1092E000484C4E86D285310597300000E780200C2F
:1092F0007146CA8517A5FF1F1305851097600100E9
:10930000E780E0C4FC5C82970326C90097D7FF1F63
:1093100023AAA7A411CABC4C854517D5FF1F034536
:10932000A5A682970145BDBF97000000E78060D1E8
:10933000D5BF411106C622C426C217D4FF1F13048D
:10934000A4A497000000E78060B4B7E40400FC4CDC
:10935000034504008545829703450400224403A386
:10936000C405B2409244A14541010283411126C285
:1093700097D4FF1F938404A19C4006C622C44AC010
:10938000D5C3DC43C5C35CC12300B5002A849785DF
:10939000010093856543177501001305A5269760A5
:1093A0000100E78020C6294597600100E78060CA78
:1093B0009C4023A4070023A2070097A7FF1F9387C1
:1093C000E701DC4FDC4B91C7295597000000E7808F
:1093D00040DC97A7FF1F9387A702DC4FDC4B89C7B0
:1093E00097000000E78020F537E904008327C905CE
:1093F000894517D5FF1F0345259982978327C905FE
:10940000914517D5FF1F0345259882979C4003A3DC
:1094100047016309030022852244B2409244024975
:1094200041010283B24022449244024941018280B8
:109430000111328506CE22CC26CA2E849730000038
:10944000E7806007AA84978501009385253B1775FF
:1094500001001305251B97600100E780A0BA0307F0
:1094600084000356640083554400A68617850100D6
:109470001305054197600100E780C0B82945976052
:109480000100E78000BD97A7FF1F83C787F5639D95
:109490009700014597000000E780A0CF81450A852D
:1094A00097000000E780C0ECF2406244D2440561BE
:1094B00082806D71232481102326111023229110A4
:1094C00093F745002E84638707143C083EC0B70716
:1094D000E5003EC23C083EC42317010023180100EA
:1094E00023190100231A0100231B010097A7FF1F66
:1094F00083D7C7EE99E3C167FD172316F10097A73D
:10950000FF1F83D7C7ED91EB97D7FF1F93878787FF
:109510009C439C43DC4783D7070017A7FF1F130713
:10952000E7EB2317F100544F835747002318F1004E
:10953000DC4AA1E797850100938585301775010006
:109540001305450C97600100E780C0AB178501004B
:109550001305C53F97600100E780C0AA29459760C1
:109560000100E78000AF134544008320C1100324AD
:109570008110832441105161828097A7FF1F83C708
:1095800057E62555D9C3FD1717A6FF1FA30BF6E411
:1095900003D6060183470701CC460A85230BF10059
:1095A00097300000E780A0E097C7FF1F9387877D73
:1095B0009C4317A7FF1F130767E297860100938656
:1095C000262988430A866C0097100000E780001E59
:1095D000AA8451D9978501009385852617750100C6
:1095E0001305450297600100E780C0A1A685178595
:1095F00001001305653697600100E780A0A02945AA
:1096000097600100E780E0A4268597000000E780CE
:1096100040B891BF93F725009DC7B7E70400BC474A
:109620004146814528088297255597000000E7802C
:1096300040B628089305F00F97000000E78040D35C
:10964000134524001DB793F7150081CB9700000048
:10965000E780209F1345140009BF93F7850001455B
:1096600089D717A7FF1F034717DA97A7FF1F93870D
:1096700027D90DC3D84F584B11CF37E70400384FC7
:109680009047854517C5FF1F034505700297134591
:109690008400E1BD97F0FFFFE780407FCDBF5C4DC8
:1096A000411106C688C317C7FF1F232DF76CB7E704
:1096B000040083A70708170500001305C5DF82977C
:1096C000B24097C7FF1F2381A76C014541018280EB
:1096D00001113335A000A307A100B7E7040083A759
:1096E000471706CE1306F1008545130550308297C3
:1096F000F240056182808280411122C406C697B77C
:10970000FF1F83C7F7B3054489EF97C7FF1F83C7C0
:1097100067F3014499E717B4FF1F034464B213448D
:109720001400228597000000E780C0FA1785010029
:109730001305452909E4178501001305A5292244CD
:10974000B2404101176301006700C38B797122D4D5
:10975000A30F010037E404008327841726D24AD0E0
:1097600006D6AA842E89130550309305F10132C61E
:10977000829732468347F10193150601C18185CB5B
:1097800001452EC697000000E780C0F483274417E8
:10979000B2454A8626858297054597000000E780F6
:1097A00060F3B2502254925402594561828083275B
:1097B00044174A8626858297EDB741119397050194
:1097C00022C406C626C2C1872E8463D40702B7E42A
:1097D0000400FC5417A5FF1F034585C5829719C1D6
:1097E000BC5482972165218DB240224492444101AC
:1097F000828093F715008DC7B7E7040083A7471A47
:1098000017A6FF1F1306C6C197C5FF1F938585586E
:1098100017A5FF1F0345C5C1829713451400E9B77B
:1098200093F725000145E9D397C7FF1F83C7075862
:1098300085E7B7E7040003A8871A1307401F97A717
:10984000FF1F83C7E7BE814613064006994517C52B
:10985000FF1F0355255502981345240071B797C77C
:10986000FF1F83D727546398A70217C7FF1F231C26
:10987000B75217C7FF1F2319C75217C7FF1F231659
:10988000D7522E86178501001305451BBE85175339
:10989000010067002377178501001305A51B1763D7
:1098A00001006700038E0357450097C7FF1F83D74A
:1098B000674F6318F702C167F91717C7FF1F232304
:1098C000F74E97C7FF1F23A1074E97C7FF1F238996
:1098D000074C97C7FF1F238B074C17030000670037
:1098E000E3E1178501001305E51617630100670022
:1098F00043897D15954763E2A71C1787010013076D
:10990000E70A0A053A951C41011122CC06CEBA9706
:109910002E84828717850100130545149760010086
:10992000E7802086A1A203C7250099476311F702AB
:109930002E8597000000E78040F783456400178577
:1099400001001305A51297500100E780A06B97B79F
:10995000FF1F2387078E178501001305E5127DBFC2
:1099600003C7250095476319F702C16717C7FF1F93
:1099700003574743F91703D5A5006309F702B7E773
:10998000040083A7C7178297178501001305C51028
:1099900097500100E780E07E854717B7FF1F23013E
:1099A000F78A178501001305A5118DBF97C7FF1F03
:1099B000239AA73E83D7E50097C6FF1F2395F63E5F
:1099C00083D7050197C6FF1F2390F63E83D7250155
:1099D00097C6FF1F239BF63C97C7FF1F2382073CB8
:1099E000631BE502B7E70400BC4F09661306069047
:1099F000894517A5FF1F0345A5A382970356E400D9
:109A00008355A400178501001305450A97500100EE
:109A1000E780405F51B79307700F2316F100B7E757
:109A2000040083A7870D17A6FF1F034666A06C00DE
:109A300082974DF9854717C7FF1F2303F7365DB798
:109A40001785010013058508D1BD83C52500914701
:109A50006392F502178501001305C50897500100B0
:109A6000E780207297000000E78040C9F24062441E
:109A70000561828099476392F50222859700000074
:109A8000E780A0E28345640017850100130505FE09
:109A900097500100E7800057D1BF9547639AF500C2
:109AA00083471400E1F3178501001305E505BDB5F3
:109AB000178501001305C505E1BF82803757315F67
:109AC00097A7FF1F93870798130777D598C39356D7
:109AD000C50017870100130727F3BA9683C5060050
:109AE00093568500BD8ABA9603C606009356450074
:109AF000BD8A3D89BA962A9783C6060003470700A8
:109B0000238407002383D700A383E7002382B700C1
:109B1000A382C70097A7FF1F9387C7932383B7002C
:109B2000A383C7002384D700A384E7008280411168
:109B300006C697000000E780A0F8B7E7040083A7F7
:109B4000871417A6FF1F1306E68FD5450145829798
:109B5000B2404D4697A5FF1F9385C58F1305703002
:109B60004101170300006700A3BE61712324811A1D
:109B700037E40400832704082326111A2322911AAC
:109B80002320211B232E311917050000130525C39F
:109B9000829717A9FF1F1309A989994785442300B4
:109BA000A900231CF100978501009385E5E4930744
:109BB0004006177501001305E5A4231CF1082308CE
:109BC000910097C9FF1F938949B897500100E7801A
:109BD000604383D50900178501001305E5E0975020
:109BE0000100E7802042294597500100E780604648
:109BF00003D5090097000000E78080EC8327441715
:109C0000100885451305503082978327441717A6FF
:109C1000FF1F13062684CD451305703082978327D6
:109C2000441717A6FF1F1306E680B54513056030DD
:109C3000829783274417300889451305103182978E
:109C400083274417300989451305203182978327DC
:109C500044159305000A0D45829783274415930503
:109C6000000A11458297A30591002306910002CDB9
:109C700023080100230C0100832784163009914535
:109C8000130570408297832784161306B10085451B
:109C900013050040829783278416700085451305BD
:109CA000104082978327841630088545130520408D
:109CB00082978327841610088545130550408297A4
:109CC000832704157D558297832744137D558297FA
:109CD0007D5597A0FFFFE780409B8327440C829728
:109CE0009790FFFFE780A076832784141796FF1FC5
:109CF00013064675D5450145829789471306700FAF
:109D0000814528092306F1009780FFFFE780204066
:109D10008D471306000881452808230CF108978019
:109D2000FFFFE780C03E9147230CF10097670100D9
:109D30009387C77E984383C747003AC8230AF10038
:109D400097D0FFFFE780A09C70008545054597A050
:109D5000FFFFE780A09A30099305700F094597A08F
:109D6000FFFFE780A0993008930500080D4597A0F4
:109D7000FFFFE780A09810089545114597A0FFFFC9
:109D8000E780C097C16717C7FF1F1307A701F9171F
:109D90001CC3232207001795FF1F1305256997A0F1
:109DA000FFFFE78080948327C41D17C5FF1F13059D
:109DB000E5FD82973C48034509008545829783204D
:109DC000C11A0324811A8324411A0329011A832901
:109DD000C1195D618280C16717C8FF1F035888FCE5
:109DE000F9176301F8083DCDB5CD011126CAB7E4D6
:109DF000040083A7841222CC2E862315B10006CE40
:109E00002A8401478146ED45428582972AC611ED95
:109E100017850100130585C097500100E780603663
:109E2000F2406244D24405618280FC440356A100A2
:109E3000A28582972C0017C5FF1F0355A5F697A092
:109E4000FFFFE780409769DD17850100130545BED8
:109E500097500100E780E03283A7C412ED45280047
:109E600082977DBF82800DC585471797FF1FA30886
:109E7000F75C9797FF1F2385075C35469795FF1F73
:109E80009385455B13056030170300006700438C22
:109E90009797FF1FA385075AE9BF97C7FF1F83C77F
:109EA000E7F0A9EFC16717C7FF1F0357A7EFF9171F
:109EB0006306F7044111854722C417C7FF1F230714
:109EC000F7EE37E404007C4C06C689451795FF1F62
:109ED0000345055682970323841A2244B24097977C
:109EE000FF1F83C7E75417C5FF1F0355A5EB1307D3
:109EF000401F8146314699454101028382806D7140
:109F0000232481102326111023229110328401CDA5
:109F10008947630AF5028320C1100324811083243A
:109F200041105161828017850100130525BFAE8461
:109F300097500100E780E024A285268597B0FFFFB7
:109F4000E78080BBC9BFB7E70400FC4728008297C1
:109F500017850100130545BD97500100E780602279
:109F60008347810039C41307000B6380E70213871E
:109F7000A7051377F70F8D4663EDE602A28528004B
:109F800097C0FFFFE78000F879B78547E3F587F8CA
:109F900083459100177501001305059EB335B00088
:109FA00097A7FF1F2382B71097500100E780800515
:109FB0009DB703479100A207B966D98F1387E6556D
:109FC0006384E70C636DF7042D671307B755638F40
:109FD000E708636AF70029671307A755638FE70847
:109FE000A2852800A1BF31671307C7556388E7061C
:109FF00035671307D755E395E7FE8947E3FD87F0FB
:10A0000097000000E780A0E99305E4FFC205C18145
:10A010001305A1009790FFFFE780801CEDBD3D6711
:10A020001306F7556389C706636DF6009386E665E8
:10A03000E398D7FAA285280097C0FFFFE780003297
:10A04000D9BD9306F766638DD7041307F777E399B5
:10A05000E7F897C0FFFFE780205D75BD0146A28548
:10A06000280097C0FFFFE780801575B5A2852800FE
:10A0700097C0FFFFE780C02279BDA285280097C066
:10A08000FFFFE780A02341BDA285280097C0FFFF06
:10A09000E780C02349B597C0FFFFE7804035A5BDE5
:10A0A00097C0FFFFE780E03ABDB5C16717C5FF1F46
:10A0B000035545CFF9176307F500B7E7040003A37D
:10A0C000C7170283828017F3FFFF6700236317839C
:10A0D000FFFFE70223FF2A8408452E89B28919C9A8
:10A0E00000C1971500009385A58661059730010092
:10A0F000E780600481447D5A97100000E780E039D2
:10A1000063C7A404814497100000E780003A63C845
:10A11000A40497C7FF1F9387A7C99C43DC47B307D5
:10A12000F94091872302F400638309048327C9005F
:10A13000B307F4409587A302F4001C4C89C79C47E1
:10A1400099C3228582971783FFFF6700E3FA5C4477
:10A15000139714008504BA972390470171BF1C48D8
:10A16000139714008504BA972390070069BF8327CB
:10A1700089000547B307F4409587A302F40083578D
:10A180000400638EE7028DC309476384E7040D472B
:10A19000E395E7FA978701009387C7EB1CCC978775
:10A1A0000100938727EC11A897870100938707B2D6
:10A1B0001CCC97870100938767B25CC8BDBF9787A7
:10A1C00001009387A79D1CCC978701009387079E6A
:10A1D000EDB7978701009387A7EC1CCC9787010008
:10A1E000938707EDD9BF95E51783FFFFE70223EFBC
:10A1F000004618448347940075839D8B6317F700CE
:10A2000097100000E78060B448C41783FFFF670021
:10A2100043EF82801783FFFFE702C3EA138935000B
:10A22000C16442094111AA890144F1141359090179
:10A23000054A2EC697100000E7802026B2456348E5
:10A24000A400014541011783FFFF6700E3EA83A7EC
:10A25000090013171400BA9783D707006388B70063
:10A260006394970063742A010504E1B70545D9BFDB
:10A270001783FFFFE70223E4AA892E89328BB68475
:10A280003A8ABE8A97A00000E78000FE71C9268541
:10A2900097200000E780C00C8D4763E7A7007D553D
:10A2A0001783FFFF6700A3E483DB440097100000DF
:10A2B000E780A0242A8497100000E78040259307B8
:10A2C000740031443305850263CDA7029710000066
:10A2D000E780A02297100000E78020222A849710B0
:10A2E0000000E780C02293077400314433058502E3
:10A2F00063C3A70497100000E78020209307450060
:10A3000029A897100000E7808020330585021307F5
:10A31000F0179307C017E35FA7FA2D55E3C277F94B
:10A3200063040B02D6865286A6854A8597200100D3
:10A33000E78000BDB5B797100000E780401D3305EA
:10A3400085029307C5FFD1BF832749001385C90044
:10A3500083D5270097000000E78000EC61F581B706
:10A3600069553DBF97C7FF1F2396A7A497C7FF1F37
:10A37000938707A4904381470C463307F5004207B3
:10A3800041836393B7008280544613984700850742
:10A39000C2962390E600D5B797C7FF1F938747A1C2
:10A3A0009C4303C58700828017C5FF1F035585A006
:10A3B00082801783FFFFE70283D2C1671387D7FF2D
:10A3C000630BE502636AA700F1176300F50201451C
:10A3D0001783FFFF6700E3D21387E7FF6302E502FD
:10A3E000FD171D8D13351500E5B797500000E78068
:10A3F000A0297D15C5BF97500000E78020FED5BF7E
:10A4000097500000E78040FCEDB71783FFFFE7029D
:10A4100003CD4111AA8401442EC697100000E780A5
:10A42000C008B2456348A400014541011783FFFFFE
:10A43000670023CD9C48131514003E9583570500F3
:10A44000E385B7FE0504C9BF03485500814693F76D
:10A45000F60F63E5070181473E8582805845939753
:10A460005600BA9703D727006316B70003D7070033
:10A47000E304C7FE8506E1BF8346450001479377A5
:10A48000F70F63E4D700814711A81C451316570046
:10A490000507B29703D60700E313B6FE3E85828018
:10A4A0001783FFFFE70203C293170501C18797CA0D
:10A4B000FF1F938AEA8F635BF00883A70A00C047F7
:10A4C0009C4703570400198D420541816368F500DC
:10A4D000014422851783FFFF670003C212052A94F7
:10A4E000CDBFDC4713944900014A3E9483474400A2
:10A4F0006341FA02014A834754006349FA0285091D
:10A50000C20993D9090183A70A009847E3EBE9FC44
:10A51000C1B71C4413195A00A6853E994A85970075
:10A520000000E780C0EE05E1050AC9B75C441319D5
:10A530005A00A6853E994A8597000000E78020EDE5
:10A5400019E1050A4DBFE30C09FA61B7AA848149F4
:10A550005DBF1783FFFFE70283B81C452A8481E7AC
:10A560009307C5001CC51C44231204001CC093079C
:10A57000F00F63EDB70093F5F50F228597200000EB
:10A58000E780C0E51783FFFF6700A3B79394050139
:10A59000C167C18063F9F500A68522859720000078
:10A5A000E780E0E8C5B7C18193F5F50F22859720D4
:10A5B0000000E780A0E2A685228597200000E780C2
:10A5C000E0E3C9B797B7FF1F9387877E88438280F0
:10A5D0001C4599C797B7FF1F23ACA77C0145828014
:10A5E0007D55828097B7FF1F9387877C9843834769
:10A5F0004500484792073E9582801783FFFFE70298
:10A6000003AE617100451C183EC6B70780013EC805
:10A610001C183ECA8357440002CE02D002CC231E2F
:10A62000F100834784002A8902D22301F1023C0809
:10A630003ED402D697000000E78000FB8357050058
:10A640002316F10297500000E78040C72307A102BC
:10A650005C4003556400F18313F717008347F10250
:10A6600052055181F99BD98FA307F1029710010080
:10A67000E780607839CDAA840355050097A00000D3
:10A68000E78060BF83D704002AD26800231CF10052
:10A6900083D72400231DF1001C4803D647008C43B8
:10A6A00097200000E780A0D08347B400CA861776C1
:10A6B0000100130626488117A305F4006C0048101A
:10A6C00097200100E780C0835D611783FFFF67006B
:10A6D00043A32155D5BF1C45B1CF03C5A70089466B
:10A6E00013576500630BD7028D46630ED70285466C
:10A6F0006300D702130740063305E50203C7B7001E
:10A70000418B15CB83C7B700BD8B3355F540828095
:10A710001375F5031307803EC5B709671375F50375
:10A7200013070771D1BF372709001375F503130706
:10A73000077CD9B7014582801783FFFFE702239A80
:10A7400003A98500630C09048347B900AE8493F71D
:10A75000070E85C303459900930520030D81050568
:10A76000B305B5028844610597300100E780C0ACAD
:10A7700035A02E8597000000E78020F62A8419CDA9
:10A7800097000000E780605C8325C900B307B540EF
:10A7900063FA87002E94B305A440E9F51783FFFF01
:10A7A0006700239685457DBF1783FFFFE70223934C
:10A7B0002A8403D50500011132C636C43AC22EC020
:10A7C00002CA02CC02CE97A00000E780C0AA824550
:10A7D0002ACA22852ECC97000000E780E0E00357CC
:10A7E0000500231EE10097500000E78020ADA2463F
:10A7F00032469247230FA10036874C08B286228545
:10A80000014697000000E780E0A605611783FFFF7F
:10A810006700238F1783FFFFE702638C61711C18A9
:10A820003EC6B70780013EC81C183ECA3C0800451A
:10A830003ED4AA8402CC02CE02D002D202D6970025
:10A840000000E78060DA8357050035592316F102CE
:10A8500097500000E78080A62307A10209C4835710
:10A86000440081EB21594A855D611783FFFF670032
:10A870004389035564005205518197100100E78018
:10A8800080572A8965D18347B40093F7070E99C78B
:10A890001305840197300100E780409C83574400F2
:10A8A000231EF100834784002301F1025C4003551D
:10A8B0000900D98313F7070883471102231CA1005D
:10A8C00093F7F707D98FA300F10283572900231DBF
:10A8D000F1005C40F18313F717008347F102F99B05
:10A8E000D98FA307F10297A00000E780C0982AD271
:10A8F00035D9834794006800139757008347B40005
:10A90000FD8BD98FA305F4001C4803D647008C4368
:10A9100097200000E780A0A9A687177701001307FA
:10A920006721740005464C10268597000000E780DB
:10A9300060942A890DD98347B400A685FD8BA305B1
:10A94000F40097000000E78060DF31BF1773FFFF5E
:10A95000E702E378832485FE2A8441112685970047
:10A960000000E78080D7834734FF93F7070E8DCB35
:10A970002AC6268597000000E78060C809CD834776
:10A9800034FFB245FD8BA309F4FE91C522859730B3
:10A990000100E780608A41011773FFFF670063765B
:10A9A0007DD98327C4FF2685829775F5834734FFB9
:10A9B00093F7070E91C7228597300100E780008A40
:10A9C000032584FE97000000E78000E5E9B71773D0
:10A9D000FFFFE702C36D9C4141112A8903C70700AD
:10A9E00089472E84935667006380F6040D4663887A
:10A9F000C6049307F0076304F7022E859720000032
:10AA0000E78060ABAA848149C16B130C490097B7FA
:10AA1000FF1F9387E7399C43984763E4E9044101AA
:10AA20001773FFFF6700636C03D745008547E3F8A2
:10AA3000E7FE2E8597200000E78040ADE1B703D701
:10AA40004500E3FEE7FC2E8597200000E780A0A6E6
:10AA5000AA84228597200000E78000A8C204C98C40
:10AA60005DB7DC470355A900139A49003E9A931736
:10AA70000501C187635DF00083570A006397A70251
:10AA800063E774038327CA00034D5A002DA0A16712
:10AA90002167A98F1307F7EFE374F7FE63970900A7
:10AAA00097000000E780209161FD85098DB783271D
:10AAB0008A00034D4A00835DA90003576900216A9B
:10AAC000138BC7003AC6814A33CA4D01631E5D012C
:10AAD00097B7FF1F9387472E9C43E1DBA2866286D0
:10AAE000814526858297D1B7A1679387F7EF930CAD
:10AAF0004BFF63F24703B2455A8597F0FFFFE780AB
:10AB0000A0710DC103278B00104709CE104363824B
:10AB1000C4023107D5BFEE85668597000000E78047
:10AB2000008F71F993861A0093FAF60F130B0B023C
:10AB300071BF835644005C43E3E9F6F622853AC6CA
:10AB400097200000E7802081A1679387D7042A8A95
:10AB5000035D4400324763E897008347D90093E7D9
:10AB600007F8A306F9001C4766852286E2858297CE
:10AB7000C1670844FD17337AFA00529508C02312C2
:10AB8000A40125B797B7FF1F938787229843814772
:10AB900015C31447814763FFD500939745004C4781
:10ABA000BE9519C903C7550081476375E600DC45AA
:10ABB0001606B2973E85828003C745008147E37B36
:10ABC000E6FE16069C45F5B71773FFFFE702834FB5
:10ABD000AA892E8A814497BAFF1F938A6A1D83A788
:10ABE0000A00984763E6E4001773FFFF6700C3504D
:10ABF000DC471394440001493E9413BB140083477F
:10AC00004400634BF900014913BB1400834754000F
:10AC1000634FF9008504E1B7084493175900528740
:10AC2000DA860146A2853E9582990509C9BF484446
:10AC3000931759005287DA860546A2853E95829978
:10AC40000509E9B71773FFFFE7026349814517F567
:10AC5000FFFF1305054897B7FF1F239D07149700B3
:10AC60000000E780A0F61773FFFF6700834997B7DE
:10AC7000FF1F9387E7139C4395C31773FFFFE702FA
:10AC80000346814517F5FFFF1305A5449700000013
:10AC9000E780C0F31773FFFF6700A3468280177336
:10ACA000FFFFE702234237E40400832784124111A7
:10ACB0002315E100AE893289368A3A8681460147FA
:10ACC000ED45AA8482972AC621C90356A100D285E0
:10ACD00097400100E780A0278327C413CE852685EF
:10ACE0008297058905C98327440D23142101014654
:10ACF0002C00268582972A8401C9B7E7040083A720
:10AD0000C712ED4528008297228541011773FFFF86
:10AD10006700833E4944D5B76554FDB75C41FD17D4
:10AD20005CC182801773FFFFE702633BB7E7040053
:10AD3000FC5F829795473305F50281450D811773B6
:10AD4000FFFF6700033C1773FFFFE7024339B7E7D4
:10AD50000400FC5F829795473305F5020D81177358
:10AD6000FFFF6700033A1773FFFFE7024337B7E7B8
:10AD7000040083A7870B0355050082971773FFFF15
:10AD8000670023381773FFFFE7026335035505009B
:10AD90003287AE861786FF1F0356E67197B5FF1FF1
:10ADA0009385C50197000000E780A0EF1773FFFFB0
:10ADB000670023351773FFFFE7026332B7E704002C
:10ADC00083A7C71782971773FFFF67008333177333
:10ADD000FFFFE702C330B7E7040083A7871397B5E7
:10ADE000FF1F9385A5FD829701451773FFFF67003D
:10ADF00043311773FFFFE702832EB7E7040083A7F1
:10AE0000C71F81451785FF1F0355E5668297177396
:10AE1000FFFF6700032F1773FFFFE702432CB7E71D
:10AE2000040083A7871397B5FF1F938525FA8297A0
:10AE300001451773FFFF6700C32C1773FFFFE7027D
:10AE4000032AB7E7040083A7C71F81451785FF1FA3
:10AE50000355656882971773FFFF6700832A17738E
:10AE6000FFFFE702C3272E8597800000E780C0B26E
:10AE700097800000E780C0EF1773FFFF670063282B
:10AE80001773FFFFE702A32597800000E780C0F952
:10AE90001773FFFF6700E3265C49E1175CC95CC5D7
:10AEA00083572501A1072319F50083570501A10741
:10AEB0002318F5008280F1473305F50297B7FF1F8D
:10AEC0009387C7F29C433E9582808D476315F608B1
:10AED00003D74600854763F0E7081773FFFFE702D3
:10AEE0000320368536842E8997100000E780A05C09
:10AEF00029C98357440093140501C18063E3970473
:10AF0000228597100000E780005BFD142312940057
:10AF10009307A0026300F5029307B0026307F502EE
:10AF200093079002631FF500228597000100E780D8
:10AF3000A08801A80146CA85228597A00000E78065
:10AF400040B31773FFFF6700C31B228597100000F3
:10AF5000E7806007FDB7828097B6FF1F938646E9BA
:10AF60009C42014599CF9843D44217B6FF1F232135
:10AF7000E6E86396D70097B6FF1F23ADE6E6138594
:10AF8000C7FE82801773FFFFE7026315970000007A
:10AF9000E780A04B714433058502914597900000EE
:10AFA000E78000EC11E565551773FFFF6700631537
:10AFB00097B7FF1F23AAA7E297000000E780E048A9
:10AFC00033058502914597900000E78060E961DDD7
:10AFD00097B7FF1F23ACA7E097000000E780E0468B
:10AFE00097B7FF1F239CA7DE97000000E780E0458E
:10AFF00097B7FF1F2395A7DE977701009387C7B800
:10B0000017B7FF1F2320F7DE97070000938707E994
:10B0100017B7FF1F2326F7DC014579B71773FFFF2A
:10B02000E702E30BAA8517B5FF1F130525DB971071
:10B030000000E780605F1773FFFF6700830C1773E2
:10B04000FFFFE702C30997000000E78060FD97104B
:10B050000000E780E05E97B7FF1F938767D99C43A6
:10B0600091CF1387C7FE19CB83D5C7FF17B5FF1F35
:10B07000130585D897200100E780001C1773FFFF98
:10B08000670023081773FFFFE702630597000000BE
:10B09000E780C0EC09CD834785002A8493F7070435
:10B0A00099EB0355E50097000000E78080F91773DE
:10B0B000FFFF670003058347C5009304450117B9E7
:10B0C000FF1F1309E9D285E3832709005CC997B7FD
:10B0D000FF1F23AF97D083274900F1FB97B7FF1FCE
:10B0E00023AA97D0E9B7FD172306F50061059780DD
:10B0F0000000E780A0D98307840063CB070483475F
:10B10000840093E707F82304F400B7E704009C5F8A
:10B1100082974205A94741813375F5028347840030
:10B1200093F707FCC98F2304F4008347D4003E95AE
:10B130001C402318A40089CF984319CB8347C4002F
:10B140005040814585073305F5024205418102974C
:10B15000832709005CC897B7FF1F23AB97C88327D5
:10B16000490089E797B7FF1F23A697C88347C40004
:10B170009DDF8355040117B5FF1F1305E5C7972011
:10B180000100E780600B25B71773FFFFE70223F587
:10B1900097B7FF1F938787EB9C4701448583858B77
:10B1A00085E3AE84B2853A8697100000E780204F91
:10B1B0002A8419C597100000E7806045829408CC66
:10B1C00022851773FFFF6700C3F31773FFFFE702C2
:10B1D00063EF41112E8932C6AA8997000000E780EB
:10B1E000C031324713060502CA86970500009385D1
:10B1F000C5CC17B5FF1F130565BE97000000E7809B
:10B20000E0F82A8425C99304C50097000000E78070
:10B21000E0411946AA85268597100000E78020198D
:10B220008545268597100000E780001517750100F9
:10B23000130545934E95834505002685971000001C
:10B24000E780C0195C4831468145A1075CC85CC4F1
:10B2500083572401E1172319F40083570401E117F0
:10B260002318F4001C4C3E859770FFFFE78020EA0E
:10B27000A3042501228541011773FFFF6700C3E77F
:10B280001773FFFFE702A3E54111AA842EC632C45B
:10B2900097100000E780003A004DB24522468347F0
:10B2A00084000CC050C093F7F70393E7070423040E
:10B2B000F40023180400268597100000E78020354D
:10B2C00083479400A9462317A40013D73700050726
:10B2D0003307D7029D8B85072306F400A306E400FD
:10B2E00083C70401D8488507230FF7FE17B7FF1F50
:10B2F000130707B05843232A04009307440129E3A6
:10B3000017B7FF1F2328F7AE17B7FF1F2322F7AE8B
:10B3100017B4FF1F130444AE228597200100E78075
:10B32000E0E31C44858B5D8D19E5814522859720DE
:10B330000100E78060F041011773FFFF670063DCE5
:10B340001CC317B7FF1F2327F7AAD9B71773FFFF2F
:10B35000E702E3D897050000938565B7014597009C
:10B360000000E78000B001451773FFFF670063D955
:10B370001773FFFFE702A3D697000000E78080B0B5
:10B380001773FFFF6700E3D78347C500A5E3177373
:10B39000FFFFE702C3D42A840355E50097000000AD
:10B3A000E78000C821C18347840093F7F7FB23049B
:10B3B000F4001C4091C7DC4381C74C400145829793
:10B3C00097000000E78080B917B5FF1F1305C5A2DD
:10B3D00097200100E78080E80355E4009700000013
:10B3E000E78020C61773FFFF6700A3D18280177321
:10B3F000FFFFE702C3CE97B7FF1F9387679F9705AD
:10B400000000938565C817B5FF1F1305E59E23A0AF
:10B41000070023A2070097200100E780C0D117731F
:10B42000FFFF670003CE1C4D91CFDC4381CF177324
:10B43000FFFFE702C3CA8345070082971773FFFF28
:10B44000670023CC828097B7FF1F9387279D9C437B
:10B4500003C50700828097B7FF1F9387279C9C43F3
:10B4600003C51700828097B7FF1F9387279B9C43D4
:10B4700003C52700828097B7FF1F9387279A9C43B5
:10B4800003C54700828097B7FF1F938727999C4386
:10B4900003C53700828097B7FF1F938727989C4387
:10B4A00003C55700828097B7FF1F938727979C4358
:10B4B00003C56700828097B7FF1F938727969C4339
:10B4C00003C57700828097B7FF1F938727959C431A
:10B4D00003C58700828097B7FF1F938727949C43FB
:10B4E00003C59700828097B7FF1F938727939C43DC
:10B4F00003C5A700828097B7FF1F938727929C43BD
:10B5000003C5B70011E11D45828097B7FF1F9387E0
:10B51000E7909C4303C5C700828097B7FF1F9387BE
:10B52000E78F9C4303C5D700828097B7FF1F93879F
:10B53000E78E9C4303C5E700828097B7FF1F938780
:10B54000E78D9C4303D50701828097B7FF1F938740
:10B55000E78C9C4303C52701828097B7FF1F938721
:10B56000E78B9C4303D54701828097B7FF1F9387E2
:10B57000E78A9C4303D56701828097B7FF1F9387B3
:10B58000E7899C4303D58701828097B7FF1F938784
:10B59000E7889C4303C5A701828097B7FF1F938765
:10B5A000E7879C4303C5B701828097B7FF1F938746
:10B5B000E7869C4303C5C701828097B7FF1F938727
:10B5C000E7859C4303C5D701828097B7FF1F938708
:10B5D000E7849C438857828097B7FF1F938707842F
:10B5E0009C4303D5C702828097B7FF1F93870783C9
:10B5F0009C4303D5E70219E11305800C828097B7BD
:10B60000FF1F9387A7819C4303C50703828097B7D9
:10B61000FF1F9387A7809C43C85B828097A7FF1F6B
:10B620009387477F8843828097A7FF1F9387C77EB2
:10B630008843828019E17D558280F5DE984265DF7E
:10B64000FDD917B7FF1F130767A01847AA877155C1
:10B65000058B631D072403C507001547E37DA7FC81
:10B6600003C737001305F0057D171377F70FE36461
:10B67000E5FC03C35700E30003FC83C86700E38CC9
:10B6800008FA03C77700494579171377F70FE36482
:10B69000E5FA03C7A70011481305F7FF1375F50F67
:10B6A000E36BA8F803CE97000D481305FEFF137552
:10B6B000F50FE362A8F803C8B7006309080065182E
:10B6C0001378F80F1305600DE36705F703C5C7008E
:10B6D000794879151375F50FE36FA8F403C8D700FF
:10B6E0000D457D181378F80FE36705F503D80701BA
:10B6F000930E40175118420813580801E3ED0EF35A
:10B7000003C8E7007D181378F80FE36605F303C854
:10B7100027017D181378F80FE36F05F103C8870040
:10B72000C54E75181378F80FE3E70EF103D86701DB
:10B73000856E938EBEE06D18420813580801E3EC45
:10B740000EEF03D847016D18420813580801E3E4CF
:10B750000EEF03D887017918420813580801E36CEB
:10B7600005ED03C8A7017D181378F80FE36505ED13
:10B7700003C5B7011D487D151375F50FE36DA8EAE4
:10B7800003C5D701714879151375F50FE365A8EA6C
:10B7900003D5E7011308E00F7D1542054181E36CF5
:10B7A000A8E803C50702494879151375F50FE36446
:10B7B000A8E8C85301C937C834005915130858BF41
:10B7C000E36BA8E603A8870237C53400130555BF0D
:10B7D0005918E36205E717A5FF1F232FC56203C6AB
:10B7E000050117A5FF1F232BF5620545E375C5E489
:10B7F00003D82501D04933760603E31E06E203C6CB
:10B800001501E30A06E217A6FF1F2325B66083C5CC
:10B81000270001466387A50003C61700F1453306DC
:10B82000B60283C707039305C00272971A0713076E
:10B83000C70516031A9796084697B387B70241556E
:10B840003E973297420741836362E8061773FFFF12
:10B85000E702E388368597800000E780806B9700D9
:10B860000100E780004B2A8497A00000E780605D1C
:10B870002A9497F00000E78040292A9497900000CE
:10B88000E78080842A9497F0FFFFE780E06F2A9496
:10B8900097400000E78000972A9497700000E780A7
:10B8A000809F22951773FFFF6700A385828017731F
:10B8B000FFFFE702C3824111A307A10097A0000088
:10B8C000E78080C89305F100170500001305E5B572
:10B8D00097F0FFFFE780802F014541011773FFFFBD
:10B8E000670023821763FFFFE702E37C17A4FF1FB3
:10B8F0001304C4750328840079599368180097A429
:10B90000FF1F23A914751378180063100802BA8466
:10B91000BE89368B328A2E89AA8A97F0FFFFE7808C
:10B92000E0A77D15269519E531594A851763FFFF74
:10B930006700E37B97F0FFFFE78040A67D15269523
:10B94000A167E353F5FE97B7FF1F938727A7984397
:10B950003E8C814B01CB014597F00000E78000470A
:10B96000933B15004A85DA865686D285979000006B
:10B97000E780A0502A8911CD1C44F99B17A7FF1F0F
:10B98000232AF76C83270C00CDD3E3800BFA829730
:10B9900069BF268597A7FF1F23AC076A97F0FFFFB3
:10B9A000E780809C4146CE8517A5FF1F1305857350
:10B9B00097300100E780A05997D00000E780209CD5
:10B9C0000325040B97D00000E780E09F054597D042
:10B9D0000000E780E0A6054597000000E78060EDE5
:10B9E000A9B797A7FF1F938767669C47858BEDC70D
:10B9F0001763FFFFE702A36E17A5FF1F1305C56CB2
:10BA000097A7FF1F23A4076497A7FF1F23A207641C
:10BA100097A7FF1F23A0076497200100E7800084F9
:10BA200097500000E780C0F897100100E780804F32
:10BA300097100100E780805597A7FF1F9387875FC6
:10BA40009C4391C7054597800000E780202397A776
:10BA5000FF1F9387E7479C4399C741657D15977002
:10BA60000000E78020A597F00000E780C04097D055
:10BA70000000E780609297A7FF1F938727729C437F
:10BA8000139717016356070097F00000E780E0AFB7
:10BA900097A7FF1F23A8076497A7FF1F23A6076484
:10BAA00097A7FF1F23A4076497A7FF1F23A207647C
:10BAB00097000000E780008C97000000E780A075E9
:10BAC00097F0FFFFE780401897F00000E78020D94B
:10BAD0001763FFFF6700E362828097A7FF1F9387CA
:10BAE000E7568843828097A7FF1F93872756C8434E
:10BAF0008280B7E7B0009387075063E1A70297A75A
:10BB0000FF1F9387A754D843FD576367E50097A7A6
:10BB1000FF1F23AFA75281473E858280B957EDBFF3
:10BB20001763FFFFE702A35B97800000E780A07424
:10BB300097800000E78000771763FFFF6700635C72
:10BB40001763FFFFE70203582A84930414020111CC
:10BB50002E85B289A685214636C63A8997300100DE
:10BB6000E780803C0DE9B24638082686CE8513056D
:10BB7000940497500000E780A04021462C084A8595
:10BB800097300100E780403A1335150005611763CF
:10BB9000FFFF670063560145D5BF1763FFFFE7024C
:10BBA00003549305450617A5FF1F13056527971036
:10BBB0000100E78060681763FFFF67008354176325
:10BBC000FFFFE702C35141112EC697F0FFFFE78048
:10BBD000C017B24588C141011763FFFF6700635278
:10BBE0001763FFFFE702034EAA842E8497800000AC
:10BBF000E780406BAA898545228597000000E78091
:10BC0000E07D83C7E4011389940899E31389040351
:10BC1000CE85228597000000E780407C2146930571
:10BC20001902228597000000E780607897A7FF1F20
:10BC30009387C7418C43228597100000E780C0821C
:10BC4000214693858402228597000000E7802076B4
:10BC50001763FFFF6700434A1763FFFFE702A3452F
:10BC6000397197F00000E78020B49305400661E940
:10BC700097800000E780405F6302051497A7FF1FCD
:10BC800083C7C71B13B7170097A6FF1F2388E61AA1
:10BC9000014499CFC16417A9FF1F1309293B9309D8
:10BCA000400EFD1497000000E78020836342A40A41
:10BCB00097F0FFFFE78060094169B7290900096A29
:10BCC000FD7A2A8B81447D199389F97B130A0A71C5
:10BCD000938A8AC797000000E780208063D7A40476
:10BCE0001304400EB387840217A7FF1F13070736FC
:10BCF0000324070B3E948357C4016382270B18402B
:10BD00003307EB4063EAE900834744008507B387C4
:10BD10004703D6976365F70801468145094597F0C3
:10BD2000FFFFE780C04AAA8B29E597400000E78023
:10BD3000C08285476317F50689659385057117A548
:10BD4000FF1F1305E50D97100100E780E04E95A059
:10BD5000B30734030327090BBA9703D7C701630856
:10BD6000970003C75700A38207002382E70005045A
:10BD700015BF9305C500228597000000E78080E687
:10BD80005E85228697650100938505DF97F0FFFFAA
:10BD9000E780404F5E8597100000E780608A850449
:10BDA00015BF97A7FF1F9387672A9C478D83858BB5
:10BDB000C1F721611763FFFF6700633301468545C3
:10BDC000094502D002D202D402D697F0FFFFE780E5
:10BDD0000040AA8479DD97F00000E780209C138959
:10BDE000C4002A8481454A8597000000E780005FEF
:10BDF0000C4041464A8597000000E780405B83295C
:10BE000044006385090C4E8502D802DA02DC02DEAA
:10BE100097300100E78020382ACE141005462C0800
:10BE200008184ECC97500000E780200A1375F50FD4
:10BE300051ED8355840093E525004A859700000065
:10BE4000E780E05E11460C104A8597000000E7800D
:10BE50000056014697650100938585D2268597F0A7
:10BE6000FFFFE7802042268597000000E780407DA5
:10BE70005C40A1D3014685450D4597F0FFFFE78063
:10BE80000035AA841DD548401389C40097300100AD
:10BE9000E78060302AC64A8597000000E780404C62
:10BEA0003246636FC5004C404A8597000000E7802A
:10BEB000005001468145268597F0FFFFE780803CD2
:10BEC000268597000000E780A077E5B583558400BC
:10BED000ADB71763FFFFE702832097A7FF1F938784
:10BEE000E7169C471DC193E7870017A5FF1F1305A1
:10BEF00025F317A7FF1F232FF71497100100E780E2
:10BF000080311763FFFF6700C31FDD9B17A7FF1F6B
:10BF10002322F71497300000E78020647DF117A5F5
:10BF2000FF1F1305E5EF97100100E7802033D1BF15
:10BF30001763FFFFE70223184169AA892E8AB28A94
:10BF4000368BBA8B814417ACFF1F130C2C10930C4B
:10BF5000400E7D1997F0FFFFE780205863C4A400CE
:10BF600001443DA03384940383270C0B3E948357F4
:10BF7000C401638627055A87D6865286CE85130567
:10BF8000040397000000E780E0BB01C923800B0099
:10BF900022851763FFFF670083158347F40185C37C
:10BFA0005A87D6865286CE851305940897000000DE
:10BFB000E78040B909C585472380FB00D1BF8504D0
:10BFC00051BF835745006380071E1763FFFFE702D9
:10BFD000630F01112A8497000000E780C04D09C952
:10BFE00085476309F50605611763FFFF6700C31006
:10BFF00097E00000E780407B7DF583574400494788
:10C00000ED9BE392E7FEC145228597000000E780A3
:10C010004033AA84228597000000E780204F035711
:10C02000440002CE91472A89631AF70022859700BF
:10C030000000E780A0513C082ACC3ECE97E00000EB
:10C04000E780C0755C55C5D374084A86A68505454A
:10C05000829751BF03574400D147E3F6E7F8032A1C
:10C060000400C169014997AAFF1F938A2AFE130B96
:10C07000400EFD1997F0FFFFE7802046634FA90EA1
:10C080002285032A040097000000E780C042A145F2
:10C090002A89228597000000E780A02AAA842285A9
:10C0A00097000000E780804A14402A86AA89780811
:10C0B0002685CA8597000000E780C0E7AA8405D5D9
:10C0C00003C7F40189476315F7008347C10181DF86
:10C0D0005546D2851385640097300100E78020E73C
:10C0E000014597800000E780001901C583D7C4018E
:10C0F000A5E797A7FF1F938767F59C4793551900FE
:10C10000858913D73700058B01CF8983858B639988
:10C11000B70001452EC697000000E780C0DBB2459E
:10C120004E8597800000E780A01E0346C1012A8447
:10C1300093751900268597900000E780203935C156
:10C14000268597800000E7802018268511C00145CC
:10C1500097800000E780404B97300000E780E03F89
:10C160008547E312F5E883C754001307F00FE38C0B
:10C17000E7E68507A382F400BDB5B304690383A78E
:10C180000A0BBE9483D7C401638B37015546D28511
:10C190001385640097300100E78000D955DD05095B
:10C1A000D1BD5DD86DB782801763FFFFE70283F1D1
:10C1B00097800000E780400B05C1C164014417A9C6
:10C1C000FF1F1309A9E89309400EFD1497F0FFFF24
:10C1D000E780A030634EA40017A5FF1F130545C4D8
:10C1E00097100100E78020031763FFFF6700C3F08B
:10C1F000330534038327090B3E958357C5016388B4
:10C2000097002312050097800000E780E00B0504EB
:10C2100075BF97A7FF1F938767E39C478D83858B27
:10C220008DE31763FFFFE70283EB17A5FF1F1305DD
:10C2300025BF97100100E78060021763FFFF6700CA
:10C2400043EC82801763FFFFE70263E99705000074
:10C250009385C5A017A5FF1F130585BC9710010086
:10C26000E78060ED1763FFFF6700A3E91763FFFF37
:10C27000E702E3E68841B7E70400BC5B0505420539
:10C280004181829709C585472300F500050517639D
:10C29000FFFF670003E783C7F5FF2E858507A38FA0
:10C2A000F5FE828083C7F5FFFD1793F7F70FA38F85
:10C2B000F5FE99EF1763FFFFE70263E2B7E70400BB
:10C2C000BC571385F5FF82971763FFFF670063E391
:10C2D00082801C41035745008D8FBA951CC12312E3
:10C2E000B5003E85828093D78500A2051441DD8D7F
:10C2F000835745001387E6FF18C189072312F5000D
:10C3000013D685004111238FB6FEA38FC6FE4101CF
:10C31000828018419307F7FF1CC1835745008507AA
:10C320002312F500A30FB7FE8280835745008D8F3F
:10C330002312F5001C41BE950CC12E858280AA8770
:10C3400003D7470008410D8FAA952392E7008CC3BD
:10C350008280184108453305A740828083574500F5
:10C36000035765001D8F1C4108453385A7403305E1
:10C37000A74082801763FFFFE70263D641112EC6F4
:10C380002A8497000000E780A0FDB2456373B500E2
:10C3900001A0835744000840BE952312B4003E9587
:10C3A00041011763FFFF6700C3D51763FFFFE70273
:10C3B00003D341112E84B28532C697000000E78076
:10C3C000A0FB3246A28597300100E78040B84101CA
:10C3D0001763FFFF6700E3D21763FFFFE70223D075
:10C3E0002E84854597000000E78000F92300850032
:10C3F0001763FFFF6700E3D01763FFFFE70223CE59
:10C4000041112317B100894597000000E780C0F66D
:10C410008347E1002300F5008347F100A300F50006
:10C4200041011763FFFF6700C3CD1763FFFFE702FA
:10C4300003CB93D78500A2054111DD8D2317B100F1
:10C44000894597000000E78020F38347E10023003F
:10C45000F5008347F100A300F50041011763FFFFDA
:10C46000670023CA1763FFFFE70263C713978501BD
:10C4700093D78501C166938606F0D98F13D78500BF
:10C48000758FD98FA2053707FF00F98D4111DD8D1A
:10C490002EC6914597000000E78000EE6C00114623
:10C4A00097300100E780A0AA41011763FFFF6700F2
:10C4B00043C51763FFFFE70283C21C41854503C4E0
:10C4C000070097000000E78080E622851763FFFFE2
:10C4D000670023C31763FFFFE70263C01C414111DC
:10C4E000894503C7070083C717002307E100A30797
:10C4F000F10097000000E78080E30355E10041016F
:10C500001763FFFF6700E3BF1763FFFFE70223BD69
:10C510001C414111894503C7070083C71700230742
:10C52000E100A307F10097000000E78040E0835797
:10C53000E100410113D58700A2075D8D42054181CD
:10C540001763FFFF6700E3BB1763FFFFE70223B931
:10C550000C4141112A841146680097300100E780A0
:10C56000009F9145228597000000E78040DCB2479C
:10C57000C166938606F01397870113D58701598DFD
:10C5800013D78700758F598DA2073707FF00F98FE2
:10C590005D8D41011763FFFF6700A3B61C45BE9583
:10C5A0000CC18280AE87944391E6584101EF0CC1E3
:10C5B0005CC1828003C7570013671700A382E7009E
:10C5C000B687D5B70CC3EDB7AA87084119CD184176
:10C5D000D44398C36313D500D8C32A8703465700B2
:10C5E0009376160081E6232007008280944381CA57
:10C5F0008C4203A847008CC363930601CCC3799A8D
:10C6000014C3A302C7003687D1BF1C45DC471D8D6C
:10C61000B777DBB6938777DB09853305F5024205EB
:10C6200041818280F147B385F50248452E9582808D
:10C630008347450085072302F50082801763FFFFCB
:10C64000E702E3A92A8409E41763FFFF670063ABED
:10C6500083474400F5DBFD1793F7F70F2302F4003F
:10C66000E5F71C4403D7270005072391E700DC43C7
:10C6700099C3228582974C4889CD83475400898B82
:10C6800099E71C4422859C479C439C478297232A18
:10C6900004000040232004007DB71763FFFFE7027A
:10C6A00003A48357250041112EC681EB0144228546
:10C6B00041011763FFFF6700C3A4035705008147CB
:10C6C000F146E305F7FEB385D702404585072E9472
:10C6D0008345440008C4F5F5B247AA8481E7232ABC
:10C6E000040009A81C456C0022859C439C4382974A
:10C6F00048C84DDD85472312F400B24723200400CB
:10C70000231804002319F4005C485CC483D7240078
:10C71000FD172391F40061BF1763FFFFE702239C1D
:10C720009797FF1F9387C77188432326050023240B
:10C730000500410597100100E78040B21763FFFF35
:10C740006700239C1763FFFFE70263991794FF1F9D
:10C750001304046F1C40411199CF9C472300B5007E
:10C760002AC65CC197000000E78040FB1C40DC4308
:10C7700099C33245829741011763FFFF67006398B1
:10C780000347450029E3584DAA877D551DCF176300
:10C79000FFFFE702C3941CC3DC479796FF1F23A14A
:10C7A000E66AF156130507012390D70097050000AC
:10C7B0009385050297100100E780E0970145176314
:10C7C000FFFF670003947D55828082801763FFFF1F
:10C7D000E702E39001116146814528009760FFFF61
:10C7E000E780E0929797FF1F938787659C43280017
:10C7F0009305F00FDC473EC697000000E780C0F4C9
:10C8000005611763FFFF6700C38F9797FF1F93872B
:10C8100027639C43D847A1679387C702631EF70A23
:10C82000397106DE22DC26DA80004AD84ED652D490
:10C8300056D23285B28497000000E780C0C7AA892B
:10C84000268597000000E78020C92318A4FC2685D0
:10C8500097000000E78040C82319A4FC26859700B4
:10C860000000E78060C783D744000A8A231AA4FC2B
:10C87000858393F7F70F230EF4FC8607BD0793F724
:10C88000073F3301F1408A8A01498347C4FD63674A
:10C89000F902CE85130584FC232C54FD970000007B
:10C8A000E78080EA5281130104FCF2506254D254B2
:10C8B0004259B259225A925A2161828026859700A4
:10C8C0000000E78060C193171900D69705092390EF
:10C8D000A7001379F90F55BF82809797FF1F9387A1
:10C8E00027569C43D847A1679387A702631AF70A84
:10C8F000397106DE22DC26DA80004AD84ED652D4C0
:10C9000056D23285B28497000000E780C0BAAA8967
:10C91000268597000000E78020BCFD572318A4FC63
:10C9200026852319F4FC97000000E780E0BA83D73E
:10C9300044000A8A231AA4FC858393F7F70F230E79
:10C94000F4FC8607BD0793F7073F3301F1408A8A5D
:10C9500001498347C4FD6367F902CE85130584FC52
:10C96000232C54FD97000000E78000DE5281130164
:10C9700004FCF2506254D2544259B259225A925A8B
:10C9800021618280268597000000E780E0B493173C
:10C990001900D69705092390A7001379F90F55BF01
:10C9A00082809797FF1F9387A7499C43D847A16729
:10C9B00089076310F70A397106DE22DC26DA800067
:10C9C0004AD84ED652D456D23285328997000000CA
:10C9D000E78060AEAA894A8597000000E780C0AF73
:10C9E000835749000A8A2318A4FC858393F7F70F1D
:10C9F000230CF4FC8607BD0793F7073F3301F14092
:10CA00008A8A8144834784FD63E7F402CE85130557
:10CA100084FC232A54FD97000000E780E0D2528175
:10CA2000130104FCF2506254D2544259B259225AB2
:10CA3000925A216182804A8597000000E780C0A950
:10CA400093971400D69785042390A70093F4F40FCE
:10CA500055BF82809797FF1F9387873E9C43D84797
:10CA6000A1679387E704631EF70A397106DE22DCAB
:10CA700026DA80004AD84ED652D456D23285B284B5
:10CA800097000000E78020A3AA8926859700000070
:10CA9000E78080A42318A4FC268597000000E78087
:10CAA000A0A3231AA4FC268597000000E780C0A25B
:10CAB00083D744000A8A2319A4FC858393F7F70FD0
:10CAC000230EF4FC8607BD0793F7073F3301F140BF
:10CAD0008A8A01498347C4FD6367F902CE8513053D
:10CAE00084FC232C54FD97000000E780E0C55281B0
:10CAF000130104FCF2506254D2544259B259225AE2
:10CB0000925A21618280268597000000E780C09CB0
:10CB100093171900D69705092390A7001379F90FE9
:10CB200055BF82809797FF1F938787319C43D847D3
:10CB3000A1679387C704631AF70A397106DE22DCFE
:10CB400026DA80004AD84ED652D456D23285B284E4
:10CB500097000000E7802096AA89268597000000AC
:10CB6000E7808097FD572318A4FC2685231AF4FC40
:10CB700097000000E780409683D744000A8A231973
:10CB8000A4FC858393F7F70F230EF4FC8607BD07FB
:10CB900093F7073F3301F1408A8A01498347C4FD77
:10CBA0006367F902CE85130584FC232C54FD97009E
:10CBB0000000E78060B95281130104FCF250625416
:10CBC000D2544259B259225A925A21618280268502
:10CBD00097000000E780409093171900D697050949
:10CBE0002390A7001379F90F55BF82809797FF1FF5
:10CBF000938707259C43D847A167DD076317F70490
:10CC00001753FFFFE702A34D7971328532849700F5
:10CC10000000E780408A2AC6228597000000E7804E
:10CC2000A08B2311A102228597000000E780A08835
:10CC3000B2452300A102280897000000E780C0B099
:10CC400045611753FFFF6700C34B82809797FF1F13
:10CC50009387071F9C43D847A1679387870463176F
:10CC6000F7041753FFFFE702834779713285328457
:10CC700097000000E78020842AC6228597000000E4
:10CC8000E78080852311A102228597000000E780BC
:10CC90008082B2452300A102280897000000E780A7
:10CCA000A0AA45611753FFFF6700A34582809797AD
:10CCB000FF1F9387E7189C43D847A1679387A70472
:10CCC0006312F7021753FFFFE702634101112800C7
:10CCD000814597000000E78020A705611753FFFFFB
:10CCE0006700234282809797FF1F938767159C43B5
:10CCF000D847A167938757026319F7021753FFFFBD
:10CD0000E702E33D0111328597F0FFFFE780A07A4B
:10CD10002308A1008145280097000000E780C0A2F9
:10CD200005611753FFFF6700C33D82809797FF1F80
:10CD3000938707119C43D847A1679387E702631B3A
:10CD4000F7041753FFFFE70283390111328532845C
:10CD500097F0FFFFE7804078AA84228597F0FFFFD5
:10CD6000E7808077854709E9228597F0FFFFE78014
:10CD700080744205B337A000280081452318910034
:10CD80003ECA97000000E780209C05611753FFFF13
:10CD90006700233782809797FF1F9387670A9C431A
:10CDA000D84799476313F7081753FFFFE702233368
:10CDB00079713285328497F0FFFFE780C06F2AC611
:10CDC000228597F0FFFFE78020712310A1022285C2
:10CDD00097F0FFFFE780206E2301A102228597F0E4
:10CDE000FFFFE780406DA301A102228597F0FFFFBE
:10CDF000E780606C2302A102228597F0FFFFE780A5
:10CE0000806B2313A102228597F0FFFFE780A06AC1
:10CE1000B2452314A102280897000000E780C092C1
:10CE200045611753FFFF6700C32D82809797FF1F4F
:10CE3000938707019C43D847A1679387C703631370
:10CE4000F7081753FFFFE70283297971328532848F
:10CE500097F0FFFFE78020662AC6228597F0FFFF44
:10CE6000E78080672310A102228597F0FFFFE7800B
:10CE7000A0662311A102228597F0FFFFE780A0633F
:10CE80002302A102228597F0FFFFE780C062A30280
:10CE9000A102228597F0FFFFE780E0612303A10252
:10CEA000228597F0FFFFE7800061B245A303A1024E
:10CEB000280897000000E780208945611753FFFF8D
:10CEC0006700232482801753FFFFE70243210111EB
:10CED0002A8497F0FFFFE780005EAA84228597F0FE
:10CEE000FFFFE780605F228597F0FFFFE780C05E6D
:10CEF000035744008D4763F7E700228597F0FFFF53
:10CF0000E780805D228597F0FFFFE780E05C2800E6
:10CF1000A68597000000E780208305611753FFFF77
:10CF20006700231E9797FF1F938787F19C43D8477D
:10CF3000A167FD07631FF7001753FFFFE702231ADE
:10CF4000328597000000E78040F81753FFFF670025
:10CF5000431B82809797FF1F938787EE9C43D84798
:10CF6000A167E5076315F7081753FFFFE7022317CB
:10CF700079713285328497F0FFFFE780C0532AC66B
:10CF8000228597F0FFFFE7802055228597F0FFFF6D
:10CF9000E78080542310A102228597F0FFFFE780ED
:10CFA000A053520551812311A102228523020102BF
:10CFB00097F0FFFFE7802050A302A102228597F09F
:10CFC000FFFFE780404F2303A102228597F0FFFF78
:10CFD000E780604EB245A303A102280897F0FFFF47
:10CFE000E780807645611753FFFF670083118280D9
:10CFF0009797FF1F9387C7E49C43D847A167938700
:10D00000E703631FF7001753FFFFE702430D328565
:10D0100097000000E78060EB1753FFFF6700630E87
:10D0200082809797FF1F9387A7E19C43D847A1670A
:10D0300093874704631EF7021753FFFFE702230A93
:10D0400079713285328497F0FFFFE780C0462AC6A7
:10D05000228597F0FFFFE7802048B245280897F027
:10D06000FFFFE780606E45611753FFFF67006309AC
:10D0700082809797FF1F9387A7DC9C43D847A167BF
:10D08000938787026310F7041753FFFFE702230516
:10D0900079713285328497F0FFFFE780C0412AC65C
:10D0A000228597F0FFFFE7800041B2452300A102EF
:10D0B000280897F0FFFFE780206945611753FFFFBD
:10D0C0006700230482801753FFFFE7024301011129
:10D0D00097F0FFFFE780203EAA85280097F0FFFF2A
:10D0E000E780806605611753FFFF6700830197970C
:10D0F000FF1F9387E7D49C43D847A167D107631FDD
:10D10000F7001753FFFFE70283FD32859700000009
:10D11000E780A0FB1753FFFF6700A3FE828097976D
:10D12000FF1F9387E7D19C43D847A167C507631FBB
:10D13000F7001753FFFFE70283FA328597000000DC
:10D14000E780A0F81753FFFF6700A3FB8280979743
:10D15000FF1F9387E7CE9C43D847A167B907631F9A
:10D16000F7001753FFFFE70283F7328597000000AF
:10D17000E780A0F51753FFFF6700A3F88280979719
:10D18000FF1F9387E7CB9C43D847A167AD07631F79
:10D19000F7001753FFFFE70283F432859700000082
:10D1A000E780A0F21753FFFF6700A3F582809797EF
:10D1B000FF1F9387E7C89C43D84789476318F70246
:10D1C0001753FFFFE702A3F10111328532C897F030
:10D1D000FFFFE780402EAA85280097F0FFFFE78039
:10D1E000A05605611753FFFF6700A3F18280979750
:10D1F000FF1F9387E7C49C43D847A1678D0763113E
:10D20000F7041753FFFFE70283ED011132853284E3
:10D2100097F0FFFFE780202A13066100AA844C00E4
:10D22000228597300000E78000232800A68597F02C
:10D23000FFFFE780605105611753FFFF670063EC54
:10D2400082809797FF1F9387E7BF9C4381CFDC4382
:10D2500091CB1753FFFFE70283E882971753FFFF35
:10D26000670023EA82801753FFFFE70243E77971E3
:10D270003C08AE843ED2A165B7070A002A843ED49A
:10D2800048103C08DD053ED636C432C63AC297D0B7
:10D29000FFFFE780402C12474810BA8597F0FFFF48
:10D2A000E780C01332464810B28597F0FFFFE78051
:10D2B000E014A2464810B68597F0FFFFE780001201
:10D2C000501001478146A685228597D0FFFFE78051
:10D2D000E04D45611753FFFF6700A3E21753FFFFBF
:10D2E000E702E3DF01117C000329C501AE843ECAD9
:10D2F000A165B70707002A843ECC48087C00C50515
:10D300003ECE97D0FFFFE78000258345D90048082F
:10D3100097F0FFFFE780800C500801478146A68503
:10D32000228597D0FFFFE780604805611753FFFF14
:10D33000670023DD1753FFFFE70263DA83C7950019
:10D3400093F7F707A384F50097000000E78040F902
:10D350001753FFFF6700E3DA1753FFFFE70223D8F5
:10D3600079713C08AE843ED2A165B70709002A84D2
:10D370003ED448103C08938545043ED632C636C498
:10D3800097D0FFFFE780201DA2464810B68597F092
:10D39000FFFFE780A00432464810B28597F0FFFFF8
:10D3A000E780C005501001478146A685228597D0A9
:10D3B000FFFFE780A03F45611753FFFF670063D47D
:10D3C0001753FFFFE702A3D183C7950041112A84B9
:10D3D00093F7F707A384F50032852EC697F0FFFF79
:10D3E000E780800F85672AC46370F502977000009C
:10D3F000E78060E82246B24509ED11478146228563
:10D4000097000000E78060E641011753FFFF6700C7
:10D4100043CF01478346F501DDB71753FFFFE7020E
:10D4200063CA01113C003ECAB7070A003ECC3C006B
:10D430003ECE83C79500AA89328593F7F707A38468
:10D44000F5002E8497F0FFFFE78000098567637D74
:10D45000F504A165AA8493858504480897D0FFFF49
:10D46000E780600F268597700000E780C0E02A897A
:10D4700029E19145480897F0FFFFE78020F6A6854F
:10D48000480897F0FFFFE78060F7CA85480897F0E3
:10D49000FFFFE780A0F4014781465008A2854E8532
:10D4A00097D0FFFFE780803005611753FFFF6700CB
:10D4B000A3C48145480897F0FFFFE78020F20349A5
:10D4C000090275BF1753FFFFE702C3BF79711C1034
:10D4D0003ECAB7070F003ECC404D1C10AA84AE894F
:10D4E0004808994532C636893ECE97D0FFFFE7807F
:10D4F000800632464808B28597F0FFFFE78000EECD
:10D50000630C0902A545480897F0FFFFE780C0E6D5
:10D510002546CA8597200100E78060A3500801478F
:10D520008146CE85268597D0FFFFE780202845617C
:10D530001753FFFF670043BC8355C402480897F0A8
:10D54000FFFFE780A0EB0355E402814505C5854751
:10D5500085456301F502C167FD179305F00F630B65
:10D56000F5007D1597700000E780608D930515002C
:10D5700093F5F50F480897F0FFFFE78020E6834515
:10D580000403480897F0FFFFE78040E58345140354
:10D59000480897F0FFFFE78060E4835524034808BC
:10D5A00097F0FFFFE78080E583554403480897F034
:10D5B000FFFFE780A0E49DB71753FFFFE70223B208
:10D5C00083C795008146014693F7F707A384F500CA
:10D5D00097000000E78040EF1753FFFF670063B23A
:10D5E0001753FFFFE702A3AF79713E841C103ECAB8
:10D5F0002E89B7070F00A1653ECCFD051C10AA843B
:10D60000480842C03AC23ECE36C432C697D0FFFF69
:10D61000E78060F432464808B28597F0FFFFE78064
:10D62000E0DBA2464808B68597F0FFFFE78000DD03
:10D6300012474808BA8597F0FFFFE78020DC0248D0
:10D64000630C08029145480897F0FFFFE780C0D2BD
:10D650001146A28597200100E780608F500801479E
:10D660008146CA85268597D0FFFFE7802014456153
:10D670001753FFFF6700E3A88945480897F0FFFFAD
:10D68000E78080CF834704002300F5008347140020
:10D69000A300F500E1B71753FFFFE702A3A283C77A
:10D6A000950001112A8A93F7F707A384F5003285C4
:10D6B000AE8432C697F0FFFFE78000E232462A8947
:10D6C000328597F0FFFFE78000DF85676373F9021B
:10D6D000AA894A8597700000E780E0B92A8419ED8D
:10D6E000114781464A86A685528597000000E7804B
:10D6F000C0B705611753FFFF670003A09387E9FFD9
:10D7000093F7F70F0547E366F7FE8347F50195EBBF
:10D710008947E380F9FE8346F401528501474A8632
:10D72000A68597000000E78040B4A167D9074808A4
:10D730003ECC230A010002CE97000000E780A0B093
:10D740004DBF639EE7008947639EF9009307102051
:10D75000231FF50097700000E78000B76DBF0947F1
:10D76000E39BE7FA8D47E398F9FA2285977000006A
:10D77000E780C0DE9797FF1F9387C78B9C4399E78D
:10D780009787FF1F9387C7749C4399C703D50400ED
:10D7900097800000E780E0CD231F040022855DBF55
:10D7A0001753FFFFE702A39301113C003ECAB707DE
:10D7B0000B003ECC3C003ECE83C795002A893285C3
:10D7C00093F7F707A384F500AE8497F0FFFFE78097
:10D7D000A0D093170501C187635AF006A1652A847A
:10D7E0009385E502480897D0FFFFE780C0D6A28561
:10D7F000480897F0FFFFE78060C09787FF1F938777
:10D80000276D9C43A9EB01449375F40F480897F0EA
:10D81000FFFFE780A0BC9355844093F5F50F4808BF
:10D8200097F0FFFFE78080BB9355044193F5F50F18
:10D83000480897F0FFFFE78060BA0147814650082B
:10D84000A6854A8597D0FFFFE78040F6056117530C
:10D85000FFFF6700038B416585460546A2857D1560
:10D8600097500000E780A0BC59DD510597000100EA
:10D87000E780C08E130440063344850271B7175306
:10D88000FFFFE702C3850111B70706003EC683C745
:10D89000950021642A8993F7F707A384F500AE84E5
:10D8A00028009305A4040AC40AC897D0FFFFE780A4
:10D8B00080CA300001478146A6854A8597D0FFFF80
:10D8C000E780C0EE97E0FFFFE780E01113049404C7
:10D8D000480822CC230A010002CE97000000E7800E
:10D8E000809605611753FFFF6700A3811743FFFF71
:10D8F000E702437DC1642A8901449789FF1F938908
:10D90000E974130A8002FD1497E0FFFFE780E0BD91
:10D910006347A40001451743FFFF6700E37DB3079A
:10D92000440303A7C90ABA9703D707006306970001
:10D9300083D72700638427010504F9B70545E1BFB4
:10D940001743FFFFE70203782A8A2E8999C123A093
:10D95000050081498144978AFF1F938AEA4E614BF3
:10D9600097E0FFFFE780A0BE63C7A4004E85174382
:10D97000FFFF670063783384640383A70A003E9443
:10D980008357040099E76304090023208900850474
:10D99000C1BF4146D2851305440097100100E780BE
:10D9A000A05875F5A289E5B71743FFFFE702837119
:10D9B00039717C083ED4B7070A003ED67C083ED8B1
:10D9C00083C795002A8A328593F7F707A384F50069
:10D9D0002E8932C697F0FFFFE78000B0856763733A
:10D9E000F5083246AA84328597F0FFFFE780A0ACA5
:10D9F0008547AA8963E8A706A16593858504281051
:10DA000097D0FFFFE78020B5268597700000E7805C
:10DA100080862A8429ED9145281097F0FFFFE78042
:10DA2000E09BA685281097F0FFFFE780209DCE851C
:10DA3000281097F0FFFFE780609A01478146301079
:10DA4000CA85528597D0FFFFE78040D6A1679387AC
:10DA5000770448183EDC230A010202DE97F0FFFF3C
:10DA6000E780607E21611743FFFF6700E36881451F
:10DA7000281097F0FFFFE7806096A685281097F0A2
:10DA8000FFFFE780A0979797FF1F9387E7929C433C
:10DA900081CB22856389090097D00000E78080232D
:10DAA0008345040271B797D00000E7800022CDBF04
:10DAB0001743FFFFE702036183C795004111AA895D
:10DAC00093F7F707A384F5003285AE84328A97F086
:10DAD000FFFFE78060A08567637FF5022A89976072
:10DAE0000000E78040792A84914631C58347F501DB
:10DAF00005476387E70291C70D476366F704AD46A4
:10DB00001DA89305050303250A004146971001004F
:10DB1000E78080410DE941011743FFFF6700C35DC6
:10DB20009305950803250A00414697100100E780F8
:10DB3000A03F814669F54A86A6854E85970000007C
:10DB4000E780C081C9BF83250A0013059408977038
:10DB50000000E780E02819C1C146F1BF9787FF1F89
:10DB60009387474D9C4399E79787FF1F93874736D5
:10DB70009C4399C7228597800000E780608969FDF2
:10DB80008547A30FF400228597B00000E780A083AB
:10DB9000228597600000E78020734E8581464A8683
:10DBA000A68597F0FFFFE780607BA1679387570406
:10DBB00048003EC42302010002C697F0FFFFE78041
:10DBC000806891BF1743FFFFE702E34E83C79500CC
:10DBD0004111AA8993F7F707A384F50032852E89AE
:10DBE000B28A97F0FFFFE780208F85676374F50E98
:10DBF000AA8497600000E78000682A840DED416BDD
:10DC0000014A978BFF1F938B6B44130C400E7D1BB7
:10DC100019A833048A0383A70B0B3E948357C401CE
:10DC200063836705050A97E0FFFFE780008BE34207
:10DC3000AAFE95460DA08357C501639697029305EA
:10DC4000050303A50A00414697100100E780C02D97
:10DC5000994611E181462686CA854E8597F0FFFFD9
:10DC6000E780C06F85A883A50A0013050403977099
:10DC70000000E780E016C14679FD2285231E94004E
:10DC800097A00000E7802074228597600000E7805D
:10DC9000A0639787FF1F938727729C43A9C3230024
:10DCA0000402228597D00000E78080EF4E858146F0
:10DCB0002686CA8597F0FFFFE780406AA1679387B1
:10DCC000070448003EC42302010002C697F0FFFF8C
:10DCD000E780605741011743FFFF670043418947D1
:10DCE0002300F402E1B7397106DE22DC4AD8800055
:10DCF00052D456D25AD026DA4ED65ECE2E8A3289E9
:10DD00002A8B97D0FFFFE780407A0605710541997D
:10DD10008A8A3301A140232224FC231404FC97D0D7
:10DD2000FFFFE780807883479A000605350593F763
:10DD3000F7072315A4FCA304FA004A85232624FC34
:10DD400097E0FFFFE780407993170501C1876340A3
:10DD5000F0025681130104FCF2506254D25442592D
:10DD6000B259225A925A025BF24B21618280AA84F4
:10DD70004A8597E0FFFFE7802076AA894A8597E0E9
:10DD8000FFFFE7806075A1659385C5022A891305A9
:10DD900044FC97C0FFFFE780007C268597C0FFFF0B
:10DDA000E7804070854511C94A86CE8597C0FFFF40
:10DDB000E780C069AA8B21E98945130544FC97E0F7
:10DDC000FFFFE780A061A685130544FC97E0FFFFF5
:10DDD000E780C062CE85130544FC97E0FFFFE78033
:10DDE000E061CA85130544FC97E0FFFFE78000610E
:10DDF00001478146130644FCD2855A8597D0FFFF20
:10DE0000E780C09AB9B78145130544FC97E0FFFF4E
:10DE1000E780C05CA685130544FC97E0FFFFE78020
:10DE2000E05DCE85130544FC97E0FFFFE780005DD1
:10DE3000CA85130544FC97E0FFFFE780205C81441E
:10DE400097D0FFFFE7806066E3D4A4FA83A70B01B5
:10DE500013971400BA9783D5070099C5130544FC9E
:10DE600097E0FFFFE78080598504D9BF797106D616
:10DE700022D44AD000184ECE52CC56CA26D25AC806
:10DE8000AE893289AA8A97D0FFFFE7800062060533
:10DE9000690541990A8A3301A140232A24FC231CE5
:10DEA00004FC97D0FFFFE780406083C79900060518
:10DEB0002D0593F7F707231DA4FCA384F9004A85D9
:10DEC000232E24FC97E0FFFFE780006193170501F4
:10DED000C187634FF0005281130104FDB2502254F8
:10DEE00092540259F249624AD24A424B45618280B9
:10DEF000AA844A8597E0FFFFE780005EA1659385CD
:10DF0000A5022A89130544FD97C0FFFFE780A0649E
:10DF1000268597C0FFFFE780E058854509C9CA8577
:10DF200097C0FFFFE78080552A8B29E189451305BB
:10DF300044FD97E0FFFFE780604AA685130544FD96
:10DF400097E0FFFFE780804BCA85130544FD97E00B
:10DF5000FFFFE780A04A01478146130644FDCE85B6
:10DF6000568597D0FFFFE7806084B5B781451305DC
:10DF700044FD97E0FFFFE7806046A685130544FD5A
:10DF800097E0FFFFE7808047CA85130544FD97E0CF
:10DF9000FFFFE780A046814497D0FFFFE780E05075
:10DFA000E3DBA4FA83270B0113971400BA9783D5F8
:10DFB000070099C5130544FD97E0FFFFE780004483
:10DFC0008504D9BF1743FFFFE7026311834745006C
:10DFD000404DD5EFFD575DC4834694000947636308
:10DFE000D70A0346B400854663EEC6088306E400FC
:10DFF00063CA06085C45F9562390D7009787FF1F30
:10E0000083C7C7E499E3A304E4009787FF1F9387BE
:10E0100027EC9C4381E78947A306F4009787FF1FFD
:10E02000938787399C4381E789472306F400970546
:10E03000000093854506AA841305040197F00000AB
:10E04000E780600FFD57231AF40281471CDC01486A
:10E050009787FF1F23A887DE9787FF1F9387C7DE59
:10E06000232E040304C0804397D0FFFFE780204E97
:10E0700061463306C502814522859740FFFFE78050
:10E08000000981473E851743FFFF67008307FD575F
:10E09000D5BF1743FFFFE70283042A8403554502D7
:10E0A00097600000E780201D19E5231E0400174338
:10E0B000FFFF670003058357E401F5DB930504FFC9
:10E0C00017450100130585E597E00000E78020145F
:10E0D000F9BF1743FFFFE70283002E89A1654111B5
:10E0E0009385E5032A8436C432C6BE843AC297C0FB
:10E0F000FFFFE780404612472285BA8597E0FFFF81
:10E10000E780C02D32462285B28597E0FFFFE78089
:10E11000E02EA2462285B68597E0FFFFE780002E1D
:10E12000630309029145228597E0FFFFE780C02441
:10E130001146A68597100100E78060E14101174371
:10E14000FFFF670003FC8945228597E0FFFFE7801A
:10E15000A02283C704002300F50083C71400A30096
:10E16000F500E9BF1743FFFFE70263F783C7950098
:10E17000444D054793F7F707A384F5001C4241116E
:10E1800083C707006367F7062E842A89B1C003C7D7
:10E19000D400630FF7021787FF1F130767D31843D5
:10E1A00005C3A386F40097A00000E780804983C7D9
:10E1B000D40099E741657D1597400000E780802FE6
:10E1C00083D72403918B89C797E00000E780001371
:10E1D0004A85A28597F0FFFFE7808010A167C107FD
:10E1E00048003EC42302010002C697F0FFFFE7800B
:10E1F000800541011743FFFF6700A3F01743FFFFAE
:10E20000E702E3ED03D745008D47AA8441112E8430
:10E2100032892E8563E3E70297E0FFFFE780C02B9A
:10E22000AA8523000900268597C0FFFFE780002507
:10E2300041011743FFFF6700C3EC97E0FFFFE78052
:10E24000A0292AC6228597E0FFFFE780E028B24593
:10E2500085472A862300F900268597C0FFFFE780BF
:10E26000E01EF9B7397106DE22DC26DA80004ED6D0
:10E2700052D456D24AD85AD05ECEAE89B284AA8A37
:10E2800097D0FFFFE780602106051305250241991D
:10E290000A8A3301A140232224FC231404FC97D0D2
:10E2A000FFFFE780801F83C7990006054D0593F7A0
:10E2B000F7072315A4FCA384F9002685232624FC54
:10E2C00097E0FFFFE780402193170501C187634076
:10E2D000F0025281130104FCF2506254D2544259AC
:10E2E000B259225A925A025BF24B21618280AA8B68
:10E2F00003AB040097C0FFFFE780C01A51E583D746
:10E30000440001498544F11793B71700A301F4FCB9
:10E31000834734FCA165C9C79385E504130544FC14
:10E3200097C0FFFFE7802023A685130544FC97E0F4
:10E33000FFFFE780A00ADE85130544FC97E0FFFF9E
:10E34000E780C00B834734FC114691E30946DA8528
:10E35000130544FC97E0FFFFE78060058144630AF2
:10E360000900416B7D1B97D0FFFFE780001363CC52
:10E37000A40201478146130644FCCE85568597C00A
:10E38000FFFFE780A042B1B7A685130634FC9700D3
:10E390000000E780E0E6933415002A8986048DBFEB
:10E3A0009385C504A5BF8327C90013971400BA97A6
:10E3B00083D5070063886501130544FC97E0FFFFE0
:10E3C000E780C003850445B71743FFFFE702A3CEEC
:10E3D00079711C103EC4B7070F003EC61C103EC822
:10E3E00083C79500AA8A328593F7F707A384F500BF
:10E3F000AE89328497E0FFFFE780000E9317050196
:10E40000C187635AF0062A8A228597E0FFFFE780DA
:10E41000A00C2A895285032B040097C0FFFFE780D8
:10E42000600839ED8357440081440544F11793B7E0
:10E430001700A303F10083457100DA872287CA869B
:10E440005286280097000000E780E0C80147814617
:10E450003000CE85568597C0FFFFE7802035A16745
:10E460009387D70348083ECC230A810026CE97F035
:10E47000FFFFE78040DD45611743FFFF670023C7CB
:10E48000A2851306710097000000E78060D7AA8478
:10E49000094455D13544E30055FB4A8597F0FFFF09
:10E4A000E78000450D4441D9014497D0FFFFE78044
:10E4B000C0FE634DA400C16B0144FD1B97D0FFFF5C
:10E4C000E780A0FD634EA4001544B5B7DC441317E4
:10E4D0001400BA9783D70700638327030504F1B7B5
:10E4E000D84493171400BA9703D70700631B77012A
:10E4F00023902701268597A00000E780C0DA014419
:10E500001DBF050465BF1743FFFFE702A3BB83C719
:10E51000950041112A8A93F7F707A384F500328505
:10E520002E89328497E0FFFFE78000FB93170501F7
:10E53000C1876353F006AA89228597E0FFFFE78031
:10E54000A0F92311A1004E85832A040097C0FFFF84
:10E55000E78040F539E58357440085440144F117CD
:10E5600093B71700A300F1000348110003572100DF
:10E57000D6875285CE862686CA8597F0FFFFE7802C
:10E580006006A167F10748003EC42302910022C63D
:10E5900097F0FFFFE78020CB41011743FFFF6700A3
:10E5A000A3B5A2851306110097000000E78040C5BF
:10E5B0002A84894455D98357210011678544BA9725
:10E5C000C2071167C1831307F7EFE36FF7F8978767
:10E5D000FF1F938727A69C4381CB85451305210008
:10E5E00097500000E78060748355210022858144A4
:10E5F00097C0FFFFE780A0E125D923100500228501
:10E6000097A00000E78080CC85B71743FFFFE702A3
:10E6100083AA83C7950041112A8B93F7F707A38438
:10E62000F50032852E8A328497E0FFFFE780C0EA4A
:10E6300093170501C1876351F006AA8A228597E0E6
:10E64000FFFFE78060E92A895685832B040097C085
:10E65000FFFFE78020E531E583574400814405440E
:10E66000F11793B71700A301F10003483100DE87CB
:10E670005A854A87D6862286D28597F0FFFFE780A3
:10E6800060F6A167ED0748003EC42302810026C65C
:10E6900097F0FFFFE78020BB41011743FFFF6700B2
:10E6A00003A5A2851306310097000000E78040B55E
:10E6B000AA8409445DD99167CA97C2071167C183CB
:10E6C0001307F7EF0544E362F7FACA8597C0FFFF27
:10E6D000E780E0D3014451F9814997D0FFFFE780FB
:10E6E000C0DC63DBA900984893971900BA9703D759
:10E6F000070005EF2390270197D0FFFFE780E0DABE
:10E700001544E384A9F6268597A00000E78000BCA5
:10E710009787FF1F938707929C430144B9D74A8587
:10E7200097500000E780005889B785097DB71743E7
:10E73000FFFFE702239979713E847C083EC82E8A48
:10E74000B7071400A1653ECAE5057C08AA89080838
:10E7500036C4428932C6BA8AC6843ECC97C0FFFF0F
:10E76000E78060DFCA85080897E0FFFFE78000C701
:10E7700032460808B28597E0FFFFE78020C8A2462E
:10E78000630A09049D45080897E0FFFFE780C0BEC3
:10E790001D4681459740FFFFE780609763890A081F
:10E7A0009145080897E0FFFFE78000BD1146A68568
:10E7B00097000100E780A079100801478146D285C3
:10E7C0004E8597C0FFFFE78060FE45611743FFFF5E
:10E7D00067008392B685080897E0FFFFE78000C2D4
:10E7E0001C400808D8439355C701858912075183F7
:10E7F000B205D98D97E0FFFFE78040C01C400808B4
:10E8000083C5870097E0FFFFE78040BD1C400808F4
:10E8100083C5A70097E0FFFFE78040BC1C400808C5
:10E8200083C5970097E0FFFFE78040BB85BF894520
:10E83000080897E0FFFFE78020B483C704002300A7
:10E84000F50083C71400A300F500BDB71743FFFF11
:10E85000E702438783C795004111AA8993F7F70719
:10E86000A384F5003285AE84328497E0FFFFE78011
:10E87000A0C693170501C187635DF0042A89032AA6
:10E88000040097C0FFFFE780E0C119E98357440007
:10E890000548F11793B71700A307F100814631A887
:10E8A0001306F100A28597000000E78060951DC562
:10E8B0001C459DC783D6470001480347F1009307D5
:10E8C0008500D2884A86A6854E8597000000E7809D
:10E8D00040E641011743FFFF6700038209487DBFFF
:10E8E0001D486DBF1733FFFFE702C37D65715C08EC
:10E8F0003EC4B7077B013EC65C083EC883C795008F
:10E900002A8A328593F7F707A384F500AE8997E04A
:10E91000FFFFE78040BA8357E100E1C7894528003F
:10E9200097C0FFFFE78020C38145280097E0FFFFE5
:10E93000E780C0AA97C0FFFFE78000C99787FF1F45
:10E94000938787A79C431774FF1F03442450AA840E
:10E950003334800099C3136424009777FF1F938793
:10E9600027579C4399C3136444009777FF1F9387ED
:10E97000676C9C4399C31364840083D5040028000A
:10E98000014997E0FFFFE78060A783D524002800B6
:10E9900097E0FFFFE78080A683D54400280097E03A
:10E9A000FFFFE780A0A597D0FFFFE78000AB93159E
:10E9B0000501C181280097E0FFFFE78020A4A28520
:10E9C000280097E0FFFFE78060A39C446360F902A2
:10E9D000014781463000CE85528597C0FFFFE78012
:10E9E000E0DC59611733FFFF67000371DC44131447
:10E9F000490028003E9497E0FFFFE7806096834738
:10EA000044000347540089070607BA978607E36A5C
:10EA1000F5FC835524002800814A97E0FFFFE7803A
:10EA2000E09D83454400280097E0FFFFE780009BBE
:10EA300083455400280097E0FFFFE780209A834732
:10EA4000440063C9FA00814A8347540063C1FA0253
:10EA50000509A5BF1C4413975A002800BA9783D50F
:10EA60000700850A97E0FFFFE7804099C9BF032BA5
:10EA7000C40093975A0028003E9B83552B00850ABB
:10EA800097E0FFFFE780809783550B00280097E011
:10EA9000FFFFE780A0964DBF1733FFFFE702236417
:10EAA0005C4993E717005CC997A00000E78060B558
:10EAB0001733FFFF6700E3641733FFFFE7022362AA
:10EAC0002E84814597F0FFFFE780C0E705C5835797
:10EAD0000500FD172310F50009C4835725002310F6
:10EAE000F40097000000E78060FB01451733FFFF4B
:10EAF0006700236131457DD823100400C5BF17335B
:10EB0000FFFFE702235C83C7950041112A8A93F730
:10EB1000F707A384F50032852E89328497E0FFFF42
:10EB2000E780809B93170501C1876356F006AA8989
:10EB3000C145228597E0FFFFE780A0802A8B4E85A4
:10EB4000832A040097C0FFFFE780C09531E983570F
:10EB50004400231101000544F11793B71700A300E7
:10EB6000F10081440348110003572100D6875285E4
:10EB7000CE862286CA8597F0FFFFE780A0A6A16710
:10EB80009387170248003EC42302810026C697E0FF
:10EB9000FFFFE780406B41011733FFFF6700C3555C
:10EBA00013061100A28597F0FFFFE7806065AA8435
:10EBB00009E523110100094475B7930521005A8521
:10EBC00097000000E78080EF835721002A84D9DB7B
:10EBD0009777FF1F938707469C4381CB8545130595
:10EBE000210097500000E7804014835521002685BE
:10EBF000314497C0FFFFE78080812DD523100500A9
:10EC0000268597900000E780606C0144A1BF173310
:10EC1000FFFFE702C34C41112E896C00AA8402C693
:10EC200097F0FFFFE78000D20DC1035705000507ED
:10EC30002310E50097000000E78040E681473E850D
:10EC400041011733FFFF6700C34B3247954765DB30
:10EC5000CA85268597300000E780800CC147E340D5
:10EC600005FE3244854741462310F40083570900CE
:10EC7000A685130544002311F40097000100E780E6
:10EC8000002D228545BF1733FFFFE702A34383C74B
:10EC900095004111AA8A93F7F707A384F5003285FE
:10ECA000AE89328497E0FFFFE78000839317050168
:10ECB000C1876356F0062A8AC145228597D0FFFF97
:10ECC000E7802068AA845285032B040097B0FFFFD9
:10ECD000E780407D31E983574400231101008544DA
:10ECE000F11793B71700A300F10001440348110086
:10ECF00003572100DA875685D2862686CE8597F07F
:10ED0000FFFFE780208EA1679387070248003EC47B
:10ED10002302910022C697E0FFFFE780C052410125
:10ED20001733FFFF6700433DA2851306110097F0DC
:10ED3000FFFFE780E04C2A8409E5231101008944A4
:10ED400075B726859305210097000000E78060ECE9
:10ED5000AA8449FD83552100228597B0FFFFE780F3
:10ED6000006B49F5014997C0FFFFE7800074635DC0
:10ED7000A900184893171900BA9703D707000DEF99
:10ED8000035721002390E70097C0FFFFE780E07161
:10ED9000630625039777FF1F9387C7299C4399C76D
:10EDA0000355210097500000E780C0EF228597901F
:10EDB0000000E780A0511DBF050975B795443DB718
:10EDC00005C19307F00F630FF500C547630CF5000D
:10EDD0009307F5FF05453315F50042054181828013
:10EDE0000145828041657D158280B9E91733FFFFB7
:10EDF000E702E32E03450603328497000000E78014
:10EE000060FC9305803EB305B502C205C18181CD8A
:10EE10000357E402854763F8E7001305040197E010
:10EE20000000E78060418357E40241677D176385F6
:10EE3000E700FD172317F4021733FFFF6700632C69
:10EE400082801733FFFFE7020327004283C7950044
:10EE5000444D0349140093F7F707A384F500834753
:10EE60000400220911673369F900A167B347F9006B
:10EE700041112A8BAE8A63ECE70E83472400130707
:10EE8000C00EB91793F7F70F6373F71003473400F9
:10EE9000C14763EEE70E834744001307E00793C7BB
:10EEA00007086371F70C8349840083477400A20943
:10EEB000B3E9F900856763F7F90A034A64008347F9
:10EEC00054004E85220A336AFA0097500000E7800A
:10EED000803A61C123962403834B3400137AFA00ED
:10EEE000239A3403238874032399440393890401E8
:10EEF000631C090023A60402239804024E8597E0B0
:10EF00000000E780A0353DA0034924004A85970012
:10EF10000000E78020EB2397A402834744004E853E
:10EF2000A388F402E38D0BFCE30B09FC97E00000DF
:10EF3000E780602E97900000E7804072814601468E
:10EF4000D6855A8597E0FFFFE7800058A167938731
:10EF500097033EC423020100480002C697E0FFFF6A
:10EF6000E780602E41011733FFFF67004318854497
:10EF7000A2862686D6855A8597E0FFFFE780C05493
:10EF8000A167938797033EC423029100F1B7BD4464
:10EF9000C5B79144F1BF1733FFFFE702A312011178
:10EFA0001C08404D3EC2B7070F003EC41C083EC6B9
:10EFB0002A89AE8997C0FFFFE78000D7585C1C5CA8
:10EFC0006346B70E6394E50063E2A70E3385A7405E
:10EFD000B3B7A700B305B7401306803E81469D8DA9
:10EFE00097000100E780C0B693140501C180A165B8
:10EFF0009385C503480097B0FFFFE780C055814562
:10F00000480097D0FFFFE780603D83550404480027
:10F0100097D0FFFFE780803E83552404480097D0B7
:10F02000FFFFE780A03D814589CCC167FD179305AF
:10F03000F00F6388F400268597500000E78020E0F9
:10F04000AA85480097D0FFFFE78040390355440464
:10F05000814501CDC167FD179305F00F6307F500EA
:10F0600097500000E780A0DDAA85480097D0FFFFF9
:10F07000E780C03683456404480097D0FFFFE780EF
:10F08000E03583457404480097D0FFFFE7800035E2
:10F09000500001478146CE854A8597B0FFFFE78043
:10F0A000E07005611733FFFF67000305814481B7F6
:10F0B0001733FFFFE702A30283C7950093F7F70713
:10F0C000A384F50097000000E78020ED1733FFFFD1
:10F0D000670023031733FFFFE702C3FE83C79500D2
:10F0E0004111404D93F7F707A384F5002A8A328532
:10F0F000B284AE8997D0FFFFE780003E2A8B268539
:10F1000097D0FFFFE780403D2A89268597D0FFFFF3
:10F11000E780603A93170B0163CA0702E177CA9749
:10F12000C207C183116763E3E70293070910C207AF
:10F13000C1831307B00F637BF70093170901C187E1
:10F14000AA8A634AF000C54763FE5701410117339D
:10F15000FFFF670063FA97B0FFFFE7802025E31702
:10F1600025FFD5B763080B02630609028144638952
:10F170000A02B7077F0023106405231124057CC011
:10F18000568597000000E780E0C39304803EB304F7
:10F19000950239A0B7077F00232004047CC0814476
:10F1A0000355240497E00000E780E0A2A1C497C0C3
:10F1B000FFFFE78060B7269593D7F441333795007A
:10F1C000AE97BA9708DC5CDCCE85528597000000CC
:10F1D000E780A0DC99E023220404A1679387B703AA
:10F1E00048003EC42302010002C697E0FFFFE7800B
:10F1F0008005A9BF814701481CDC232E0403E9B721
:10F200001733FFFFE702A3ED97C0FFFFE78020342D
:10F21000E1473305F502914597500000E78040C46F
:10F22000E55711C59777FF1F23A0A7C281473E85E9
:10F230001733FFFF6700E3EC1733FFFFE70223EA12
:10F240009777FF1F938707C080433DC0835704040F
:10F250006390A70683572404639CB7043689B2845D
:10F2600097C0FFFFE78040AC5C5C63C3B704639565
:10F27000B7001C5C63EEA7028347640463F3F400E9
:10F28000A6872303F4048347740463F39700A687D7
:10F29000A303F4048357440441677D176385E700A3
:10F2A00085072312F4043C4481C7CA8526858297CA
:10F2B0001733FFFF6700E3E49777FF1F938787B853
:10F2C0009C43014599C303C5870082801733FFFF24
:10F2D000E702E3E00111B70707003EC683C79500C8
:10F2E000584D0AC493F7F7070AC8A384F5002A8982
:10F2F000AE8411CB1C4283C707002304F70097900C
:10F300000000E7800034216493055402280097B080
:10F31000FFFFE780402497000000E78020FAAA85DD
:10F32000280097D0FFFFE780600B3000014781463F
:10F33000A6854A8597B0FFFFE78040471304440243
:10F34000480822CC230A010002CE97E0FFFFE780A5
:10F3500080EF05611733FFFF6700A3DA1733FFFF64
:10F36000E702E3D701117C003ECAB70707003ECC95
:10F370007C003ECE83C795002E84AA8493F7F707BE
:10F38000A384F500A16593855502480897B0FFFF57
:10F39000E780601C97000000E78040F2AA854808DB
:10F3A00097D0FFFFE7808003500801478146A28580
:10F3B000268597B0FFFFE780603F05611733FFFFA9
:10F3C000670023D49777FF1F9387C7A79C430945FE
:10F3D00099C303C5970082809777FF1F938787A6FD
:10F3E0009C43094599C303C5D70082809777FF1FC7
:10F3F000938747A59C43014599C303C5A700828015
:10F400001733FFFFE70203CC0111B70708003EC620
:10F4100083C79500404D0AC493F7F7070AC8A38431
:10F42000F5002A89AE8429C41442854703C7060023
:10F4300063E0E70A83479400094681496380C70275
:10F44000B307F740A304E400B339F00083C7160004
:10F450002305F40097900000E780A01E03572403C3
:10F46000058B19C76386090097D00000E78000E983
:10F47000216493058402280097B0FFFFE780A00D68
:10F4800097000000E78040F4AA85280097D0FFFF8E
:10F49000E780C0F497000000E78080F5AA85280087
:10F4A00097D0FFFFE78080F3014781463000A685B3
:10F4B0004A8597B0FFFFE780602F13047402480865
:10F4C00022CC230A010002CE97E0FFFFE780A0D7FD
:10F4D00005611733FFFF670023C21733FFFFE70201
:10F4E00003C001117C003ECAB70708003ECC7C0077
:10F4F0003ECE83C795002E84AA8493F7F707A38492
:10F50000F500A16593858502480897B0FFFFE78065
:10F51000800497000000E78020EBAA85480897D078
:10F52000FFFFE780A0EB97000000E78060ECAA8572
:10F53000480897D0FFFFE78060EA500801478146FE
:10F54000A285268597B0FFFFE78040260561173327
:10F55000FFFF670003BB9777FF1F9387A78E9C432E
:10F56000014599C303C5B70082801733FFFFE70247
:10F5700003B70111B70707003EC683C79500404D8A
:10F580000AC493F7F7070AC8A384F5002A89AE8452
:10F5900005C81C42054783C707006368F706034791
:10F5A000B400630FF700A305F40097900000E78014
:10F5B00040098347B400B9CF97D0FFFFE78000BF71
:10F5C00021649305B400280097B0FFFFE780A0F8FE
:10F5D00097000000E78060F8AA85280097D0FFFF19
:10F5E000E780C0DF014781463000A6854A8597B095
:10F5F000FFFFE780A01B2904480822CC230A010052
:10F6000002CE97E0FFFFE78000C405611733FFFFDC
:10F61000670023AF97D0FFFFE780E0BF55B71733F0
:10F62000FFFFE702C3AB01117C003ECAB70707002A
:10F630003ECC7C003ECE83C795002E84AA8493F7EF
:10F64000F707A384F500A165AD05480897B0FFFF53
:10F65000E78060F097000000E78020F0AA85480866
:10F6600097D0FFFFE78080D7500801478146A285E9
:10F67000268597B0FFFFE780601305611733FFFF12
:10F68000670023A89767FF1F9387C77B9C430945A3
:10F6900099C303C5C70082801733FFFFE70223A485
:10F6A00001117C00AE843ECAA165B70707002A8419
:10F6B0003ECCD1057C0048083ECE97B0FFFFE780E6
:10F6C00080E997000000E78020FCAA85480897D0D1
:10F6D000FFFFE780A0D0500801478146A68522851C
:10F6E00097B0FFFFE780800C05611733FFFF6700CD
:10F6F00043A11733FFFFE702839E83C7950093F76B
:10F70000F707A384F50097000000E78020F917337E
:10F71000FFFF6700039F1733FFFFE702A39A83C72A
:10F7200095000329C501411193F7F707A384F5005C
:10F730001C4283C90700854763E637079777FF1F99
:10F74000938787C79C432E84AA8485CF97000000A7
:10F75000E78080F389476306F50263040902834763
:10F76000C900638037032306390197900000E780C2
:10F7700040ED83572903898B89C797D00000E78024
:10F78000E0B72685A28597000000E78020F1A167F9
:10F79000CD0748003EC42302010002C697E0FFFFE8
:10F7A000E78060AA41011733FFFF6700E394976782
:10F7B000FF1F938727699C431D4599C303C5E70035
:10F7C00082801733FFFFE70283910111B70707001B
:10F7D0003EC683C79500584D0AC493F7F7070AC879
:10F7E000A384F5002A89AE8415C71C4283C707008D
:10F7F00093968701E18663C4060685466381D70632
:10F800008346E7006388F6002307F700979000001F
:10F81000E78020E321649305E400280097B0FFFF10
:10F82000E78060D397000000E780A0F8AA85280051
:10F8300097D0FFFFE78080BA014781463000A68558
:10F840004A8597B0FFFFE78060F63504480822CC70
:10F85000230A010002CE97E0FFFFE780C09E05610A
:10F860001733FFFF6700E3891733FFFFE7022387A2
:10F8700001117C003ECAB70707003ECC7C003ECE9B
:10F8800083C795002E84AA8493F7F707A384F50015
:10F89000A165B905480897B0FFFFE780C0CB970086
:10F8A0000000E78000F1AA85480897D0FFFFE780B5
:10F8B000E0B2500801478146A285268597B0FFFF38
:10F8C000E780C0EE05611733FFFF670083831723CE
:10F8D000FFFFE702237FAA8401441769FF1F130972
:10F8E000A956E14997C0FFFFE78060C66344A400C2
:10F8F000014519A833053403832709003E95835732
:10F9000025006397970011051723FFFF6700C37E4B
:10F910000504C9BF032E8500630A0E121763FF1F7B
:10F92000130343710323030063150300294363900A
:10F93000061203234E01631503001D43639907104C
:10F940001723FFFFE7022377C689428A3E89BA8AD6
:10F95000B684328BAE8B2A84B5E103554E0019E58F
:10F9600001431A851723FFFF67006378A167A98FFA
:10F97000116763FBE70097000000E78080F5814591
:10F9800097F0FFFFE78080130844B70700E0584175
:10F99000F98F18455CC1B707001FF98F1CC55C497A
:10F9A00091C7610597E00000E780408BE38A09FA80
:10F9B000228597900000E78060C65DB7328597C0CA
:10F9C0000000E78040430D4349DD1C44116703D527
:10F9D0004700A167A98F63FBE70097000000E7805D
:10F9E00040EF814597F0FFFFE780400D032384003F
:10F9F00093164B01D1828347B30003566300858879
:10FA0000FD8BA305F300FD777D8E558EFD76FD16EB
:10FA1000B204F18E83274301C58E23127301231391
:10FA2000D3002304530123052301A3044301BDDFB5
:10FA3000228597B0FFFFE78040CAAA850844B5D168
:10FA4000610597D00000E780207F8DB71D431A85A0
:10FA500082801723FFFFE702E3660569AA84AE8967
:10FA6000328A0144FD5A7D1997C0FFFFE780E0A26A
:10FA70006347A40001451723FFFF6700E367D844ED
:10FA800093171400BA9703D70700631F3703239017
:10FA9000570163070A00268597900000E780A08041
:10FAA0009C449DC383D76700B3F72701639E37014A
:10FAB000D288014881470147814601468145268514
:10FAC00097000000E78040E5050479BF1723FFFF9A
:10FAD000E702435F79711C103EC4B7070F003EC6B2
:10FAE0001C103EC883C79500AA8A328593F7F70792
:10FAF000A384F5002E89328497D0FFFFE780C09D54
:10FB000093170501C187635AF006AA89228597D009
:10FB1000FFFFE780609C2A8A4E85032B040097B084
:10FB2000FFFFE780209839ED835744008144054466
:10FB3000F11793B71700A303F10083457100DA872B
:10FB40002287D2864E86280097E0FFFFE780A058E4
:10FB5000014781463000CA85568597B0FFFFE78090
:10FB6000E0C4A1679387F70348083ECC230A8100CD
:10FB700026CE97D0FFFFE780006D45611723FFFF7A
:10FB800067008357A2851306710097E0FFFFE780A7
:10FB90002067AA84094455D1528597E0FFFFE7808A
:10FBA00020D50D4459D90546D285268597000000F9
:10FBB000E78060EA2A8451B71723FFFFE702235248
:10FBC000835507000346270041112A842E8532C63B
:10FBD0002EC497E0FFFFE780A0D101C93246A245BD
:10FBE000228597000000E78000E741011723FFFF0F
:10FBF000670023511723FFFFE702E34B83C79500FC
:10FC00004111AA8A93F7F707A384F5003285AE89DC
:10FC1000328497D0FFFFE780208C93170501C187BE
:10FC20006357F00AC1452A8A228597C0FFFFE78003
:10FC300040712A8D228597D0FFFFE780E0892A89CD
:10FC4000228597D0FFFFE7800087930705F893F799
:10FC5000F70F1307E007AA8B637BF706228597D07F
:10FC6000FFFFE78040852A8C228597D0FFFFE78041
:10FC70008084AA8C5285032B040097B0FFFFE78095
:10FC8000608239E983574400231101008144F11750
:10FC900093B71700A300F1000544034711008356F2
:10FCA0002100938784005685DA8822885286CE8583
:10FCB00097F0FFFFE780E0A7A167E90748003EC48F
:10FCC0002302810026C697D0FFFFE780C05741017D
:10FCD0001723FFFF6700A34113061100A28597E0D9
:10FCE000FFFFE780E051AA8409E5231101000944E0
:10FCF0006DB7930521006A8597F0FFFFE78060F1FB
:10FD00002A8441FD835521009356C90013164901E9
:10FD100085486688E2875E87858A518226859700B6
:10FD20000000E78060BF2A848DBF1723FFFFE70232
:10FD3000833883C7950041112A8B93F7F707A38473
:10FD4000F5003285AE89328497C0FFFFE780C07826
:10FD500093170501C1876352F00A2A8A228597C04A
:10FD6000FFFFE7806077AA8A228597C0FFFFE780C0
:10FD7000A0762A89228597C0FFFFE780C07393078A
:10FD800005F893F7F70F1307E0072A8C6377F70658
:10FD9000228597C0FFFFE7800072AA8C228597C05A
:10FDA000FFFFE78040712A8D5285832B040097A0C6
:10FDB000FFFFE780206F39E5835744008544014405
:10FDC000F11793B71700A301F10003473100930720
:10FDD00084005A85DE882688D6865286CE8597F09E
:10FDE000FFFFE78000958D4748003EC42302910045
:10FDF00022C697D0FFFFE780004541011723FFFF90
:10FE00006700E32EA2851306310097E0FFFFE7802D
:10FE1000203F2A84894455D99356C90013164901B5
:10FE200085486A88E6876287858A5182D6859700E9
:10FE30000000E78060AEAA8449BF1723FFFFE702F6
:10FE400063282A8981440144617A916A176BFF1FF4
:10FE5000130B4B1E97B0FFFFE780206563C7A4001C
:10FE600022851723FFFF6700232983270900939921
:10FE70001400CE9703D5070033074501420741839D
:10FE80006364570305C103270B0019C785453E85E9
:10FE900097400000E78060E9832709000504CE97BA
:10FEA0002390070085047DB797000000E78060A2DB
:10FEB000832709000504CE972390070065D5814567
:10FEC00097F0FFFFE78080BFF1BF1723FFFFE70236
:10FED000631F83C7950041112A8A93F7F707A3840C
:10FEE000F50032852E89328497C0FFFFE780C05E1F
:10FEF00093170501C187635AF004AA89832A040075
:10FF000097A0FFFFE780005A31E5835744008544FE
:10FF10000144F11793B71700A301F1000348310022
:10FF2000D68752850147CE862686CA8597D0FFFFA1
:10FF3000E780406BA167F50748003EC423029100AB
:10FF400022C697D0FFFFE780003041011723FFFF53
:10FF50006700831AA2851306310097E0FFFFE78050
:10FF6000202A2A8489445DD99767FF1F9387870CCD
:10FF70009C4381CF044997B0FFFFE7800053AA85D7
:10FF8000268597400000E78040DA130504019700BA
:10FF90000000E780C0EA228597800000E7800033F8
:10FFA0008144ADBF1723FFFFE702E31083C795002D
:10FFB0004111AA8A93F7F707A384F5003285AE8929
:10FFC00032842311010097C0FFFFE780E0509317B0
:10FFD0000501C1876354F0062A8AC145228597C06E
:10FFE000FFFFE7800036AA8B5285032B040097A001
:10FFF000FFFFE780204B21E98357440085440144FB
:020000040001F9
:10000000F11793B71700A300F1000348110003573D
:100010002100DA875685D2862686CE8597D0FFFFC7
:10002000E780405CA1679387270248003EC4230213
:10003000910022C697D0FFFFE780E02041011723FF
:10004000FFFF6700C30AA2851306110097E0FFFFB8
:10005000E780001B2A8489444DD99767FF1F938747
:1000600067FD98433E8901CF044997B0FFFFE780C1
:10007000C043AA85268597400000E78000CB130582
:10008000040197000000E78080DB97B0FFFFE78066
:10009000C04195443DD9930521005E8597F0FFFF4F
:1000A000E78020B7AA8435F11C4803572100228538
:1000B0002390E70097800000E78040218327090014
:1000C000A9D70355210097400000E780A0BD35BFA8
:1000D0001723FFFFE70223FE83C795004111AA8A79
:1000E00093F7F707A384F5003285AE89328497C071
:1000F000FFFFE780603E93170501C1876351F0065B
:100100002A8A228597C0FFFFE780003D2A89528511
:10011000032B040097A0FFFFE780C03831E5835729
:10012000440085440144F11793B71700A301F1007F
:1001300003483100DA8756854A87D2862686CE85DF
:1001400097D0FFFFE780004AA167F90748003EC447
:100150002302910022C697D0FFFFE780C00E410125
:100160001723FFFF6700A3F8A2851306310097E06D
:10017000FFFFE780E0082A8489445DD99167CA9728
:10018000C2071167C1831307F7EF8544E362F7FAEB
:100190009767FF1F938707EA9843BE8B01CF0449F7
:1001A00097B0FFFFE7806030AA8526859740000062
:1001B000E780A0B71305040197000000E78020C87E
:1001C00097B0FFFFE780602E95443DD11C48228503
:1001D00081442390270197800000E780200F83A7A8
:1001E0000B00B9D74A8597400000E780A0AB89B7DC
:1001F0001723FFFFE702A3EE2A844105B28497008C
:100200000000E780C0C311C5228597800000E78009
:10021000E00B81460146A685228597800000E78095
:10022000C04E1C4C89C7DC4799C32285829717238F
:10023000FFFF670003ED9767FF1F9387A7C09C43ED
:10024000014599C31385070182809767FF1F938734
:1002500067BF884382801723FFFFE70243E89317B5
:10026000C600DD8DC2054111C1812A8432C697C006
:10027000FFFFE780A0183246228511829375F60FA2
:1002800097C0FFFFE780801541011723FFFF67003C
:1002900043E71723FFFFE702E3E279713C083ED210
:1002A000B7070C003ED43C083ED683C79500AE8409
:1002B0002A8993F7F707A384F500A1659385350490
:1002C000481097A0FFFFE7800029C165FD15014494
:1002D000176AFF1F130A8AD7930A400EAE892E8B26
:1002E0002EC697B0FFFFE780401F42059317040119
:1002F0004181C183B24563E9A702C167FD176387E6
:10030000F500481097C0FFFFE780400F50100147ED
:100310008146A6854A8597A0FFFFE7802049456171
:100320001723FFFF670043DD3307540383270A0BBE
:10033000BA9703D6C701630A3601638A35014810AC
:1003400097000000E78060F1DA85050451BFB285AF
:10035000EDBF1723FFFFE70203D679717C083EC883
:10036000B70711003ECA7C083ECC83C79500AA8916
:10037000328593F7F707A384F5002E8997C0FFFF16
:10038000E780801585676378F504A165AA848905EF
:10039000080897A0FFFFE780001C26859740000013
:1003A000E78060ED133415000A04A285080897C0A1
:1003B000FFFFE780A002A685080897C0FFFFE7803F
:1003C000E00325CC014781461008CA854E8597A0D9
:1003D000FFFFE780A03D45611723FFFF670023D1A2
:1003E000B30754030327CA0ABA9703D70700631C4D
:1003F000970003D627006380650508089700000072
:10040000E780A0E5DE8505042EC697B0FFFFE780F4
:10041000C00D4205931704014181C183B245E3E158
:10042000A7FCC167FD17E38FF5F8080897C0FFFF29
:10043000E780C0FC41BFB285F9B7C165FD15014435
:10044000176AFF1F130A8AC0930A80022E8BAE8B95
:1004500065BF1723FFFFE70283C8184183471700D2
:1004600083460700A207D58FD207D1832390F500DA
:1004700083472700034717008D45A207D98F918333
:100480002310F60097C0FFFFE78060EA1723FFFF05
:10049000670023C71723FFFFE702C3C2C1640144FB
:1004A0001769FF1F130989BA93098002FD1497B0D9
:1004B000FFFFE78080036347A40001451723FFFF88
:1004C000670083C3330534038327C90A3E958357E6
:1004D0000500E38597FE0504D9BF1723FFFFE70258
:1004E00063BE2A8AAE89B284B68A97400000E7804C
:1004F00080D819E591473E851723FFFF6700C3BFEA
:100500002A894E8597C00000E780E08E2A84638E9A
:100510000A048D476DD103570500C547E31D47FD0C
:100520000347F9018546AD47E317D7FC83474500EC
:1005300081CF4146A6855D0597F00000E780C09E0B
:10054000814755D9AD4745BF130965012302E50031
:10055000CA85268597100000E780606231C1A547F3
:10056000E38B0AF82302040079B705C1835705001D
:10057000E39247F94146A685190597F00000E78008
:10058000A09A81472DD99947BDB74E8597000000A5
:10059000E78080F02A84954739DD130955004DBF67
:1005A0004146A68523104401231134011305190087
:1005B00097F00000E780A099228597800000E780EF
:1005C000A0EA81470DBF1723FFFFE70243B179710E
:1005D0007C003ECCB7070A003ECE7C003ED083C7ED
:1005E0009500B2842E8493F7F707A384F5001306D1
:1005F000A1002A892C00268597000000E780A0E54D
:10060000A16528088D0597A0FFFFE780C0F4904002
:100610008355A10003558100854697000000E780BF
:1006200000ECAA84AA85280897C0FFFFE78000DBBA
:100630000356A10083558100280897000000E78039
:10064000C0C1300801478146A2854A8597A0FFFFB7
:10065000E780C015854748103ED42302910202D698
:1006600097D0FFFFE78020BE45611723FFFF67009B
:1006700043A91723FFFFE70283A679717C003ECCD4
:10068000B7070A003ECE7C003ED083C79500B284F7
:100690002E8493F7F707A384F5001306A1002A8997
:1006A0002C00268597000000E780E0DAA165280885
:1006B0008D0597A0FFFFE78000EA90408355A100D9
:1006C00003558100814697000000E78040E1AA843D
:1006D000AA85280897C0FFFFE78040D00356A100F5
:1006E00083558100280897000000E78000B7300894
:1006F00001478146A2854A8597A0FFFFE780000B4E
:1007000048102302910202D402D697D0FFFFE7805F
:1007100080B345611723FFFF6700A39E1723FFFFE8
:10072000E702E39B97000000E78060DB1723FFFFF1
:100730006700239D9757FF1F938707718843828027
:100740001723FFFFE702A399835725004111AE84C9
:100750002A842307B10017F5FFFF130525466C0017
:100760002316F10097A0FFFFE780404691C4228541
:1007700097800000E780E0D6FD572310F4001306B1
:1007800020028145130554009720FFFFE780209841
:1007900041011723FFFF6700C3961723FFFFE702FE
:1007A000639279717C003ECCB7070A003ECE7C0094
:1007B0003ED083C79500AA89AE8493F7F7073285A8
:1007C000A384F5001306A1002C0097000000E78029
:1007D00080C803558100114497400000E780A0A91C
:1007E00015C50355A100014497B00000E780A06043
:1007F00011CD035705008357810045446318F70066
:10080000854597000000E780E0F3014421699305E6
:100810003900280897A0FFFFE780E0D3A2852808C9
:1008200097C0FFFFE78080BB0356A100835581007E
:10083000280897000000E78040A230080147814661
:10084000A6854E8597A0FFFFE78040F648104AD462
:100850002302810202D697D0FFFFE780C09E456148
:100860001723FFFF670043891723FFFFE7028385F4
:100870009757FF1F9387075D2A8488432E8915C5E4
:10088000035745038357C4016311F702232605026A
:1008900023180502410597D00000E780209C6306DD
:1008A000090097800000E78060DB81449759FF1FB3
:1008B0009389C979130A800297B0FFFFE780E0C2ED
:1008C00063C4A4049757FF1F938787609C4399C70D
:1008D0000355C40197200000E780C0BD63070900ED
:1008E000228597800000E780C0A01306400E814556
:1008F00022859720FFFFE7808081FD57231EF400AB
:100900001713FFFF6700437F3385440383A7C90A9A
:100910003E95035705008357C4016317F700CA8546
:1009200097000000E78000E2850479B71713FFFF06
:10093000E702437983C795004111AA8993F7F70726
:10094000A384F5003285AE8497C0FFFFE780C0B86E
:1009500085676378F5042A8997400000E780A091B5
:10096000014401CD83D704003144638827018545C4
:1009700097000000E78080EF01444E85A2864A86FA
:10098000A68597D0FFFFE780609DA1679387170436
:1009900048003EC42302810002C697D0FFFFE780D3
:1009A000808A41011713FFFF670003751713FFFFCC
:1009B000E70243719757FF1F9387C748804329C4B5
:1009C000014597C00000E780002181470148C164CC
:1009D0001CDC232E0403232004041759FF1F1309D2
:1009E000E96601449309400EFD1497B0FFFFE780CC
:1009F000C0AE634FA400814517F5FFFF1305857F47
:100A000097A0FFFFE780801C1713FFFF6700C36EEE
:100A1000330534038327090B3E958357C50163874C
:100A20009700854597000000E78040E4050475BF06
:100A30009357050113D78700A380F500931705018D
:100A4000C183A1832380E5002381F500A381A50054
:100A500082801713FFFFE70283682300050083C726
:100A60001500A300F50083C725002301F50083C707
:100A70003500A301F50083C745002302F50083C7B5
:100A80005500A302F50083C7650093059500A303F5
:100A900005002303F50023040500328597000000BC
:100AA000E78040F91713FFFF6700A3651713FFFFE7
:100AB000E70243614111E9540DCD85CD93F9C5FF9E
:100AC0002E842A89AA84338AA900B7EA040063180D
:100AD0009A020D88854411CCB7E704009C5F829789
:100AE0002AC622866C003305390197E00000E780B2
:100AF0000046268541011713FFFF6700E35F83A7C8
:100B00008A039104829793170501C183A183A38E61
:100B1000F4FE93570501238FF4FEA183238EA4FED8
:100B2000A38FF4FE6DB763E6D5021713FFFFE7024C
:100B3000035BB28741113686BE8536C697E000005A
:100B4000E780E040B246410136851713FFFF67009A
:100B5000435B814636858280838705001387F500D5
:100B60003D05FD8793F77708834607007D158606C8
:100B7000B58FA300F5006307B7007D178347170003
:100B80009D83DDB782801713FFFFE7024355B7E768
:100B9000040083A7070932872A863A85829713358E
:100BA00015001713FFFF6700C35515C181478DC19D
:100BB0001713FFFFE702A352414697E00000E780CA
:100BC000003985473E851713FFFF67008353814730
:100BD0003E8582801DCD1713FFFFE702435041463B
:100BE00081452A849710FFFFE78060524146814586
:100BF000130504039710FFFFE78060510147C167A9
:100C00002322040438C87CC805451713FFFF67007A
:100C1000434F0145828081473DCDB5CD1713FFFF7E
:100C2000E702E34BB2842E891306800581452A84AE
:100C30009710FFFFE780A04DCA8524C42685970042
:100C40000000E780C0F64146814522859710FFFFEE
:100C5000E780E04B3044A285228597000000E780C2
:100C6000C0F293040401A285268597000000E78066
:100C7000E0EEA6851305040297000000E78000EE71
:100C8000228597000000E78020F585473E851713F1
:100C9000FFFF670003473E8582801713FFFFE702CF
:100CA00063424111E9540DCD85CD93F9C5FF2E84E2
:100CB0002A89AA84338AA900B7EA04006398440306
:100CC0000D88814411CCB7E704009C5F82972AC647
:100CD00022866C003305390197E00000E780202769
:100CE000268541011713FFFF6700034183A78A038D
:100CF0009104829793170501C183A183A38EF4FE0B
:100D000093570501238FF4FEA183238EA4FEA38FA6
:100D1000F4FE6DB765CD1713FFFFE702A33AB28467
:100D200011E605451713FFFF6700033D2A842E894E
:100D30000145EDD93C487848B3E6E700E5D693860F
:100D4000F7FFB3B7F6007D17032A4404BA9734C8F7
:100D50007CC863050A06C14913050A03B3894941E2
:100D60002295637D3601B2862E86A6859700000007
:100D7000E780A0DB7C40BE9464C065B7CE862E863B
:100D8000CE8597000000E78040DAC114D2944E99D6
:100D900023220404A2879306040103C7070003C6A5
:100DA00007038507318FA38FE7FEE398F6FE3044F3
:100DB000A285228597000000E78020DD2699C149A1
:100DC0003306994063EC9900A9DCA686A685130535
:100DD000040397000000E78040D579BF8147B30640
:100DE000F4003307F6000347070083C506008507B4
:100DF0002D8F2380E600E39437FF3044A2852285BF
:100E000097000000E78060D8C1145DBF0145828073
:100E10000DC11713FFFFE702832C130680058145E0
:100E20009710FFFFE780A02E05451713FFFF67000F
:100E3000432D01458280814749C5C1C51713FFFF76
:100E4000E702E329FC4141462E84AA846399C70442
:100E500013860501A2878146C14503C7070003C564
:100E600007038507298F3305D6000345050085064E
:100E7000298FA38FE7FEE392B6FE3044A285268534
:100E800097000000E78060D0228597000000E7808F
:100E900060F885473E851713FFFF6700832613859B
:100EA00007031D8E814522959710FFFFE7802026BE
:100EB0007C40130700F813060402A2972388E70278
:100EC00051BF3E8582801713FFFFE70243216D71FA
:100ED0002E84B284AA8590102800368997000000DD
:100EE000E780A0D309EDD55725A050400C4028003D
:100EF00097000000E78040E27DD5FD142104F5F461
:100F00002C004A8597000000E78020F3814761DDCF
:100F10003E8551611713FFFF6700A31E1713FFFFE4
:100F2000E702E31B41112EC432C62C000546970090
:100F30000000E78080F941011713FFFF6700631C81
:100F40001713FFFFE702A31901112A842EC602C856
:100F500002CA02CC02CE97E00000E780C023B2466E
:100F60002A86A285080897000000E78060FB1375B9
:100F7000F50F05611713FFFF6700A3181713FFFF95
:100F8000E702E3157971B2872A8421462308B1006C
:100F900013051101BE853AC436C697E00000E7800C
:100FA00000FBB24693059101368597000000E7806B
:100FB00060A82285141035460C0897000000E780D1
:100FC00020F62A84224701E921460C103A8597E051
:100FD0000000E780C0F7228545611713FFFF670017
:100FE00043121713FFFFE702830F7171AE84AA85C6
:100FF0000A85328497000000E78060BB11C90A8629
:10100000A685228597000000E78020B8814711E17E
:10101000C5473E854D611713FFFF6700830E171309
:10102000FFFFE702C3081D712A8AB289BE843546D4
:101030008547130511012E8CB68A3A8BC28C468DDA
:101040002308F10097E00000E78060F010100C0822
:101050005285231F010097000000E780C0F82A8412
:101060003DEDA1476313FD089307900591E0E54727
:101070003546E2851305110113990A012308F10091
:101080001359090197E00000E78060EC13578900CD
:1010900093978A00D98F90080C085285231FF1007E
:1010A00097000000E78020F42A8415E9A1E49387E3
:1010B000FA0091831379F9003EC663130900414990
:1010C000668B8144C14B854DB247639F970C6A86FE
:1010D0008C0033855C0197E00000E78040E72285C3
:1010E00025611713FFFF6700430093079004C9F0C1
:1010F000A547BDBF834701050947C14B2308F10040
:1011000083471105A58FA308F1009387240081442C
:1011100063E1FB04014714083386E6008C08B386BC
:10112000E400BA95DA9683C6060083C50500050774
:10113000AD8E2300D600E390E7FE4147639CE704B1
:1011400090080C08528597000000E780C0E925D17F
:1011500081A0B3069B00BA871008B305F60090087B
:101160003E9603C506000346060085078506298EC0
:101170002380C500E39277FF998F90080C08528571
:10118000BE9497000000E78000E68947014749D1F7
:101190002A84B1B790083E96034606001408BE960E
:1011A0002380C600850759BFB2478504638797141B
:1011B00081471808B306F70098083E973386F90070
:1011C00003470700034606008507318F2380E600AA
:1011D000E39177FF90080C08528597000000E780A4
:1011E00080E05DF53546E285130511012308B10164
:1011F00097E00000E780A0D51397040141839397FF
:1012000084002183D98F10180C085285231FF10008
:1012100097000000E78020DD25FD81471018338707
:10122000F9003E960347070003460600B306FB009D
:101230008507318F2380E600E39277FF65A81808C1
:10124000B306F70098083E973386F9000347070076
:10125000034606008507318F2380E600E3E127FF80
:10126000CA87639E770990080C0852859700000092
:10127000E78060D711FD81479800B306F70090081A
:1012800018103E973E960347070003460600850761
:10129000318F2380E600E39177FF3546E285130521
:1012A00011012308B10197E00000E78040CA1397BD
:1012B00004014183939784002183D98F10180C086F
:1012C0005285231FF10097000000E780C0D1E31191
:1012D00005EC814710183387F9003E960347070055
:1012E00003460600B306FB008507318F2380E60026
:1012F000E3E227FFC109410BC1BB814785B79408D1
:10130000BE9683C6060018083E972300D7008507BF
:1013100089BF638006321713FFFFE70243D9597173
:101320002A84BE89B28B85473546130511022E8B60
:10133000468C4289BA8A368A2300F10297E000007F
:10134000E780E0C010180C102285231701029700D7
:101350000000E78040C963180512A147631FFC061F
:101360009307900563930900E5473546DA85130531
:10137000110293140A012300F102C18097E00000DA
:10138000E780E0BC93178A0013D78400D98F9008B8
:101390000C1022852317F10297000000E780A0C4FB
:1013A0007DE1639209049307FA00BD88918391E07F
:1013B000C144C207C183DE8C814A3EC6414DB2475B
:1013C00063E2FA0E6286B3854B01881097E0000055
:1013D000E78080B54DC93D557DA093079004E39605
:1013E00009F8A54759B7834701050947C14C2300B0
:1013F000F10283471105B3C7F900A300F1029387F7
:101400002900814963E1FC04814618103306D700A6
:101410008C083387D900B69556970347070083C5D4
:10142000050085062D8F2300E600E390D7FE414797
:101430006390E70690080C10228597000000E78073
:1014400080BA35D189A0B3863A01BA871010B305A6
:10145000F60090083E9603C5060003460600850781
:101460008506298E2380C500E39297FF3387EC40E1
:1014700090080C102285BA9997000000E780A0B66A
:101480008947014741D165611713FFFF6700E3C535
:1014900090083E96034606001410BE962380C600B0
:1014A000850779B7B247850A93990A01939D8A0007
:1014B00093D909016391570F85473546DA8513059E
:1014C00011022300F10293D9890097E00000E78020
:1014D00000A8B3ED3D0190000C1022852317B10345
:1014E00097000000E78020B059FD8147A68963EA94
:1014F000970626860C084A8597E00000E78020A51D
:1015000081471810B306F700100898083E973E96DA
:1015100003470700034606008507318F2380E60056
:10152000E3E197FE639FA90590080C1022859700C0
:101530000000E78040AB21F981479810B306F7001F
:10154000900818183E973E9603470700034606008A
:101550008507318F2380E600E391A7FF4109C10C85
:10156000B9BD18089000B306F7003E963387FC001B
:1015700003470700034606008507318F2380E600F6
:10158000B5B798084E97034707001C10CE972380E5
:10159000E700850941BF85473546DA851305110205
:1015A0002300F10293D9890097E00000E780209A98
:1015B000B3ED3D0190000C1022852317B103970075
:1015C0000000E78040A2E31005EC81471808900076
:1015D000B306F7003E963387FC0003470700034637
:1015E00006008507318F2380E600E391A7FF41467F
:1015F0000C084A8597E00000E78060958147181045
:10160000B306F700100898083E973E960347070078
:10161000034606008507318F2380E600E391A7FF8C
:1016200090080C10228597000000E780C09B1DD514
:1016300099BD7D5582801713FFFFE70243AA011170
:101640002A842E8593055100328902C002C202C449
:1016500002C69304740097F0FFFFE780A03D1D468B
:10166000A6851305910097E00000E780408E1008E2
:101670008A854A8597000000E780E09619ED930778
:101680001400180883C607000346070085070507EE
:10169000B18EA38FD7FEE397F4FE05611713FFFF0A
:1016A000670023A61713FFFFE702C3A12E848C4116
:1016B0004111AA89838715003289914463D30700B9
:1016C000A1449757FF1F938727CF9C43A1C7C1CA47
:1016D0008D472310F10083C725004A852301F100BF
:1016E00083C73500A301F10083C745002302F10041
:1016F00083C75500A302F10083C7650093059100DD
:10170000A30301002303F1002304010097F0FFFF6E
:10171000E78040320C404A860A8597F0FFFFE78059
:1017200080330328040083564400A6881D0881479F
:101730000147E51642868A854E8597000000E780BE
:10174000408E2A8919E5A685228597B0FFFFE7809C
:10175000A0C24A8541011713FFFF6700E3994A863B
:101760000A8597F0FFFFE780002F6DB71713FFFF83
:10177000E70243952E848C414111AA898387150085
:101780003289914463D30700A1449757FF1F938781
:10179000A7C29C43A1C7C1C68D472310F10083C7D0
:1017A00025004A852301F10083C73500A301F1001C
:1017B00083C745002302F10083C75500A302F1004F
:1017C00083C7650093059100A30301002303F10083
:1017D0002304010097F0FFFFE780C0250C404A86F4
:1017E0000A8597F0FFFFE78000278356440003280F
:1017F00004008A85858EC2061D08C1822312D4008A
:10180000A68881470147E51642864E85970000006D
:10181000E78060B041011713FFFF6700E38D4A8640
:101820000A8597F0FFFFE78000234DBF1713FFFFE6
:10183000E702E38AB335B000011185052A89131543
:10184000F601336515012308B100930511013684B3
:101850003AC632C03EC442C297F0FFFFE780801D07
:10186000A2471248425593D68700230BF1009305F7
:10187000910193578800A30AD100A30BF100230C18
:10188000010197F0FFFFE780E01A32470246032884
:101890000400B337E000835644009207914411C21C
:1018A000A1444A85A68842860C0897F0FFFFE7808E
:1018B00040772A8919E5A685228597B0FFFFE78042
:1018C000A0AB4A8505611713FFFF670083831703E9
:1018D000FFFFE702237F01113EC68647B335B00004
:1018E0008505AA891315F6015D8D2308B1009305BE
:1018F000110136843A89B28442C446C297F0FFFF90
:10190000E780401322489248164593578800A30A5F
:10191000F1009305910193D78800230B0101A30BDC
:10192000F100230C110197F0FFFFE780A010324770
:10193000104083564400B337E000920703280900A3
:10194000914891C0A1480C084E8597000000E7809F
:10195000809CAA8401E9835544004A8597B0FFFF23
:10196000E78080A1268505611703FFFF6700C37824
:10197000AA959307F00F170701001307A75D6317D8
:10198000B50013C5F7FF1375F50F82800505834673
:10199000F5FFB58FBA9783C70700D5B70357450042
:1019A00014419307F00F170601001306A65A369745
:1019B00042074183139506014181631BE500AD8F0A
:1019C000B29703C50700130515F313351500828080
:1019D000850603C5F6FFA98FB29783C70700D9BF55
:1019E0001703FFFFE702A36FB28736842E86BA86FD
:1019F000AA853E85BA8497F0FFFFE7806052634F67
:101A00000500228597D00000E780E0782A86A68628
:101A1000A285268597F0FFFFE78080501703FFFF20
:101A20006700236E1703FFFFE702C3695D712A8B0E
:101A3000AE8A170501001305654F2C00B284368A63
:101A4000BA893E8997F0FFFFE780C04F2A845DE1A5
:101A500034104146DA85280097F0FFFFE780404CBC
:101A60002A8449E98547A303F100A6C293077100C0
:101A70002408BEC4A68685470D462C18281002DC13
:101A800002DED6C0BEC697F0FFFFE78000442A847E
:101A900035E183477102A6860D4693F7F7072300C9
:101AA000FA00C1473EDE2C188947281026DCA30324
:101AB000F10097F0FFFFE78040412A8405ED4146A1
:101AC000A6854E8597D00000E78060488D47A686A2
:101AD0000D462C182810A303F10097F0FFFFE780B4
:101AE000C03E2A8401E94146A6854A8597D0000078
:101AF000E780E045228561611703FFFF6700C35F50
:101B00001703FFFFE702A35D97F70000938787A104
:101B1000984383C7470079712A89AE84170501006D
:101B2000130545410C083AC42306F10097F0FFFF66
:101B3000E78040412A8405ED14104146CA85080813
:101B400097F0FFFFE780C03D2A8415E11408154691
:101B50002C00081097F0FFFFE780803C2A8401E901
:101B600021462C08268597D00000E780403E22853C
:101B700045611703FFFF6700C3581703FFFFE70224
:101B8000035697F700009387E7999C477971AA84D9
:101B90002E84170501001305653A0C083EC697F020
:101BA000FFFFE780203A0DE914104146A68508089A
:101BB00097F0FFFFE780C03605E1140811466C007E
:101BC000081097F0FFFFE780A03519E58347F10182
:101BD00093F7F7032300F40045611703FFFF670045
:101BE00043521703FFFFE702834F3688A14881471E
:101BF0000147E54697F0FFFFE780A0421703FFFF8C
:101C0000670023501703FFFFE702634D3688A148A2
:101C100081470147E54697F0FFFFE780C06F170354
:101C2000FFFF6700034E1703FFFFE702434B01115D
:101C30002A842E850C0832C697F0FFFFE78080309B
:101C400009ED3247970601009386C62D1008C1455D
:101C5000228597000000E780E0D805611703FFFFA9
:101C60006700234A1703FFFFE70263474111C1479B
:101C70002EC032C48A8509463EC23EC697F0FFFF99
:101C8000E780A02441011703FFFF67008347170384
:101C9000FFFFE702C3444111AE8613061009AA856F
:101CA0000A8502C002C202C402C697F0FFFFE780A5
:101CB000202741011703FFFF6700A3441703FFFF1D
:101CC000E702E3413287970601009386A6272E8616
:101CD0009305000297000000E780C0D01703FFFFC4
:101CE000670023421703FFFFE702633F7971C14793
:101CF0002ACC2ED032D42C080D4628003ECE3ED21F
:101D00003ED602C402C602C802CA97F0FFFFE780AF
:101D1000C01B45611703FFFF6700A33E1703FFFFCA
:101D2000E702E33B0111AA842E8417050100130585
:101D3000E5218A8597F0FFFFE780C02015E51408AC
:101D40004146A6850A8597F0FFFFE780601D09EDF3
:101D50008347E1010347F101A207D98FCA07C9836D
:101D60006177D98F2310F40005611703FFFF670027
:101D7000433915CD1703FFFFE70263369747FF1F6F
:101D80009387071190439745FF1F9385A51017452B
:101D9000FF1F1305E50B97D00000E78000C517452E
:101DA000FF1F1305E50A1703FFFF6700833517457B
:101DB000FF1F1305E50982808DCD1703FFFFE702A2
:101DC00003329747FF1F9387A70C944301112E847A
:101DD0000A869745FF1F9385E50B97D00000E780A3
:101DE00040C60A850294014505611703FFFF67009D
:101DF00043317D5582801703FFFFE702432E97D0C2
:101E00000000E78080D19747FF1F23A3A70817F59D
:101E1000FFFF1305E5C997B00000E780C074170302
:101E2000FFFF6700032E1747FF1F1307A70893172D
:101E3000150008433E95FD572310F50082801703D7
:101E4000FFFFE702C3292A84084009E51703FFFFC3
:101E50006700232B1C4158401CC06313E5005CC085
:101E60008347550023200500F99BA302F50097A0A6
:101E7000FFFFE780E07CC9BF1703FFFFE702832471
:101E80009747FF1F9387070598432A8411CB834701
:101E9000350093F7070289C7035505008945029766
:101EA0001305440197B00000E780403B83550400D0
:101EB0000355E40097300000E780A00C485819C58E
:101EC00097A0FFFFE780C077232A0402130584034D
:101ED00097000000E780E0F68144B1499790FFFF4A
:101EE000E780E06A63CBA402834734002320040424
:101EF00093F727FCA301F40000489790FFFFE780C9
:101F0000006A13161500814522859700FFFFE780C0
:101F100000201703FFFF6700231EB3873403032944
:101F2000040385043E994A8597000000E78060F12C
:101F30002304090065B78347350093F7070299E347
:101F4000014582808357E500E39CB7FEC167FD171A
:101F50006316F60005458280054599A81703FFFF23
:101F6000E702E31793170601C187B2842A84014967
:101F70006359F002835705009DCB01456367F60066
:101F8000034584003E953325A6001375F50F0DA07B
:101F90001C4813171900BA9783D70700E38E97FAE6
:101FA00005099790FFFFE780805FE343A9FE0145A5
:101FB0001703FFFF6700E3141703FFFFE702831017
:101FC000AE89AA849790FFFFE78020532A8497D098
:101FD000FFFFE780A02EAA8601471306840197051C
:101FE0000000938585E41745FF1F1305E5EC9790E6
:101FF000FFFFE780A0192A8925C98C441304C50076
:1020000022859E0593F5050897A0FFFFE780003D18
:10201000CC4083877400E18163DD070493E5050804
:10202000228597A0FFFFE780603B0D469385440023
:10203000228597A0FFFFE780803783D504002285A3
:1020400097A0FFFFE780A03E83D52400228597A0BC
:10205000FFFFE780C03D03D6490083A50900228524
:1020600097A0FFFFE780A0344A851703FFFF6700B2
:10207000A30893F5F5076DB71703FFFFE7022306E3
:1020800001112A84328532C697A0FFFFE780A0287D
:102090009780FFFFE7808031835704001747FF1FB9
:1020A0001307C7FA3246231BF100930700F8A30D6C
:1020B000F1001C471843231AA1008983858BB307BD
:1020C000F740B28548083ECE231C0100230D0100D5
:1020D00097000000E78080EE05611703FFFF6700AF
:1020E00043021703FFFFE702E3FD004101453DC442
:1020F0009304C40026853289AE8997A0FFFFE7804C
:10210000802595452A8A2685035B040197A0FFFF59
:10211000E780E021268597A0FFFFE780203F8D45DF
:10212000AA8A268597A0FFFFE7806020268597A0D2
:10213000FFFFE780A03D5C48420A135A0A01D2978C
:102140005CC423186401814763983A0146054D81B8
:10215000330625419337160013F5F70F1703FFFFDA
:10216000670083F91703FFFFE702E3F489692A8B0D
:10217000AE8B328AB68A81440144314CFD19979066
:10218000FFFFE780C04063CDA4009790FFFFE7808A
:102190000043018D33B5AA001703FFFF670023F545
:1021A0003389840383270B003E9963170A00834712
:1021B000890085043E94E1B703560A00DE854A850E
:1021C00033F6C90097000000E780E0F16DD10545C6
:1021D000E1B71703FFFFE70283F001112A847C00B7
:1021E0000355E5003ECAB70707003ECC7C003ECE53
:1021F00097200000E78020082A898545480897A095
:10220000FFFFE780E0399945480897A0FFFFE78086
:10221000A016AA844A8597200000E780A0082380A2
:10222000A4009747FF1F938767E29C43416613060C
:1022300006F09396870113D78701558F93D68700B1
:10224000F18E558FA207B706FF00F58FD98F114683
:102250002C00138514003EC497D00000E78020CFE7
:102260005008A38204008945228597000000E7807A
:10227000E0E019C9AA851305840397A0FFFFE78052
:10228000A0323C4085073CC005611703FFFF670093
:1022900043E71703FFFFE70283E49790FFFFE78020
:1022A00000322A8405049790FFFFE7804030330511
:1022B000A402F14791453305F50297200000E7801D
:1022C00020BA11E565551703FFFF670083E39747C1
:1022D000FF1F23A9A7BE9790FFFFE780402E2A8407
:1022E00005049790FFFFE780802C3305A402894501
:1022F000060597200000E780A0B669D59747FF1F25
:1023000023AAA7BA9790FFFFE780602B2A840504D1
:102310009790FFFFE780A0293304A4029747FF1F8F
:10232000239C87B89790FFFFE78060292A849790C5
:10233000FFFFE780C027930714003385A702974764
:10234000FF1F239CA7B6970701009387E7831747D2
:10235000FF1F2327F7B60145BDB71703FFFFE702AD
:1023600063D6AA842E8901449749FF1F938909CE19
:10237000130A80069790FFFFE78060236347A4005D
:1023800001451703FFFF670023D73305440383A7E5
:1023900009024A86A6853E9597000000E780E0B9CD
:1023A00019E10504C1BF0545E9BF1703FFFFE702B7
:1023B00083D0AA8A2E8BB28B368C3A8A8144014410
:1023C0008149974CFF1F938C6CC8130D8006979022
:1023D000FFFFE780C01D63C9A40011E085494E8559
:1023E0001703FFFF6700A3D03389A40383A70C0260
:1023F0005E86D6853E994A8597000000E780E0B367
:102400001DC19790FFFFE780801B0544636D450168
:10241000D2866286DA851305090397000000E780FB
:10242000A0D411C1854985045DB71703FFFFE702FA
:1024300063C9C16441112A8901449749FF1F9389E7
:10244000E9C0130A8006FD1436C632C42EC2979026
:10245000FFFFE780C01592452246B2466348A400BC
:10246000014541011703FFFF670003C9330544031A
:1024700083A709023E9509C683473500C18B9DC7D6
:1024800091C68347350093F707028DC36306990011
:102490008357E500639C27010357050001CB63E7E1
:1024A000E50083478500BA97E3CDF5FA050469BFD7
:1024B0001703FFFFE70203C1C1642A89014497495A
:1024C000FF1F9389A9B8130A8006FD149790FFFF98
:1024D000E780E00D6346A4001703FFFF6700C3C158
:1024E0003305440383A709023E958357E500638AB9
:1024F0009700630499006396270197000000E78026
:10250000E0970504E1B71703FFFFE70243BA8969C3
:102510002A8AAE8A328BB68B8144174CFF1F130C6C
:10252000ECB2930C8006314DFD199790FFFFE780C8
:10253000000863C6A4001703FFFF670003BB3389CD
:10254000940383270C028355CA015A863E994A8513
:1025500097000000E780609E31C1814D15A0338453
:10256000AD038327090303D60B00D68533F6C900D4
:102570003E94228597000000E780E0B609E9850DCA
:102580009790FFFFE780A000E3CBADFC01A8228578
:1025900097000000E780E08A23040400850471B7F7
:1025A0001703FFFFE70223B14169AA8A014A174BCB
:1025B000FF1F130BABA97D19C14B054C9790FFFF73
:1025C000E780E0FE6346AA001703FFFF670023B21F
:1025D00093098006B3073A0383290B02BE9983D778
:1025E000E900638E270163842A01639A570103A4DB
:1025F000890301E84E8597000000E780C0BD050A09
:1026000075BF83570401639977099304C400268535
:1026100097A0FFFFE78020D485452A8D2685835C1F
:10262000040197A0FFFFE78080D0268597A0FFFFD9
:10263000E78060E862056185635905048D4526855C
:1026400097A0FFFFE780A0CE8945268597A0FFFFD2
:10265000E780E0CD8945268597A0FFFFE78020CD64
:102660008545268597A0FFFFE780A0CD834705001D
:10267000094793F7F707639AE7009945268597A0DE
:10268000FFFFE78000CCA30285014848337D2D0180
:10269000231894016A9548C40040A1BF1703FFFFA7
:1026A000E702E3A337E404008327041D82979747DA
:1026B000FF1F83C7A7861715FF1F130525E7A30074
:1026C000F5008327441C82978327841C81461306C8
:1026D000F00F8145014582971703FFFF670063A252
:1026E0001737FF1F1307877318439745FF1F83C5CD
:1026F000E5829747FF1F9387E7808346870303465A
:1027000097036397D5009747FF1F2389C78082806F
:1027100083C587010347A7036317B6009737FF1FD9
:10272000238EE77E828003C687016317C700973731
:10273000FF1F2385D77E828083C68701130750023F
:102740006319D700930760021737FF1F2308F77C30
:10275000828083C68701130660026315D600930743
:102760007002DDB783C7870155BF9737FF1F938777
:102770006779D44B0947638DE6081703FFFFE7022B
:1027800003961739FF1F130929753E8483470900F3
:10279000918B9DCFB7E4040083A7041D829783A784
:1027A000441C1735FF1F1305A573829783A7841C4C
:1027B00081461736FF1F0346A6748145014582975F
:1027C00021C583470900ED9B1737FF1F2306F770CC
:1027D0008347040093F7F70F85CB91471737FF1F07
:1027E000232CF77297000000E78080EB9700000031
:1027F000E78040EFB7E70400BC4F414691451735ED
:10280000FF1F0345A57082971703FFFF6700638FC3
:1028100082801703FFFFE702838C8D474111630617
:10282000F504C5476308F50285476310F50297373D
:10283000FF1F2387A76EB7E70400BC4B930500106A
:102840001735FF1F0345856C829741011703FFFF72
:102850006700238B85471737FF1F2303F76CB7E704
:102860000400BC4B93050020E1BF9737FF1F9387FF
:102870006769D44B1147638DE600B7E7040083A76F
:10288000071D8297B7E70400BC4B930500044DBFBA
:1028900005491737FF1F2321276983C7070032C661
:1028A0002E8493F7F70FD5D3B7E4040083A7041D54
:1028B0007D141374F40F8297E37689FCB24599472F
:1028C00003C61500E3F0C7FCFC4409061735FF1FDB
:1028D000130545658297BC48930500081735FF1F0F
:1028E0000345C562829779BF17F3FEFFE702237F96
:1028F0001737FF1F130707614047184B1C409736D7
:10290000FF1F23A7F6606316E4001737FF1F23237A
:10291000F760130584FE9790FFFFE78020A703551B
:1029200064FF9780FFFFE780A06F97A0FFFFE7801D
:1029300020D117F3FEFF6700C37C17F3FEFFE70209
:10294000037A9737FF1F9387E75BD84BDC4789C72C
:1029500097000000E78080F985471737FF1F232D78
:10296000F75A9737FF1F9387674B9C4393050002E5
:102970001735FF1F0345855983C787031737FF1F87
:10298000230EF758B7E70400BC4B829717F3FEFFFE
:10299000670023779737FF1F23A8A756828017F376
:1029A000FEFFE702237237E404007C4CA145173593
:1029B000FF1F0345A55582977C48A1451735FF1F8A
:1029C0000345C5549734FF1F9384C4538297DC4456
:1029D00089EB97000000E78080D917F3FEFF6700BE
:1029E000A37103D567FF9780FFFFE7806063AA8923
:1029F0006DD1D84891476310F7027C4C914517354B
:102A0000FF1F0345A55082977C4891451735FF1F4E
:102A10000345C54F829703A9490103D4090189479A
:102A2000B7E904001737FF1F2328F74E83A7091DB6
:102A300021044204829783C784011715FF1F1305E1
:102A4000E5AE61191717FF1FA302F7AE83A7491C54
:102A5000418082979737FF1F2384074C83A7C91CA7
:102A6000814609469375F40F4A85829711E9973795
:102A7000FF1F83C7275B89C79700FF1FE780801769
:102A8000B7E70400BC4F2146A1451735FF1F03459A
:102A9000E547829799B717F3FEFFE702436493F780
:102AA000052001112E8481CF97000000E78020E9E6
:102AB00013450420056117F3FEFF6700836493F755
:102AC0000510A9CF9734FF1F9384C443DC489700B7
:102AD0000000E78020C11737FF1F13072734184372
:102AE00083C78401034787036318F700DC4489C761
:102AF00097000000E78080DF85471737FF1F232DF1
:102B0000F740B7E70400BC4B930500021735FF1FE1
:102B10000345C53F82971345041069BF93F7050825
:102B2000BDC79737FF1F83C7F73FE917194697358A
:102B3000FF1F9385453F1305D10093F4F70F173915
:102B4000FF1F0349293E97C00000E780404093974C
:102B50000401C1831737FF1F1307473D231DF100F1
:102B6000231CF1009737FF1F9387C7393ACE3ACA23
:102B7000D8432306010009CBDC439315890154088F
:102B80000D46E185680082971345040825B793F741
:102B90002500A5C39737FF1F9387C736D84B8947B2
:102BA0006306F7029737FF1F83C7073313F7270022
:102BB00011EF918B99CFB7E70400BC4F1306000AC1
:102BC00089451735FF1F0345653482971345240057
:102BD000D5B59737FF1F938767249C4383C7870327
:102BE0001737FF1F230CF73297000000E78060DBE8
:102BF000F1BF93F7050281CB97000000E78060DA10
